:100000000C94580A0C94890A0C94890A0C94890A55
:100010000C94890A0C94890A0C94890A0C94890A14
:100020000C94890A0C94890A0C94890A0C94890A04
:100030000C94890A0C94890A0C94890A0C948159AD
:100040000C94890A0C94890A0C94890A0C94890AE4
:100050000C94890A0C94890A0C94890A0C94D17323
:100060000C94890A0C94E1750C94B7750C94890A68
:100070000C94890A0C94890A0C94890A0C94890AB4
:100080000C94890A0C94890A0C94890A0C94890AA4
:100090000C942A7B0C949A7A0C94E17A0C94995AD9
:1000A0000C94890A0C94890A0C94890A0C94890A84
:1000B0000C94890A0C94890A0C94890A0C94890A74
:1000C0000C94890A0C94890A0C94890A0C94817501
:1000D0000C9457750C94890A0C94890A0C94890A1B
:1000E0000C94890AB10E7B0F9410CA10CA10AB1081
:1000F000710FCA10CA10CA107B0F7B0F7B0F360F0F
:10010000CD0EDA0E360F360F580F680FDA0E580F75
:10011000360FF40FDE0FDE0FF40FF40F01100C108A
:10012000D50FF40FF40F0B18E6172618261826180B
:1001300026182618261826182618261847143F179A
:1001400064174E175D172618261826182618261825
:1001500026182618FA17541E481E481E541E541EF0
:100160002F1E3C1E3C1E541E541E20263D266D266E
:10017000752678266D264C266D26822685265C26D9
:10018000902693269631853188319031903188318F
:1001900085319031903190318531853185314336CB
:1001A000403640364336433645364536F8354336D5
:1001B0004336C743C743C743C743C443C443CB4382
:1001C000CB43CB43CB43CB43CB43CB43CB43C443C6
:1001D000C443CB43CB43CB43CB43CB43C943C743BC
:1001E0004149A04A70498E49A04AAB49A04ADA4920
:1001F000F849154A484A764A0B4B224B0F4B0F4B96
:10020000224B134B224B174B174B174B174B174BCC
:100210000F4B09640C64FB63FF6305644364106463
:1002200014641A641E64226428642C643064436479
:1002300036643A643E64D864DD64E264EC64F66477
:100240006F650065086510651A6524652E653D6556
:1002500047656F6551655B656565F37CF67C0E7D72
:10026000257D6E7D817DA17D07634236B79BD8A732
:100270001A39685618AEBAAB558C1D3CB7CC5763CB
:10028000BD6DEDFD753EF6177231BF000000803F79
:1002900008000000BE922449123EABAAAA2ABECD95
:1002A000CCCC4C3E00000080BEABAAAAAA3E000007
:1002B0000000BF000000803F0000000000084178FF
:1002C000D3BB4387D1133D190E3CC3BD4282AD2B36
:1002D0003E68EC8276BED98FE1A93E4C80EFFFBE2E
:1002E00001C4FF7F3F00000000000C94A04A0C9462
:1002F0005B650C94D75F0C9408690C9417760C948A
:10030000D7280C94782D0C94F6640C94F37C0C9400
:1003100089680C943F680C94154A0C94F2520C9422
:1003200081680C94242A0C9482200C941F280C942D
:10033000710F0C9408650C940B4B0C94257D0C9458
:10034000E8280C9430640C941A640C9421580C9492
:1003500016690C943E640C941A650C944E170C9418
:1003600068690C94C4430C94DD520C94DD640C94C5
:100370005C280C94D2270C9420260C9426180C94FC
:1003800041490C94E2640C9478260C946D680C94AA
:100390004A280C9484280C947E730C9464170C9453
:1003A00000470C94360F0C947B0F0C948B280C9404
:1003B0005A530C9436640C943F170C9455680C9463
:1003C00093260C948A680C94972D0C940E7E0C94B2
:1003D00001730C942F730C9401100C94541E0C9404
:1003E000FB630C94981F0C94C7430C9422640C94E8
:1003F000C0520C9451650C94FA170C9439580C9413
:1004000090310C946E7D0C940E540C9409640C94F1
:1004100085260C9427580C94CA100C94A17D0C943A
:10042000C55D0C94680F0C94AB100C9405640C948F
:10043000CC6B0C9400650C942B2E0C94B4720C9421
:100440003A640C94B0690C94DE0F0C9494100C94E4
:100450003D260C94B1570C942F2E0C944F580C94AD
:1004600059680C94272E0C944C540C94954C0C9475
:1004700040360C9445360C942C640C9424650C94F2
:100480008B0A0C947E1E0C942C2E0C94F8350C9434
:1004900010650C940F730C94224B0C94EC640C9428
:1004A00043640C9422760C9414640C94F8490C94D4
:1004B000CB430C94E6170C9490260C94F40F0C94F8
:1004C000484A0C9420580C940E7D0C9403750C949F
:1004D000646A0C943D650C9496310C942F1E0C9418
:1004E000C9680C9424580C944A580C946D260C94AA
:1004F00021210C94D50F0C94F4690C948E490C9422
:100500000C640C94ED720C94BB570C9470490C94D1
:10051000174B0C94DA690C9462290C945D2B0C94A3
:10052000402A0C94EF270C942D5D0C94FC460C94FF
:1005300085310C945D680C9415290C9465650C94B8
:10054000985D0C940F4B0C940E7A0C94CD0E0C9479
:1005500031730C942E650C9474680C94B10E0C9449
:1005600082260C9410640C941E640C945D170C94F9
:1005700076680C94B7200C94134B0C9475260C944D
:1005800005290C94D6690C94DE720C94C02D0C9441
:10059000FD690C9444690C94481E0C9419760C94D3
:1005A0006F650C9488310C94C9430C9426200C94EC
:1005B0002E580C9411280C9428640C94DA490C944D
:1005C00047140C9443360C94D8640C94817D0C949D
:1005D000580F0C9447650C943C1E0C9436760C9482
:1005E000FF630C94DA0E0C945C260C940B180C949C
:1005F000F67C0C944C260C94DC790C944D580C949D
:10060000A0680C949D5D0C94C5280C942C5D0C94F2
:10061000AB490C94764A0C940C100C94EB790C9426
:10062000BE5D6364696E6F70737578585B00445289
:10063000590046414E5F4F4E4C5900584F4E0048AE
:10064000414C54003D0050696E3A003D0050696EC7
:100650003A002048616C7465640A003D005265737D
:10066000746F7265643A20003A204E6F2073746F85
:100670007265642076616C756573202D20646566F3
:1006800061756C740A00416C726561647920416324
:10069000746976650A005475726E696E6720584FEA
:1006A0004E0A00416C72656164792048616C746522
:1006B000640A00416C726561647920496E616374FB
:1006C0006976650A00416C726561647920416374E2
:1006D0006976650A005475726E696E6720584F4ED0
:1006E0000A00584F464620736B69707065642E206F
:1006F0005072657620636D643A005475726E65645D
:10070000206F66662066726F6D3A00526573746F73
:100710007265642066726F6D3A00536B6970204792
:1007200072700049676E6F7265642C206368616E39
:100730006E656C20636D643D0029003E003C002026
:100740005061723D280020436D643D002053756662
:10075000663D00205375623D00204974656D3D0083
:1007600052414D3D00476F742049502061646472CE
:100770006573733A00276970205B69705B2C646E47
:10078000735B2C67775B2C7375626E65745D5D5D62
:100790005D27202D20736574207374617469632054
:1007A00049500A004661696C656420746F20636F6C
:1007B0006E6669677572652045746865726E6574EA
:1007C000207573696E6720444843502E20596F7519
:1007D0002063616E20736574206970206D616E7591
:1007E000616C6C7921005374617274696E67206C5E
:1007F000616E00246E6F6465730024666F726D61B4
:10080000740024646174617479706500302D313036
:100810003000696E74656765720068737600636F97
:100820006C6F72004F4E2C4F46462C48414C542C56
:10083000524553542C584F4E2C584F46462C544F2B
:1008400047474C4500656E756D00666C6F617400BE
:10085000322E312E300024686F6D6965007570741A
:10086000696D652C66726565686561700036323742
:10087000376134345F323032302D30352D3039002D
:100880004C696768744875622000246E616D65006C
:100890007265616479002074727920616761696EA4
:1008A00020696E2035207365636F6E647300666126
:1008B000696C65642C2072633D00417761697469DD
:1008C0006E6720666F722072657461696E65642060
:1008D000746F7069637300636F6E6E6563746564D3
:1008E0002061732000202E2E2E0020757365723A31
:1008F000003A000A417474656D7074696E67204D2A
:1009000051545420636F6E6E656374696F6E20740A
:100910006F200024737461746500646973636F6E83
:100920006E6563746564005573696E67204D51543C
:10093000542070617373776F72642066726F6D20DC
:10094000636F6E66696700446576696365204E6112
:100950006D653A00526562696E6420737563636504
:1009600073732E20495020616464726573733A007A
:100970004572726F723A20726562696E64206661B8
:10098000696C0052656E6577656420737563636595
:1009900073732E20495020616464726573733A004A
:1009A0004572726F723A2072656E65776564206673
:1009B00061696C004E6F206C696E6B00416363650A
:1009C0007074696E6720636F6D6D616E64732E2E37
:1009D0002E0A002F00496E3A20002D3E00200023F1
:1009E0000050656E6465642073746174652072657F
:1009F000747269657665643A003D004C4547414331
:100A00005920494E3A00736174006875650066614B
:100A10006E006D6F646500536574436D643A0053F6
:100A20006574466C61673A00436C72466C61673A64
:100A3000002056616C3D002053746F726520007376
:100A40007566666978436F64653A005247420048AC
:100A50005356004C4F57004D454449554D004849A9
:100A6000474800444543524541534500494E43528F
:100A7000454153450044495341424C454400454E8D
:100A800041424C45440046414C5345005452554563
:100A900000584F464600544F47474C450052455377
:100AA000540054787432436D643A002076616C755A
:100AB00065206973200020756E6B6E6F776E0A007B
:100AC00020696E6163746976650A002061637469E8
:100AD00076650A00204772703A0020696E6163747F
:100AE0006976650A00206163746976650A00206989
:100AF0006E76616C6964004D6F64627573206F700F
:100B0000206661696C65640A003D0056432300203D
:100B1000636D643D003D0056435F6865617423006A
:100B20002D3E005075623A2000636D6400434F4FC4
:100B30004C0048454154004155544F002D3E005053
:100B400075623A2000736574002D3E005075623A5C
:100B500020002D3E005075623A2000556E6B6E6F7E
:100B6000776E20636D64200A004F4646004F4E00AA
:100B70005374617475732064656666657265640A92
:100B8000004E6F7420737570706F7274656420729C
:100B9000656720747970650A00293A0028543A0084
:100BA0003D3E00206973200044656C6574696E6782
:100BB00020636F6E662E2052414D207761733A009C
:100BC000556E6C6F636B696E6720636F6E666967E5
:100BD000202E2E2E00536B697070696E672E2E00CA
:100BE0004F4F4D21005D20000A5B003A004D41430C
:100BF0003A002C20002E0053746F72656420455813
:100C0000543A00202D3E2000202D3E2000203A2086
:100C100000494E3A000A282B29464153544C45447A
:100C2000000A282D29535049204C4544000A282BFE
:100C3000294D4F544F5220435452000A282D294128
:100C400043204841494552000A282D29434353383F
:100C5000313120262048444331303830000A282DD5
:100C600029524553544152545F4C414E5F4F4E5FA1
:100C70004D5154545F4552524F5253000A282D296A
:100C80004841524452455345542C207573696E6750
:100C900020736F6674000A282D29434F554E544522
:100CA00052000A282D29444854000A282D294F575C
:100CB000495245000A282B294D4F44425553000AFA
:100CC000282B29444D58000A282B2957697A4E654C
:100CD0007435353030000A282B29445332343832E9
:100CE0002D313030000A282B294672656552616D1E
:100CF000207072696E74696E670064653A61643A67
:100D000062653A65663A66653A6564000A466972E4
:100D10006D77617265204D41432041646472657353
:100D20007320006C617A79686F6D652E7275000AA8
:100D3000436F6E666967207365727665723A000A62
:100D4000282B295741544348444F47003230313112
:100D500030334C0020432B2B2076657273696F6E05
:100D60003A00363237376134345F323032302D302A
:100D7000352D3039000A4C617A79686F6D652E72B5
:100D800075204C6967687448756220636F6E747271
:100D90006F6C6C6572200000002000230026002983
:100DA000002C002F003200000100000301060109A1
:100DB000013D00494E3A005265747279696E6720B0
:100DC00056432074656D7020434D440A004D6F6496
:100DD00062757320706F6C6C696E67206572726FDC
:100DE000723D002D002050492056616C203A004D84
:100DF0006F6462757320706F6C6C696E67206572CA
:100E0000726F723D002D0020464D2056616C203AD5
:100E1000005265747279696E6720564320434D44D1
:100E20000A005265747279696E672064696D6D6538
:100E30007220434D440A004D6F6462757320706FD9
:100E40006C6C696E67206572726F723D002056612E
:100E50006C3A20004D423A20004E6F74207375703A
:100E6000706F727465642072656720747970650AAA
:100E700000496C6C6567616C20617267756D656EA9
:100E800074730A004C6F61646564006C6F61642068
:100E90006661696C6564004E6F2073746F7265647F
:100EA00020636F6E666967004C6F6164696E6720CE
:100EB000436F6E6669672066726F6D2045455052BC
:100EC0004F4D000A72657175657374204D5154540D
:100ED00020436F6E66696700536176656420746FA6
:100EE00020454550524F4D00536176696E6720632F
:100EF0006F6E66696720746F20454550524F4D2EC6
:100F00002E0053617665640A005365742064796E1F
:100F1000616D69632049500A00454550524F4D208C
:100F2000636C65617265640A0050617373776F72F8
:100F30006420757064617465640A00636F756C6425
:100F4000206E6F742070617273653A200055706472
:100F5000617465640A002B002D00485454502F31F1
:100F60002E312025690020485454502F312E310D48
:100F70000A486F73743A2025730D0A4163636570E4
:100F8000743A202A2F2A0D0A436F6E6E65637469C6
:100F90006F6E3A20636C6F73650D0A002573002035
:100FA000000D0A00474554006661696C6564207451
:100FB0006F20636F6E6E6563740A004552524F5224
:100FC0003A205365727665722072657475726E652B
:100FD000642000446F6E652E0A004170706C796960
:100FE0006E672E0A00436F6E6669672070617273C8
:100FF000696E67206661696C65640A00676F7420BA
:10100000436F6E6669670A00436F6E6669672055B5
:1010100052493A20687474703A2F2F002044656654
:1010200061756C7420636F6E666967207365727694
:10103000657220757365643A20006C617A79686F17
:101040006D652E72750020536176656400556E6B78
:101050006E6F776E20636D64003A204E6F2073745C
:101060006F7265642076616C756573202D206465F0
:101070006661756C740A00526573746F7265643AC8
:101080002000466F726365642065786563757469D6
:101090006F6E00696E00735F6F7574006D79686FB5
:1010A0006D6500757074696D65006672656568656B
:1010B00061700024737461747300200020000A5270
:1010C000414D3D00202D746172676574207A6F6E0A
:1010D000652D00204F464600204F4E00204F4646CB
:1010E0000020636D643A00204375723A0020536516
:1010F000743A0020457870697265640A004D6F7417
:101100006F722074696D656F757400000021002492
:101110000027002A002D00300033000101000004E8
:101120000107010A0100002200250028002B002EE3
:10113000003100340002010000050108010B010527
:10114000050505070508080808020202020A0A0840
:101150000804040404010101010101010103030366
:101160000303030303040707070C0C0C0C0C0C0C03
:101170000C0202020206060606060606060B0B0B0A
:101180000B0B0B0B0B010210202008081020401045
:10119000204080020102010804020101020408103B
:1011A0002040808040201008040201800402018059
:1011B0004020100804020108040201010204081082
:1011C000204080010204081020408000000A0B0229
:1011D000090C0D0E080703040100000000000000C8
:1011E00000000000000000000000000000000000FF
:1011F00000000000000000121110000000000000BC
:1012000000000000000000000000000000000000DE
:10121000003E3E3E004E6F204D414320636F6E66A0
:101220006967757265643A20736574206669726DCA
:10123000776172652773204D41430A0043757272CE
:10124000656E74204C414E20636F6E666967286935
:10125000702C646E732C67772C7375626E657429BD
:101260003A000A55736520746865736520636F6D75
:101270006D616E64733A202768656C7027202D209D
:101280007468697320746578740A276D61632064DB
:10129000653A61643A62653A65663A66653A303045
:1012A000272073657420616E642073746F726520EB
:1012B0004D41432D6164647265737320696E2045EE
:1012C0004550524F4D0A276970205B69705B2C6452
:1012D0006E735B2C67775B2C7375626E65745D5DF6
:1012E0005D5D27202D2073657420737461746963BC
:1012F0002049500A277361766527202D2073617677
:101300006520636F6E66696720696E204E56524194
:101310004D0A2767657427205B636F6E66696720D7
:10132000616464725D27202D2067657420636F6E91
:101330006669672066726F6D207072652D636F6ECF
:10134000666967757265642055524C20616E642031
:1013500073746F726520616464720A276C6F6164D4
:1013600027202D206C6F616420636F6E6669672093
:1013700066726F6D204E5652414D0A277077642772
:10138000202D20646566696E65204D51545420708F
:10139000617373776F72640A276B696C6C27202DF9
:1013A0002074657374207761746368646F670A27BB
:1013B000636C65617227202D20636C656172204526
:1013C0004550524F4D0A277265626F6F7427202D6A
:1013D000207265626F6F7420636F6E74726F6C6CD5
:1013E000657200536F6674207265626F6F74696E08
:1013F000672E2E2E00444D58696E20427566666534
:101400007220616C6C6F632065727200496E697442
:1014100020696E2063683A0052414D3D000A6D71AB
:10142000747420000A6D6F6462757320000A696E1F
:101430007075747320000A6974656D7320000A4327
:101440006F6E666967757265643A002C003D0050E6
:10145000696E3A002C003D4C4F5700546865726D20
:101460006F3A00444D58206F757420737461727424
:1014700065642E204368616E6E656C733A2000448B
:101480004D5820696E20737461727465642E204318
:1014900068616E6E656C733A003E3E2000496E7660
:1014A000616C696420636F6D6D616E6400000E7E17
:1014B00011241FBECFEFD1E2DEBFCDBF00E00CBFD5
:1014C00016E0A0E0B2E0EEE6F1E201E00BBF02C000
:1014D00007900D92A236B107D9F72CE0A2E6B6E04C
:1014E00001C01D92AB31B207E1F71AE0C8E5DAE0BE
:1014F00000E006C021970109802FFE010E94818B28
:10150000C735D10780E00807A9F70E94717F0C94C6
:10151000B5900C9400002F923F924F925F926F9281
:101520007F928F929F92AF92BF92CF92DF92EF9273
:10153000FF920F931F93CF93DF93CDB7DEB7AC9796
:101540000FB6F894DEBF0FBECDBF5C012B015BA3CD
:101550004AA33DA32CA3102F1701D9A2C8A2EC2D9A
:10156000FD2D309719F08081811114C0D5011D9691
:101570008C91882321F0C5010D9699A388A321148D
:101580003104A1F4E8A1F9A1309731F4F5012788DD
:10159000308C0CC0EF2851F480818823B9F3CE0140
:1015A00080960E94EB201C01892B81F3C8A0D9A052
:1015B000D5011296ED91FC911397E080F1800E9485
:1015C000105D3B014C0160E677E084EA98E00E9400
:1015D00022742AE0B401A30184EA98E00E945B74BB
:1015E00069E577E084EA98E00E942274B70184EA12
:1015F00098E00E94497563E577E084EA98E00E94EC
:101600002274B60184EA98E00E9449756CE477E0A0
:1016100084EA98E00E9422744AE050E0B10184EA32
:1016200098E00E94EC7466E477E084EA98E00E9417
:1016300022744AE050E0B20184EA98E00E94EC741F
:101640006FE377E084EA98E00E942274F5018281DA
:101650009381892B09F4AEC01B8E1A8E1D8E1C8EB1
:101660001F8E1E8E2CA13DA12115310579F1790126
:101670004E013AE1830E911CC12CD12C8AA19BA171
:10168000C816D9061CF593E0C916D104F9F0D701A4
:101690006D907D907D01F401619271924F016DE337
:1016A00077E084EA98E00E9422744AE050E0B301B7
:1016B00084EA98E00E94EC746BE377E084EA98E0B7
:1016C0000E942274FFEFCF1ADF0AD8CF69E377E0D8
:1016D00084EA98E00E94227484EA98E00E944575AA
:1016E000D5011A968C91873009F458C0E8A0F9A06A
:1016F000E114F10409F462C06DE67BE0C7010E94C9
:10170000C683892B11F40C94A01369E67BE0C70112
:101710000E94C683892B11F40C94A4136FE376E026
:10172000C7010E94C683892B11F40C94A8136BE3A4
:1017300076E0C7010E94C683892B11F40C94AC1388
:1017400062E37BE0C7010E94C683892B11F40C94ED
:10175000B0136DE27BE0C7010E94C683892B11F4B0
:101760000C94B41367E37BE0C7010E94C683892B06
:1017700011F40C94B81362E376E0C7010E94C683AB
:10178000892B11F40C94BC136EE276E0C7010E9421
:10179000C683892B11F40C94C01310C011110EC014
:1017A0006AE177E084EA98E00E94227484EA98E093
:1017B0000E9445758FEF9FEF0C94051460E070E078
:1017C000C5010E949A233C01C5010E9488357C0115
:1017D000B4E04B165104B1F04CF44114510409F437
:1017E000C6C1F3E04F16510491F024C227E042161F
:1017F0005104A9F10CF41EC24AE0441651040CF441
:1018000062C018C2181619060CF447C010C2D501E0
:101810001A968C91873009F40DC2C5010E94782474
:10182000C82ED12C853009F0D1C76BE077E084EA6F
:1018300098E00E9422744AE050E0B60184EA98E001
:101840000E94EC7484EA98E00E944575F501828557
:10185000853009F0ECC10CE0402E512CEBC1D501D4
:101860001A968C91873009F4E5C1C5010E9478244D
:10187000C82ED12C8630A9F46AEF76E084EA98E08D
:101880000E9422744AE050E0B60184EA98E00E9487
:10189000EC7484EA98E00E944575B2E04B2E512C1E
:1018A000C9C162EE76E084EA98E00E9422744AE0C0
:1018B00050E0B60184EA98E00E94EC7484EA98E073
:1018C0000E94457583C7F5010285073009F4B2C14E
:1018D0002AA13BA1232B21F08A8D9B8D892B21F4FA
:1018E00085E090E09B8F8A8F39E04316510439F4EC
:1018F0008A8D9B8D9195819591099B8F8A8FC501CA
:101900000E94802368A77AA78BA79CA7D5011B9666
:101910008D919C911C97009749F0DC01ED91FC9111
:10192000028CF38DE02D19954C0102C0802E912C74
:1019300008A5BAA5BCA3CBA4ECA5EF77DE2E6EEC70
:1019400073E084EA98E00E944975A60160E070E0C7
:101950002AE084EA98E00E945B7467ED73E084EA11
:1019600098E00E9449754AE050E06AA584EA98E050
:101970000E94F3746EED73E084EA98E00E9449756A
:101980004AE050E068A584EA98E00E94F37484EA93
:1019900098E00E94457594012150310939A728A784
:1019A00032E02316310451F024F42114310431F0D3
:1019B00039C0C1010797029760F134C08A8D9B8DB1
:1019C000800F911D8536910514F084E690E09B8F81
:1019D0008A8F8A8D9B8D97FF02C01B8E1A8E8A8CF0
:1019E0009B8C6BED73E084EA98E00E9449754AE0B5
:1019F00050E0B40184EA98E00E94EC7484EA98E034
:101A00000E94457581E090E09BA38AA3412C512C54
:101A100009C0A8A5B9A5129728F0B7E08B169104C4
:101A200009F089C6E8A5F9A5329708F003C1F7E0E7
:101A30002F163104D9F028E02216310419F133E0D1
:101A40002316310409F0F6C08A8D9B8DC80ED91E6D
:101A5000DB8ECA8E8C8D9D8D4CA1840F911D9D8F28
:101A60008C8F8E8D9F8D800F911D17C08A8D9B8DC1
:101A7000C80ED91EDB8ECA8EACA18A2F90E09D8F36
:101A80008C8F09C08A8D9B8DBCA18B0F911D9D8F62
:101A90008C8FDB8ECA8E802F90E09F8F8E8F8A8DE9
:101AA0009B8D8E36914014F01B8E1A8E8A8D9B8DE5
:101AB00097FF04C08DE691E09B8F8A8F8C8D9D8D62
:101AC0008536910524F084E690E09D8F8C8F8C8D77
:101AD0009D8D97FF02C01D8E1C8E8E8D9F8D85362D
:101AE000910524F084E690E09F8F8E8F8E8D9F8DE0
:101AF00097FF02C01F8E1E8E4E8C5F8C8C8C9D8C2F
:101B0000CA8CDB8C62EE73E084EA98E00E9449752F
:101B10004AE050E0B60184EA98E00E94EC7467ED78
:101B200073E084EA98E00E9449754AE050E0B4010D
:101B300084EA98E00E94EC746EED73E084EA98E029
:101B40000E9449754AE050E0B20184EA98E00E94A0
:101B5000EC7484EA98E00E944575A2E02A2E312CAC
:101B6000E3E0F0E0FBA3EAA3412C512C63C0D501D4
:101B70001A969C911A97973009F45CC0EAA1FBA1D0
:101B8000319709F057C01B960D90BC91A02D10976E
:101B900049F0ED91FC911197028CF38DE02DCD0170
:101BA000199502C0892F90E001970297D8F5C501D9
:101BB0000E948023AB01F7E02F163104E1F028E00A
:101BC00022163104B9F52A8D3B8D592F5F778A8F04
:101BD0005B8FB90177277D8F6C8F642F70E07F8FCB
:101BE0006E8F522FBC01C5010E94482383E090E014
:101BF0009BA38AA31FC09A8C8B8D8F779078792FA7
:101C0000782B852F90E09D8F8C8F842F90E09F8F75
:101C10008E8F692DC5010E944823A3E0B0E0BBA3CD
:101C2000AAA308C0C1010797029720F4CFC5442496
:101C30004394512CF501838494848114910409F414
:101C400084C0F5E04F16510469F126E042165104B4
:101C500031F032E04316510409F05EC03FC0EF2876
:101C600009F0AEC565ED76E084EA98E00E94227442
:101C7000D5011B968D919C911C97C8A0D9A0DC0121
:101C8000ED91FC910488F589E02D7101012F9E01F1
:101C9000265E3F4F4AA15BA161E070E019958C017F
:101CA00066E089C51E141F04B4F4C8A0D9A0D401ED
:101CB000ED91FC910488F589E02D7101012F9E01C1
:101CC000265E3F4F4AA15BA162E070E0C401199516
:101CD0008C0165E070C563EB76E074C5C5010E94B8
:101CE00078248530B1F0C8A0D9A0D401ED91FC9141
:101CF0000488F589E02D7101012F9E01265E3F4F7A
:101D00004AA15BA162E070E0C40119958C0162E018
:101D100052C563EA76E056C5C8A0D9A0D401ED91BA
:101D2000FC910488F589E02D7101012F9E01265E4A
:101D30003F4F4AA15BA1B201C40119958C01411426
:101D4000510409F43BC5642D36C5BDE04B16510462
:101D500008F020C2F2018827EE58FF4F8F4F0C94F5
:101D6000818B882483942114310421F01E141F04D4
:101D70000CF0812CC1010797029708F40BC2F50102
:101D8000828590E08A30910508F0A2C0FC01882786
:101D9000E158FF4F8F4F0C94818B8C8D9D8D892B3B
:101DA00049F42AA13BA12330310521F48FE7D50165
:101DB0001A968C93C5010E948023D62EC72E982E8A
:101DC000092FEAA1FBA1E230F105C9F0E330F105EA
:101DD00029F1319759F52A8D3B8DD22E97FF26C0D8
:101DE0009F778A8F9B8F872F90E09D8F8C8F3327D3
:101DF0003F8F2E8F23E030E03BA32AA317C09A8C9D
:101E00000B8D0F779078092BCC8C70E07F8F6E8FC5
:101E1000006883E090E09BA38AA308C09A8C0B8D96
:101E20000F779078092BCC8CDE8C00684D2D5C2DC3
:101E3000692D702FC5010E9448232114310409F037
:101E400042C01E141F0424F4D1103DC062E005C03E
:101E5000EF28C9F5DD20B9F161E0C5010E944D24EC
:101E600060E07BE0C5010E94C3302DC04A8D5B8DD0
:101E7000052E000C660B770BC5010E944823211428
:101E8000310409F51E141F0434F48A8D9B8D892BAF
:101E900061F462E007C0EF2841F48A8D9B8D892BA5
:101EA00021F061E0C5010E944D2460E07BE00DC09F
:101EB0004A8D5B8D052E000C660B770BC5010E94C9
:101EC0004823112329F060E07AE0C5010E94C33065
:101ED000811060C1D5011A968C91873009F02DC40C
:101EE00059C1E114F10409F074C466E976E084EAAA
:101EF00098E00E942274642DC5010E944D241E1496
:101F00001F0444F4112331F060E071E0C5010E9428
:101F1000C33013C4C5010E948023DC01CB01D82E3D
:101F2000C92E9A2E0B2FF5012285233018F421306B
:101F300018F012C0243009F54997A105B1053CF409
:101F4000112329F0E8E2DE2EC12C912C00E04D2D6A
:101F50005C2D692D702F0EC00097A105B10539F0D9
:101F6000F8E1F81720F0112311F078E2D72E4D2D6B
:101F7000592FBD01C5010E9448234D2D5C2D692DAF
:101F8000702F411551056105710509F449C0D5014E
:101F90001A968C9190E08A309105F0F5FC01882723
:101FA000E757FF4F8F4F0C94818B112309F4F2C038
:101FB000C5010E948835892B49F117C40F779A8E85
:101FC0000B8F8C2D90E09D8F8C8F8D2D90E09F8FAF
:101FD0008E8F112329F060E073E0C5010E94C330A9
:101FE00063E0862E912C6EC05B8F4A8F112329F0FF
:101FF00060E073E0C5010E94C33088248394912C73
:1020000061C05B8F4A8F112309F4C4C060E071E0A6
:10201000C5010E94C330E9C3112309F4E6C3F6CF1A
:102020002AE030E040E050E0BA0184EA98E00E9403
:10203000A47468E676E084EA98E00E942274F501D0
:1020400082858530C9F0A0F48150823078F584E62D
:1020500090E09B8F8A8F1D8E1C8E9F8F8E8F0078B5
:1020600044E650E064E6702FC5010E944823B1CFDA
:10207000863059F08830D1F484E190E09B8F8A8FCC
:1020800044E150E060E070E019C084E690E09B8F8E
:102090008A8F44E650E060E070E0C5010E9448236A
:1020A000112309F4AACF60E071E0A4CF84E690E0A8
:1020B0009B8F8A8F44E650E060E070E0C5010E948B
:1020C000482394CF6E01FAE1CF0ED11CE12CF12C04
:1020D000D601ED91FD916D01FDA3ECA36DE576E0D8
:1020E00084EA98E00E9422744AE050E0B70184EA52
:1020F00098E00E94EC746BE576E084EA98E00E9438
:1021000022744AE050E06CA17DA184EA98E00E942C
:10211000EC7484EA98E00E944575FFEFEF1AFF0A1D
:102120008E149F04A9F661C3C5010E9478248530EE
:1021300089F11B8E1A8E1D8E1C8E1F8E1E8E62E0E4
:10214000C5010E944D24112329F160E071E0C50111
:102150000E94C3301FC01E141F04E4F41B8E1A8E8D
:102160001D8E1C8E1F8E1E8EC5010E947824863007
:1021700011F462E001C065E0C5010E944D2460E0F9
:1021800071E0C5010E94C33062E576E084EA98E020
:102190000E942274CC8CDD8CC6010D2C000CAA0B85
:1021A000BB0B8CA39DA3AEA3BFA38E8C9F8C282DAD
:1021B00030E0AFEFB0E00E94728B24E630E040E008
:1021C00050E00E94408B79012F3F310521F01CF037
:1021D000EE24EA94F12CD5011A968C91843009F4FE
:1021E000ABC150F4813099F1C8F0823009F4BEC01F
:1021F000833009F428C2A1C2883009F496C238F4A9
:10220000863009F4DAC1873009F49CC196C289305E
:1022100009F485C28F3709F478C18FC216141704E8
:102220000CF08BC22A8D30E0AFEFB0E00E94728BD1
:1022300024E630E040E050E00E94408BB9012F3F9F
:10224000310519F014F06FEF70E0C30172C1B2E311
:10225000CB16D1040CF067C0161417040CF06CC137
:1022600082E390E08C199D09889DD001899DB00D75
:10227000989DB00D11242FEF30E00E94988B28E834
:1022800033E140E050E00E94408B622FC30103968F
:102290000E946D5A0C8D1D8D2EEF31E0D8010E94E9
:1022A000988B22E330E040E050E00E94408B6901CF
:1022B0007A012E8D30E0AFEFB0E00E94728B24E601
:1022C00030E040E050E00E94408BD9012F3F3105C3
:1022D00019F014F0AFEFB0E096010E94908B2FEF51
:1022E00030E040E050E00E94408B69017A019801A3
:1022F000A5E6BFEF0E94908B22E330E040E050E083
:102300000E94408BDA01C90181509F4FAF4FBF4FF0
:102310008C017601EFEFCE16D104C1F1BCF1EE24B1
:10232000EA94F12C33C0161417040CF005C12CA14B
:102330003DA14EA15FA12253310941095109ABE9E9
:10234000B0E00E945F8B22E330E040E050E00E946A
:10235000408BDA01C9018C599F4FAF4FBF4F8C01A1
:1023600060E0C30103960E946D5A10C01614170452
:102370000CF0E2C02FEF30E0D6010E94988B24E6EB
:1023800030E040E050E00E94408B8901EFE3F1E152
:10239000E491F0E0EE0FFF1FEB5DFE4E859194910E
:1023A000E5E8F1E1E491AA8DBB8D2FEF3FEF0E94AC
:1023B000988B2DE631E040E050E00E94408B4427AE
:1023C0005527AAEFB5E00E945F8BDC01CB01905846
:1023D000AF4FBF4FCD01BB2797FDB095AB2F8E3FC1
:1023E000F1E09F0758F48F3F910510F460E02AC098
:1023F0006EEF962F981B60E08FEF25C08C3F43E077
:10240000940770F48D3FE2E09E0720F462E0680FCD
:102410008FEF04C06CEF681B862F6FEF90E013C046
:102420008A3FF5E09F0761F08B3F44E0940728F472
:1024300094E0980F6FEF80E006C06AEF681B01C060
:1024400060E080E09FEFFF24AFEFEA1AFA0AF8019C
:10245000FF273196009510E09E9FA0019F9F500D91
:102460001124452F5527400F511F8E9F90018F9F9C
:10247000300D1124232F3327200F311F6E9FC001F1
:102480006F9F900D1124892F9927080F191FD701CD
:102490000E94988B4B015C018824AA24BB249801DC
:1024A0000E94988BBB27A92F982F872F882A992ABB
:1024B000AA2ABB2A9A01D7010E94988BDC01CB0182
:1024C0008827AA27BB27BA2FA92F982F88277501FD
:1024D0006401C82AD92AEA2AFB2AB7018827992742
:1024E000C3010E946D5A99278F2D7E2D6D2DC3013A
:1024F00001960E946D5A6C2DC30102960E946D5A7E
:1025000060E080E00E94736418C116141704A4F4FC
:1025100060E0C3010E946D5A60E0C30101960E9411
:102520006D5A60E0C30102960E946D5A6E2DC30180
:1025300003960E946D5A01C16A8D7B8DC5010E9470
:10254000C834FBC0D5011496ED91FC911597808598
:10255000853009F0F2C0A680B78080916E078F5F4A
:1025600080936E07A114B10411F1F50180858430C8
:10257000C1F461857285CE0101960E940740C8A012
:10258000D9A07101012F9E01265E3F4F4AA15BA198
:10259000B201CE0101960E948B0ACE0101960E94E3
:1025A0009740D5011296AD90BC901397DBCF8091E8
:1025B0006E07815080936E07C0C06114710409F4E6
:1025C000BCC077FE06C071946194710801E010E010
:1025D00002C000E010E0F62C61E0862D0E947364DA
:1025E000012B69F0B1E04B16510429F061E0E6E0FF
:1025F0004E16510409F460E0062F10E011C0F1E01E
:102600004F16510451F091E080E026E0421651044B
:1026100009F090E0092F182F02C001E010E0602FB0
:102620008F2D0E9444646DE476E084EA98E00E9475
:1026300022744AE050E0B30184EA98E00E94EC740E
:102640006BE476E05CC06114710409F468C077FE45
:1026500006C071946194710801E010E002C000E0CE
:1026600010E0F62C61E0862D0E9473648091A10039
:10267000887F8093A10080919100887F8093910052
:102680008091A10082608093A1008091910082607E
:1026900080939100AA8DBB8D012B99F0CD01BB0FCA
:1026A000AA0BBB0B9C01AD0124563109410951090C
:1026B000AFEFB0E00E945F8B2CE93FEF4FEF5FEF91
:1026C00008C02FEF30E00E94988B24E630E040E015
:1026D00050E00E94408B8901B9018F2D0E94AF64A8
:1026E00066E476E084EA98E00E9422744AE050E0D2
:1026F000B30184EA98E00E94EC7464E476E084EA32
:1027000098E00E9422744AE050E0B80184EA98E020
:102710000E94EC7484EA98E00E9445750EC0442D36
:102720006A8DC5010E94153408C0442D6A8DC5010B
:102730000E94033302C080E001C081E090E065C0E8
:10274000EE24E394F12C1FC072E0E72EF12C1BC0A5
:1027500065E0E62EF12C17C056E0E52EF12C13C0F3
:102760004AE0E42EF12C0FC03BE0E32EF12C0BC02D
:102770002CE0E22EF12C07C09DE0E92EF12C03C0E5
:102780008EE0E82EF12CC5010E947824082F90E0FD
:102790008E159F0509F412C863E277E084EA98E099
:1027A0000E9422744AE050E0602F84EA98E00E9480
:1027B000F3740C94D60BC5010E944D24C80125C0AA
:1027C00065EC76E084EA98E00E9422748DEF0C9428
:1027D000DB0B66E876E084EA98E00E942274F5015B
:1027E0008285873009F487CBF1CFD5011A968C9179
:1027F000813009F0CFCC8C8D9D8D892B09F0CACC0E
:102800008FE7D5011A968C93C5CCAC960FB6F89489
:10281000DEBF0FBECDBFDF91CF911F910F91FF9013
:10282000EF90DF90CF90BF90AF909F908F907F9070
:102830006F905F904F903F902F9008954F925F92CE
:102840006F927F928F929F92AF92BF92CF92DF92C0
:10285000EF92FF920F931F93CF93DF93CDB7DEB725
:10286000C65AD1400FB6F894DEBF0FBECDBF20913F
:102870006B0730916C07F9013B96E831F10508F0E0
:10288000E5C38827ED56FF4F8F4F0C94818B0E9434
:10289000C5730091840710918507209186073091B8
:1028A0008707061717072807390708F0CFC306EC74
:1028B00013E0CE56DE4F19830883C259D140CC565F
:1028C000DE4F188219821A821B82C459D140CE571A
:1028D000DE4F19830883C258D140CC57DE4F18828F
:1028E00019821A821B82C458D140CE59DE4F1983F7
:1028F0000883C256D140CC59DE4F188219821A8201
:102900001B82C456D140CE5BDE4F19830883C2546C
:10291000D140CC5BDE4F188219821A821B82C454CC
:10292000D14066EE77E084EA98E00E94227484EA5F
:1029300098E00E944575BE016E567E4F86E090E09D
:102940000E9490637C01892B09F467C169EE73E0F2
:1029500084EA98E00E9449751A830983CC56DE4FB9
:1029600088819981AA81BB81C459D1408B839C8382
:10297000AD83BE83CE0101960E94B03DBE016E576D
:102980007E4F8AE090E00E949063892B09F42EC16B
:102990006FEF73E084EA98E00E9449751A83098317
:1029A000CC57DE4F88819981AA81BB81C458D14020
:1029B0008B839C83AD83BE83CE0101960E94B03D84
:1029C000BE016E597E4F8EE090E00E949063892B8D
:1029D00009F4DFC065E074E084EA98E00E9449757C
:1029E0001A830983CC59DE4F88819981AA81BB81E2
:1029F000C456D1408B839C83AD83BE83CE010196A8
:102A00000E94B03DBE016E5B7E4F82E190E00E946D
:102A10009063892B09F477C06AE074E084EA98E057
:102A20000E9449751A830983CC5BDE4F88819981A6
:102A3000AA81BB81C454D1408B839C83AD83BE8368
:102A4000CE0101960E94B03D1A830983CC5BDE4F14
:102A500088819981AA81BB81C454D1408B839C8396
:102A6000AD83BE83CF57DF4F19830883C158D04051
:102A7000CC59DE4F88819981AA81BB81C456D1404F
:102A8000CD57DF4F88839983AA83BB83C358D04037
:102A9000CE53DF4F19830883C25CD040CC57DE4F42
:102AA00088819981AA81BB81C458D140CC53DF4F22
:102AB00088839983AA83BB83C45CD040CE5FDE4FFA
:102AC00019830883C250D140CC56DE4F888199814A
:102AD000AA81BB81C459D140CC5FDE4F88839983E2
:102AE000AA83BB83C450D1409E012F5F3F4FAE01EC
:102AF0004F575F4FBE016E537F4FCE018E5F9E4F8B
:102B00000E94E26E85C01A830983CC59DE4F88810A
:102B10009981AA81BB81C456D1408B839C83AD83AC
:102B2000BE83CF57DF4F19830883C158D040CC579D
:102B3000DE4F88819981AA81BB81C458D140CD578D
:102B4000DF4F88839983AA83BB83C358D040CE5379
:102B5000DF4F19830883C25CD040CC56DE4F88819A
:102B60009981AA81BB81C459D140CC53DF4F88835E
:102B70009983AA83BB83C45CD040AE014F5F5F4F93
:102B8000BE016F577F4FCE018E539F4F0E94BC6294
:102B90003FC01A830983CC57DE4F88819981AA816F
:102BA000BB81C458D1408B839C83AD83BE83CF57F8
:102BB000DF4F19830883C158D040CC56DE4F88813F
:102BC0009981AA81BB81C459D140CD57DF4F8883F9
:102BD0009983AA83BB83C358D040BE016F5F7F4FE8
:102BE000CE018F579F4F0E940E6312C01A83098334
:102BF000CC56DE4F88819981AA81BB81C459D140CE
:102C00008B839C83AD83BE83CE0101960E94596362
:102C100084EA98E00E9445752FC161E174E084EA7E
:102C200098E00E9449750FB6F894A89580916000CD
:102C3000886180936000109260000FBE80915409FB
:102C400090915509009711F00E94678186E690E007
:102C50000E94CF808C0186E6D8011D928A95E9F703
:102C6000C801855B9F4F0E94B26B1093550900937A
:102C7000540980915609809349098091060288235E
:102C800019F00E94712C06C06DE274E084EA98E0AD
:102C90000E94233B26E030E04EE95BE064E089E0FF
:102CA00090E00E94D72C86EC93E09A8389831B8264
:102CB0001C821D821E82CE0103960E94695960E02B
:102CC0008EE290E00E944F2C80FF90C080915409CA
:102CD00090915509FC0116A217A210A611A612A6E2
:102CE00013A614A615A616A617A610AA11AA12AE08
:102CF00013AE14AE15AEFE9640EE5EE260E070E0FC
:102D00004083518362837383349640EA5FE060E0DE
:102D100070E04083518362837383F49724E1DF0181
:102D20001D922A95E9F726E0EEE9FBE0DC01189612
:102D300001900D922A95E1F7FC01E65BFF4F1082AE
:102D40000E942B717C01019709F050C060915409D9
:102D500070915509625F7F4FCE0101960E944B75BD
:102D6000CE0103960E9469596091540970915509EA
:102D7000665E7F4FCE0101960E944B75CE01039691
:102D80000E94795960915409709155096A5E7F4F8C
:102D9000CE0101960E944B75CE0103960E94715997
:102DA00060915409709155096E5D7F4FCE01019677
:102DB0000E944B758B819C81AD81BE8180934C09B3
:102DC00090934D09A0934E09B0934F09E091540997
:102DD000F091550982899389909351098093500904
:102DE00084899589909353098093520999E288E1E7
:102DF0000FB6F894A895809360000FBE9093600082
:102E0000A895EF2819F564EA77E084EA98E00E9433
:102E1000227465E777E084EA98E00E94227486EFE6
:102E20009FEF90936C0780936B070E94C573DC0142
:102E3000CB01805A9541AF4FBF4F80938407909349
:102E40008507A0938607B093870700C165E677E002
:102E500084EA98E00E94227486EC93E09A83898346
:102E60001B821C821D821E82CE0103960E94063E9A
:102E7000CE0101960E94B03D81E090E0E3C08091D8
:102E80006E07811122C78091620681111AC060E02D
:102E900070E080E090E00E945F55D4C00E94C5734E
:102EA000009184071091850720918607309187074C
:102EB0000617170728073907D0F10E94C06C811147
:102EC000C5C082E090E0BEC0A895CE55DE4F188206
:102ED000C25AD140FE01EE56FE4F119211928EE081
:102EE000DF011D928A95E9F70091B60B1091B70B9F
:102EF0000115110529F0C8010E948A3F811173C292
:102F00000E94C06C8111A2C00091B60B1091B70B4A
:102F10000115110509F49AC0C8010E948A3FE82EE4
:102F2000F12CB2E0EB16F1040CF077C28FC020E078
:102F300030E043E050E061E48E010F5F1F4FC801B5
:102F40000E94225C6AE374E0C8010E94C08FF8010D
:102F500001900020E9F7CF01801B910B0896813882
:102F6000910538F50E94C06C882319F18091DD0924
:102F70009091DE09019611F481E090E09093DE09D2
:102F80008093DD098091DD099091DE0990936209BB
:102F90008093630947E050E06DE579E0C8010E9445
:102FA000376CAC01455051096DE579E082EA0E9429
:102FB000576C84E090E090936C0780936B076CEB08
:102FC00079E084EA98E00E94227440C00E94C573B0
:102FD000009184071091850720918607309187071B
:102FE000061717072807390788F510926C07109203
:102FF0006B072CC00E94C573009184071091850750
:103000002091860730918707061717072807390789
:1030100008F457CF1BC00E94FC54892B09F051CFF4
:103020000E94C573DC01CB0188579C4EAF4FBF4F48
:103030008093840790938507A0938607B0938707B2
:1030400086EF9FEF90936C0780936B070FB6F89411
:10305000A895809160008861809360001092600064
:103060000FBE80916B0790916C07181619060CF033
:10307000ABC160E08EE290E00E944F2C80FF51C116
:1030800000915409109155090115110509F49CC1CD
:103090000E94C5734B015C01F80182AD93ADA4ADF4
:1030A000B5AD98012A5B3F4F7901892B8A2B8B2B79
:1030B00009F4AEC0F90180819181A281B381A5019B
:1030C0009401281B390B4A0B5B0BCA01B90157FD50
:1030D00064C028EE33E040E050E00E94408BCD55C4
:1030E000DE4F688379838A839B83C35AD14024014E
:1030F000350188EE480E83E0581E611C711CCD55C9
:10310000DE4F88819981AA81BB81C35AD140481A78
:10311000590A6A0A7B0AD7014D925D926D927C92A0
:103120001397BA01A9014F5F5F4F6F4F7F4FF801AF
:1031300082A993A9A4A9B5A96A017B01CC0CDD1CC5
:10314000EE1CFF1C8C159D05AE05BF052CF412AAC4
:1031500013AA14AA15AA09C0841B950BA60BB70BBA
:10316000F80182AB93ABA4ABB5ABF80186A997A9E4
:10317000A0ADB1AD8C159D05AE05BF052CF416AA0A
:1031800017AA10AE11AE09C0841B950BA60BB70B86
:10319000F80186AB97ABA0AFB1AF6801FAE4CF0EF0
:1031A000D11CD6018C91833099F4F80182A993A99E
:1031B000A4A9B5A9181619061A061B064CF084E036
:1031C000D6018C93C8010E942B7101967C0102C02C
:1031D000E12CF12CF6018081833011F0811125C0A2
:1031E000F80186A997A9A0ADB1AD181619061A065F
:1031F0001B06DCF0D6011C9284E13E96DF011D9295
:103200008A95E9F7C8010E942B7103967C010DC0D5
:10321000D501C40188519C4FAF4FBF4FF901808346
:103220009183A283B383E12CF12CD801DA968D929D
:103230009D92AD92BC92DD97B2E0EB16F10429F0BD
:10324000E4E0EE16F10409F050C060915409709169
:103250005509625F7F4FCE0101960E944B75CE01EA
:1032600003960E9469596091540970915509665EF0
:103270007F4FCE0101960E944B75CE0103960E94AE
:10328000795960915409709155096A5E7F4FCE015A
:1032900001960E944B75CE0103960E947159609170
:1032A0005409709155096E5D7F4FCE0101960E94C1
:1032B0004B758B819C81AD81BE8180934C0990932D
:1032C0004D09A0934E09B0934F09E0915409F09134
:1032D0005509828993899093510980935009848973
:1032E00095899093530980935209F3E0EF16F10406
:1032F00009F451C064F431E0E316F10451F142E005
:10330000E416F10409F060C063E879E049C054E0D4
:10331000E516F10409F442C085E0E816F10409F06D
:1033200053C064EB79E084EA98E00E94227484EA56
:1033300098E00E9445750E94C06C81110E940E3E6B
:103340000E94C573DC01CB01805D9A48AF4FBF4F2F
:1033500013C060EA79E084EA98E00E9422740E9437
:10336000C06C81110E940E3E0E94C573DC01CB012E
:1033700088519C4FAF4FBF4F809384079093850730
:10338000A0938607B093870786EF9FEF90936C0713
:1033900080936B0719C060E779E0DDCF64E579E0E1
:1033A00084EA98E00E94227486EC93E09A838983F1
:1033B0001B821C821D821E82CE0103960E94063E45
:1033C000CE0101960E94B03D99E288E10FB6F894D3
:1033D000A895809360000FBE9093600020916B07CA
:1033E00030916C0772C460E070E0C8010E9493796C
:1033F0008C0190938B0780938A0767E479E084EAD5
:1034000098E00E942274B80184EA98E00E9449750D
:1034100084EA98E00E94457573CD61E070E0C801D0
:103420000E9493793C0192E0E916F10491F062E088
:10343000C8010E94263FFC0181849284F3E0EF16CC
:10344000F10459F063E070E0C8010E9493798C01A7
:1034500007C08BE5882E87E0982E8E010E551E4FF3
:1034600040E150E0BE016E567E4F86E390E00E9440
:10347000B854892B51F425E0E216F1040CF038C35E
:10348000AE014E565E4F7A0104C0CE018E569E4F5D
:103490007C017092F1096092F0099092F309809298
:1034A000F2098FE29EE29093E9098093E8095E01B8
:1034B0009EE7A91A9EEFB90A40E150E06AE179E07F
:1034C000C5010E94F4836E01AEE9CA1AAEEFDA0AB2
:1034D00020E030E041E050E060E2C6010E94225C62
:1034E00040E250E063E179E0C6010E94D68363EFD9
:1034F00078E084EA98E00E942274B30184EA98E0BC
:103500000E94497561EF78E084EA98E00E94227495
:103510004AE050E0B40184EA98E00E94EC746AEE5C
:1035200078E084EA98E00E942274B80184EA98E086
:103530000E94497565EE78E084EA98E00E94227462
:10354000F8018081811104C0E12CF12C00E010E031
:1035500080908A0790908B070E94C06C81114DC1AA
:1035600080915B0990915C09DC01ED91FC910688EA
:10357000F789E02D19958823B1F081E090E09093D0
:10358000DE098093DD0987E0E4E1F2E0DE011196D7
:1035900001900D928A95E1F7FE013196A2E6B9E01D
:1035A000CE01089637C06091F0097091F1098091C1
:1035B0005B0990915C094091F2095091F309DC019B
:1035C000ED91FC916115710521F00088F189E02DE4
:1035D00016C00684F785E02D26EC33E03A83298374
:1035E0004090EC095090ED096090EE097090EF0961
:1035F0004B825C826D827E82BE016F5F7F4F199528
:10360000019709F4BACF8EEF9FEF9093F70980935B
:10361000F6097EC221912D93E817F907D9F7011514
:10362000110529F0E114F10421F086EF03C086E3CF
:1036300001C086EB8093690910926A098FE080933C
:103640006B09F40101900020E9F7CF01881999096D
:1036500040968138910508F0C4C04FE050E06DE518
:1036600079E0C4010E94376CF60101900020E9F76F
:103670003197EC19FD09E80FF91F3296E138F10591
:1036800008F0AFC0AC016DE579E0C6010E94376C6F
:10369000F50101900020E9F73197EA19FB09E80FDD
:1036A000F91F3296E138F10508F09BC0AC016DE5D9
:1036B00079E0C5010E94376C0115110579F1F80117
:1036C00001900020E9F73197E01BF10B9C012E5F80
:1036D0003F4FE20FF31FE138F10508F082C0AC0163
:1036E0006DE579E0C8010E94376CE114F104B1F096
:1036F000F70101900020E9F73197EE19FF099C01CD
:103700002E5F3F4FE20FF31FE138F10508F069C06B
:10371000AC016DE579E0C7010E94376CAC01455002
:1037200051096DE579E080E10E94576C0E94C573F4
:103730006093DF097093E0098093E1099093E209B7
:103740006093E3097093E4098093E5099093E60997
:1037500080915B0990915C09DC01ED91FC91008402
:10376000F185E02D1995892BC1F40E94C573009154
:10377000E3091091E4092091E5093091E609DC01A3
:10378000CB01801B910BA20BB30B88399A43A10587
:10379000B105F0F28CEF9FEF20C0CE018F579F4F05
:1037A0000E94353B6430710581059105D1F480910B
:1037B0006009811111C00E94C5736093E309709381
:1037C000E4098093E5099093E6091092E7091092C5
:1037D000F7091092F60911C090E09093F7098093D1
:1037E000F60980915B0990915C09DC01ED91FC91F7
:1037F0000488F589E02D19958BC100918A071091F5
:103800008B0767ED78E084EA98E00E942274B801A3
:1038100084EA98E00E94497584EA98E00E94457520
:1038200081E08093620620E030E043E050E061E414
:10383000CE018F579F4F0E94225C6AE374E0CE0155
:103840008F579F4F0E94C08FCE018F579F4F0E946E
:10385000A26E20E030E042E050E061E4CE018F57FC
:103860009F4F0E94225C6EE374E0CE018F579F4F02
:103870000E94C08FBE016F577F4F84EA98E00E947C
:10388000233BCE018F579F4F0E94A26E20E030E075
:1038900041E050E061E4CE018F579F4F0E94225CCF
:1038A0006EE374E0CE018F579F4F0E94C08FBE0120
:1038B0006F577F4F84EA98E00E94233BCE018F57D9
:1038C0009F4F0E94A26EFE01EE5FFE4F1192119279
:1038D0001EE3DF01212F1D922A95E9F71A82198232
:1038E000FE0133968EE7DF011D928A95E9F720E00D
:1038F00030E041E050E060E4CE018E5F9E4F0E94D8
:10390000225C40E450E063E179E0CE018E5F9E4F9F
:103910000E94D68340E850E060E978E0CE0101964D
:103920000E94F483BE016F5F7F4FCE018E5F9E4F7A
:103930000E94FA3E20E030E041E050E060E4CE0139
:103940008E5F9E4F0E94225C40E450E06AE878E07F
:10395000CE018E5F9E4F0E94D68340E850E060E823
:1039600078E0CE0101960E94F48340E850E06DE6D5
:1039700078E0CE0101960E94D683BE016F5F7F4F33
:10398000CE018E5F9E4F0E94FA3E20E030E041E083
:1039900050E060E4CE018E5F9E4F0E94225C40E4C6
:1039A00050E063EB70E1CE018E5F9E4F0E94D683A4
:1039B00040E850E06DE578E0CE0101960E94F48386
:1039C000BE016F5F7F4FCE018E5F9E4F0E94FA3E19
:1039D00020E030E041E050E060E4CE018E5F9E4F99
:1039E0000E94225C40E450E066E578E0CE018E5F04
:1039F0009E4F0E94D68340E850E060E578E0CE011B
:103A000001960E94F483BE016F5F7F4FCE018E5FEF
:103A10009E4F0E94FA3E80916E078F5F80936E07E3
:103A2000A0916F07B0917007109709F443C080917F
:103A30001B0290911C02AE014E5B5E4FFA01819316
:103A400091932EE111922A95E9F79E012E533F4F53
:103A5000F9018193919311921A95E9F716960D91B8
:103A60001C911797E0906F07F0907007E114F10434
:103A700071F00115110559F0D80118968C91853017
:103A8000A9F7C8010E948A3F882381F36FC020E014
:103A900030E041E050E060E4CE018E5F9E4F0E9436
:103AA000225C40E450E063EF77E0CE018E5F9E4FF2
:103AB0000E94D68380916E07815080936E0783E0C9
:103AC00090E090936C0780936B070E94C573DC01B4
:103AD000CB0188579C4EAF4FBF4F80938407909384
:103AE0008507A0938607B09387076AEB78E069CAD9
:103AF00064E070E08091B60B9091B70B0E949379CF
:103B00007C0167E279E084EA98E00E942274C1CCEB
:103B10000091F6091091F7096EEA78E084EA98E0DE
:103B20000E9422744AE050E0B80184EA98E00E94C2
:103B3000EC7466E978E084EA98E00E94227484EAF2
:103B400098E00E9445750E94C573DC01CB0188573F
:103B50009C4EAF4FBF4F8093840790938507A093EF
:103B60008607B09387078CE090E06CCA60E0C801DC
:103B70000E94263FFC0181859285A385B4858A3009
:103B8000910508F463C020E030E041E050E060E4DB
:103B9000CE018E5F9E4F0E94225CF8016081718190
:103BA00040E450E0CE018E5F9E4F0E94E68F60E4BD
:103BB00074E0CE018E5F9E4F0E94C08F40E450E0C3
:103BC00062E078E0CE018E5F9E4F0E94D683BE01F8
:103BD0006E5B7E4FCE018E5F9E4F0E94FA3ECE53AB
:103BE000DF4F8881C25CD040882361F120E030E063
:103BF00041E050E060E4CE018E5F9E4F0E94225C67
:103C0000D8016D917C9140E450E0CE018E5F9E4FD3
:103C10000E94E68F60E474E0CE018E5F9E4F0E94AA
:103C2000C08F40E450E06AEF77E0CE018E5F9E4F98
:103C30000E94D683BE016E537F4FCE018E5F9E4F92
:103C40000E94FA3EF801028113810CCFFC0140E290
:103C500050E08827E555FF4F8F4F0C94818B6AE425
:103C600078E0CE018E5B9E4F0E94F483CE53DF4FEF
:103C70001882C25CD04087CF65E478E0CE018E5BCD
:103C80009E4F0E94F48340E450E064E278E017C065
:103C90006EE178E0CE018E5B9E4F0E94F48340E49B
:103CA00050E06AE178E00BC062E178E0CE018E5B23
:103CB0009E4F0E94F48340E450E06CE078E0CE0137
:103CC0008E539F4F0E94F4835ECFC901CA55DE4FC9
:103CD0000FB6F894DEBF0FBECDBFDF91CF911F911D
:103CE0000F91FF90EF90DF90CF90BF90AF909F909B
:103CF0008F907F906F905F904F90089584E690E052
:103D00000895CF93DF93009709F455C0FC012081FB
:103D1000222309F450C0EC0165E47BE00E94C683D5
:103D2000892BA1F169E27BE0CE010E94C683892B39
:103D300081F162E17AE0CE010E94C683892B61F1B4
:103D40006FE47AE0CE010E94C683892B41F16BE4D7
:103D50007AE0CE010E94C683892B21F16EE07AE0E1
:103D6000CE010E94C683892B01F16AE07AE0CE0180
:103D70000E94C683892BE1F066E07AE0CE010E94C2
:103D8000C683892BC1F488E090E017C082E090E000
:103D900014C081E090E011C086E090E00EC083E0A6
:103DA00090E00BC084E090E008C085E090E005C0A2
:103DB00087E090E002C080E090E0DF91CF9108952D
:103DC0008F929F92AF92BF92CF92DF92EF92FF922B
:103DD0000F931F93CF93DF93E0916F07F0917007DC
:103DE000309709F465C0812EF02E932EC22EA52E99
:103DF000D42EB72EE62EBC01CF010E940B3FEC0162
:103E0000892B09F458C08885853009F054C060E0DA
:103E1000CE010E94263F8C0161E0CE010E94263F28
:103E2000FC01C185D285D80119962D913C911A9734
:103E30002130310569F02CF4232BE9F56F2DCE01EB
:103E400018C02230310549F027303105A9F033C0C0
:103E50006F2DCE0103960E946D5A6E2DCE010E94E9
:103E60006D5A6D2DCE0101960E946D5A6C2DCE01BA
:103E700002960E946D5A1FC0892BE9F0808585301B
:103E8000D1F4C681D7812097B1F08885843061F460
:103E90000F2D182D2C2D392D4D2D5A2D6E2D7B2D9E
:103EA00089859A850E94E01E0A80DB81C02DEBCFB8
:103EB00080E090E002C081E090E0DF91CF911F911F
:103EC0000F91FF90EF90DF90CF90BF90AF909F90B9
:103ED0008F900895CF92DF92EF92FF920F931F93EE
:103EE000CF93DF93E091BA0BF091BB0B3097B9F011
:103EF00090859530A1F469017A01EB01682FCF011B
:103F00000E94263FFC012085243049F4818592855A
:103F1000009729F09601A701BE010E94E01EDF91E3
:103F2000CF911F910F91FF90EF90DF90CF90089568
:103F3000AF92BF92CF92DF92EF92FF920F931F93B7
:103F4000CF93DF938091B30B9091B40B892B09F43D
:103F500072C0E1E0F0E0C0E0D0E0CC24C394D12C0A
:103F6000B6010C2E02C0660F771F0A94E2F740914B
:103F70006706509168067F0184E0E80EF11CCF01CE
:103F8000B12C9C01A0910802B0910902A817B907B1
:103F900020F42091080230910902A091CD0BB0913C
:103FA000CE0BA20FB31FAC90A091B30BB091B40B8A
:103FB0009C0121503109A20FB31F0A2D10E02C9152
:103FC00030E00217130729F0462B572BAC92BB2485
:103FD000B3940196E816F906A1F65093680640934B
:103FE0006706BB2011F18091B30B9091B40BE80FE1
:103FF000F91F028110E0218130E0408150E03197CB
:10400000608170E0CE010E946A1F0E94C573DC01CE
:10401000CB01845D9E4FAF4FBF4F8093630690935B
:104020006406A0936506B09366062196F701C43036
:10403000D10509F095CFDF91CF911F910F91FF909E
:10404000EF90DF90CF90BF90AF900895CF92DF9226
:10405000EF92FF920F931F93CF93DF93CDB7DEB70D
:10406000C054D1090FB6F894DEBF0FBECDBF6115A5
:10407000710519F480E090E035C069017A018B0187
:1040800040E450E0CE0101960E9404906FE270E09F
:10409000CE0101960E94CB8F892B41F4980143E019
:1040A00050E060E4CE0101960E94225C40E450E0C2
:1040B000B601CE0101960E94E68F0E94C06C882353
:1040C000C9F280916B0790916C07049799F68091E3
:1040D0006D078111CFCFB701CE0101960E94FA3E44
:1040E00081E090E0C05CDF4F0FB6F894DEBF0FBEFA
:1040F000CDBFDF91CF911F910F91FF90EF90DF9097
:10410000CF900895CF92DF92EF92FF920F931F937B
:10411000CF93DF93CDB7DEB760970FB6F894DEBFCD
:104120000FBECDBF7C016B01CA01B901AE014F5F6B
:104130005F4F0E94B95CD701ED91FC910288F38931
:10414000E02D9801AE014F5F5F4FB601C701199591
:1041500060960FB6F894DEBF0FBECDBFDF91CF9152
:104160001F910F91FF90EF90DF90CF900895CF9225
:10417000DF92EF92FF920F931F93CF93DF93CDB710
:10418000DEB760970FB6F894DEBF0FBECDBF7C01DF
:104190006B01BA01A901CE0101960E94C75BD7014C
:1041A000ED91FC910288F389E02D9801AE014F5FFB
:1041B0005F4FB601C701199560960FB6F894DEBF40
:1041C0000FBECDBFDF91CF911F910F91FF90EF9068
:1041D000DF90CF9008950F931F93CF93DF938C01BF
:1041E000FC01C081D1816FE270E0CE010E9413908A
:1041F0000097C1F0FC011192CF010E94811EEC01D9
:104200006FE37AE084EA98E00E9422744AE050E08A
:10421000BE0184EA98E00E94EC7484EA98E00E946F
:10422000457509C0CE010E94811EEC01892B19F051
:10423000F80111821082CE01DF91CF911F910F9171
:1042400008952F923F924F925F926F927F928F923A
:104250009F92AF92BF92CF92DF92EF92FF920F9315
:104260001F93CF93DF93CDB7DEB72B970FB6F8949C
:10427000DEBF0FBECDBF4C016B01042F38872F83EB
:10428000672B09F4DDC1F901309719F080818111A4
:1042900009C0D4011D968C91882321F0C4010D968C
:1042A00098878F83EF81F885309721F4F401E788B0
:1042B000F08C0AC080818823C9F3CE0107960E9442
:1042C000EB207C01892B91F35601D5018C91882339
:1042D00049F0082E000C990B0E946C8FF501819318
:1042E0005F01F3CFD6011C911D3209F4CBC080EDE4
:1042F000810F8A3008F4C6C0153209F4F6C06DE6A5
:104300007BE0C6010E94C683892B09F4E6C069E6FA
:104310007BE0C6010E94C683892B09F4E2C06DE9E7
:104320007AE0C6010E94C683892B09F4AEC066E913
:104330007AE0C6010E94C683892B09F4AAC06FE304
:1043400076E0C6010E94C683892B09F4A6C06BE300
:1043500076E0C6010E94C683892B09F4A2C061E9F8
:104360007AE0C6010E94C683892B09F49EC062E3ED
:104370007BE0C6010E94C683892B09F49AC06DE2D6
:104380007BE0C6010E94C683892B09F496C067E3CF
:104390007BE0C6010E94C683892B09F492C062E3C8
:1043A00076E0C6010E94C683892B09F48EC06EE2B6
:1043B00076E0C6010E94C683892B09F48AC06CE8A6
:1043C0007AE0C6010E94C683892B09F486C066E89C
:1043D0007AE0C6010E94C683892B09F482C06EE789
:1043E0007AE0C6010E94C683892B09F476C065E78E
:1043F0007AE0C6010E94C683892B09F472C06CE67C
:104400007AE0C6010E94C683892B09F46EC063E678
:104410007AE0C6010E94C683892B09F46AC06EE562
:104420007AE0C6010E94C683892B09F466C067E55D
:104430007AE0C6010E94C683892B09F462C063E555
:104440007AE0C6010E94C683892B09F45EC01B373F
:1044500009F45FC0133209F461C043E050E06FE437
:104460007AE0C6010E94E683892B09F45CC043E030
:1044700050E06BE47AE0C6010E94E683892B09F0E4
:1044800057C04CC0A12CB12C56C0E3E0AE2EB12CCD
:1044900052C074E0A72EB12C4EC065E0A62EB12C00
:1044A0004AC056E0A52EB12C46C047E0A42EB12C40
:1044B00042C03AE0A32EB12C3EC02BE0A22EB12C7C
:1044C0003AC09CE0A92EB12C36C08DE0A82EB12CAC
:1044D00032C01EE0A12EB12C2EC0AA24A394B12C70
:1044E0002AC0A2E0AA2EB12C26C0F8E0AF2EB12C33
:1044F00022C0E9E0AE2EB12C1EC070E1A72EB12C77
:104500001AC061E1A62EB12C16C052E1A52EB12C25
:1045100012C04EEFA42EBB24BA940DC03DEFA32EC3
:10452000BB24BA9408C02CEFA22EBB24BA9403C0BB
:10453000AA24AA94BA2C62EA7AE084EA98E00E945B
:1045400022744AE050E0B50184EA98E00E94EC74DD
:1045500084EA98E00E944575BFEFAB16BB0609F0F0
:1045600064F4EEEFAE16EFEFBE060CF069C0FCEFA0
:10457000AF16FFEFBF0649F053C0A114B10429F0F4
:10458000C5010897029718F04BC0A12CB12CCE01A1
:1045900001961C01612C712C8A873B862301AFEFA9
:1045A0004A1A5A0A3201F60180818823D1F06F013C
:1045B0008191882329F08D3219F080538A30B8F721
:1045C000C6010E949F83182F99876CE270E0C60194
:1045D0000E94CB8F6C01892B39F0FFEFCF1ADF0AD5
:1045E00003C080E090E002C0812F9985D1018D93B6
:1045F0009D931D01C114D10439F093E04916510473
:1046000069F683E0682E712CCF80D884D401ED91B7
:10461000FC910190F081E02D2A853B85A3010CC01F
:10462000CF80D884D401ED91FC910190F081E02DF0
:1046300020E030E040E050E0B501C401199502C02F
:1046400080E090E02B960FB6F894DEBF0FBECDBF92
:10465000DF91CF911F910F91FF90EF90DF90CF905E
:10466000BF90AF909F908F907F906F905F904F9092
:104670003F902F900895DC011296ED91FC911397D5
:10468000309721F081E09085953009F080E0089521
:10469000CF92DF92EF92FF92CF93DF93DC011696D9
:1046A000ED91FC911797309721F12085223009F583
:1046B0006A017B01EC0167E37AE084EA98E00E94FA
:1046C000227461E37AE084EA98E00E9422742AE08E
:1046D00030E0B701A60184EA98E00E94A47484EA5D
:1046E00098E00E944575EE81FF81C186D286E386FF
:1046F000F486DF91CF91FF90EF90DF90CF900895F7
:10470000FC0186819781009789F0FC012085223089
:1047100041F0253059F460E00E94263F009731F0C7
:10472000FC016185728583859485089560E070E061
:10473000CB0108950F931F93CF93DF93FC01C481A6
:10474000D581209791F08885823029F4672B69F410
:1047500089859A8514C0853041F48B01CE010E9471
:104760008A3F90E0081719071CF080E090E007C02E
:10477000602FCE010E94263FFC0181859285DF914A
:10478000CF911F910F9108950F931F93CF93DF93B4
:10479000EB0163E0FC01828193810E94263F009738
:1047A00041F1AE01409550954F6F60E070E0FC0123
:1047B0000185128523853485402351236223732389
:1047C000418752876387748768E27AE084EA98E0D9
:1047D0000E9422744AE050E0BE0184EA98E00E9400
:1047E000EC7484EA98E0DF91CF911F910F910C94C3
:1047F0004575DF91CF911F910F9108950F931F93EE
:10480000CF93DF93EB0163E0FC01828193810E94EF
:10481000263F009731F1AE01442760E070E0FC01D3
:104820000185128523853485402B512B622B732BF8
:1048300041875287638774876FE17AE084EA98E062
:104840000E9422744AE050E0BE0184EA98E00E948F
:10485000EC7484EA98E0DF91CF911F910F910C9452
:104860004575DF91CF911F910F910895CF93DF93FD
:10487000EB0163E0FC01828193810E94263F009757
:1048800039F0FC018185928588278C239D2302C005
:1048900080E090E0DF91CF910895CF93C62F63E041
:1048A000FC01828193810E94263F0097F9F0FC0170
:1048B00041855285638574854427662777274C2B6D
:1048C000418752876387748767E17AE084EA98E0DA
:1048D0000E9422744AE050E06C2F84EA98E00E9423
:1048E000F37484EA98E0CF910C944575CF910895C4
:1048F00063E0FC01828193810E94263F009719F0BA
:10490000FC01818508958FEF0895CF93DF93EC012B
:10491000FB012481358140815181628173810E9434
:10492000A474CE01DF91CF9108956F927F928F9200
:104930009F92AF92BF92CF92DF92EF92FF920F932E
:104940001F93CF93DF93CDB7DEB7C054D1090FB615
:10495000F894DEBF0FBECDBF3C014B01FC01E080EF
:10496000F18062E474E0C7010E940B3F5C0167E4E0
:1049700074E0C7010E940B3F6C01A114B10419F44B
:10498000892B09F4D3C06CE474E0C7010E940B3F8B
:104990008C0161E574E0C7010E940B3F7C01F301CB
:1049A00073806BEF79E084EA98E00E9422744AE019
:1049B00050E0672D84EA98E00E94F37469EF79E093
:1049C00084EA98E00E9422744AE050E0B40184EA4C
:1049D00098E00E94EC7484EA98E00E944575C11446
:1049E000D104D1F1F60180858430B1F561857285FD
:1049F00040E450E0CE0101960E9404900E94C06CF9
:104A0000882351F180916D07811126C06FE270E01B
:104A1000CE0101960E94CB8F892B51F4F60121859E
:104A2000328543E050E060E4CE0101960E94225CB2
:104A30008114910409F469C00115110509F462C0DB
:104A4000F8018085843009F05DC0F80161857285C8
:104A5000FB018081811165C0A114B10409F466C015
:104A6000F5018085843009F061C061857285CE01D1
:104A700001960E940740CE0101960E943B238823A5
:104A8000E1F18928A9F00115110521F0F8018085CF
:104A9000843061F0C12CD12CE12CF12C01E020E01C
:104AA00030E040E050E061E070E014C0F80118C070
:104AB000E114F10421F0F7018085843081F0C12CEC
:104AC000D12CE12CF12C01E020E030E040E050E07E
:104AD00062E070E0CE0101960E948B0A0EC0F701E1
:104AE00061857285FB018081882339F020E030E008
:104AF00041E0CE0101960E942121CE0101960E9443
:104B0000974014C066E574E00CC0E114F10421F094
:104B1000F7018085843019F469E574E002C0F7017B
:104B200095CFCE0101960E94FA3E96CFC05CDF4F32
:104B30000FB6F894DEBF0FBECDBFDF91CF911F91AE
:104B40000F91FF90EF90DF90CF90BF90AF909F902C
:104B50008F907F906F900895CF92DF92FF920F9386
:104B60001F93CF93DF93EC01F62E8A018881998100
:104B7000892B09F412C1EC81FD81309709F40DC134
:104B800080819FEF691318C084FF05C14330510530
:104B900009F401C1F180F2948FE0F82261EE79E02E
:104BA00084EA98E00E9422744AE050E06F2D84EA83
:104BB00098E00E94F37402C084FDEFC0EC81FD8197
:104BC00081818F70D82EF81661F1CB806FED79E07E
:104BD00084EA98E00E9422744AE050E06C2D84EA56
:104BE00098E00E94F3746DED79E084EA98E00E9409
:104BF00022744AE050E06D2D84EA98E00E94F3743C
:104C00006AED79E084EA98E00E9422744AE050E07C
:104C10006F2D84EA98E00E94F37484EA98E00E9481
:104C200045758F2D90E08D30910508F089C0FC010D
:104C3000CC80DD808827EB54FF4F8F4F0C94818B05
:104C4000F6019181292F2F70253009F479C08881D0
:104C50009981263028F4223069F46EE574E04CC066
:104C6000273029F02A3031F464E674E060C06DE545
:104C700074E04FC061E574E034C06CE474E0888196
:104C800099810E940B3FF6012081422F4170322F03
:104C9000309530FB20F91FC06BE674E08881998164
:104CA0000E940B3FF601208121FB442740F931E0AF
:104CB000342730FB21F90FC061E774E088819981C6
:104CC0000E940B3FF601208122FB442740F931E08E
:104CD000342730FB22F9208331C061E574E08881FC
:104CE00099810E940B3F40E029C067E774E002C051
:104CF0006CE774E0888199810E940B3FF601408146
:104D000041701CC062E874E002C068E874E0888109
:104D100099810E940B3FF6014081469541700EC07B
:104D20006FE874E002C065E974E0888199810E94AF
:104D30000B3FF601408142FB442740F9009751F4B4
:104D4000EC81FD818F2D8F709181907FF92EF82A53
:104D5000F18221C0EC81FD810330110581F02F2DFE
:104D60002F703181307FF32EF22AF182BC01CE0107
:104D70000E94AB40EC81FD8180818F7E0BC08181E0
:104D80008F70982F9295907F892B8183EC81FD8184
:104D900080818061808381E001C080E0DF91CF91DC
:104DA0001F910F91FF90DF90CF900895FF920F9386
:104DB0001F93CF93DF93EC011D821C821A821B820A
:104DC000088119810115110509F456C0F801808583
:104DD000863009F051C08091880790918907892B0E
:104DE00009F44AC06CE974E0C8010E940B3F0097C7
:104DF00019F0FC0181858A83F801808191810E94EC
:104E00009F83F82E8B836EE974E0C8010E940B3FEC
:104E1000009779F51A8165ED79E084EA98E00E94BF
:104E200022744AE050E06F2D84EA98E00E94F37407
:104E300063ED79E084EA98E00E9422744AE050E051
:104E4000612F84EA98E00E94F37484EA98E00E945B
:104E5000457540E050E06EE974E0888199810E94D8
:104E6000503F6EE974E0888199810E940B3F009762
:104E700019F009969D838C83DF91CF911F910F913B
:104E8000FF900895EF92FF920F931F93CF93DF93BC
:104E90008091670690916806C4E0D0E021E030E0A0
:104EA000AC0142235323452B29F0A901409550958D
:104EB00084239523220F331F219791F7909368063F
:104EC000809367060E94C573009163061091640683
:104ED0002091650630916606601771078207930777
:104EE00008F459C0012B022B032B09F454C0109273
:104EF0006306109264061092650610926606E12C15
:104F0000F12CE091B30BF091B40BEC0FFD1F03817A
:104F100010E0228130E0418150E0608170E0C70103
:104F20000E946A1F8FEFE81AF80A249684E0E816B8
:104F3000F10439F7C1E0D0E08091080290910902B4
:104F40008C179D0728F4809108029091090201C0F6
:104F5000CE012091CD0B3091CE0BF901E80FF91F56
:104F60004AE050E0608184EA98E00E94F37460EACD
:104F700074E084EA98E00E9449752196C131D10518
:104F8000D9F684EA98E0DF91CF911F910F91FF90BD
:104F9000EF900C944575DF91CF911F910F91FF9089
:104FA000EF900895FC01A285B3851097A9F086853E
:104FB0009785029788F0CD010196938782876C933D
:104FC000868597850197978786870284F385E02DEC
:104FD000108281E090E0089580E090E00895FC0167
:104FE000868197818F3F2FEF920729F02FEF3FEFB8
:104FF000378326830895A085B185109789F024858D
:1050000035852115310561F0CD01019691878087A5
:105010008C912150310935872487082E000C990B7B
:105020000895FC0186819781019639F481E02485F9
:105030003585232B19F480E0089581E00895CF92FF
:10504000DF92EF92FF920F931F93CF93DF937C0138
:105050006A018B01C0E0D0E0CC15DD0589F0D701F5
:10506000ED91FC910284F385E02DC70119958F3FE6
:10507000BFEF9B0729F0F80181938F012196ECCFB8
:10508000CE01DF91CF911F910F91FF90EF90DF90B4
:10509000CF900895CF93C62FDC01ED91FC9100884D
:1050A000F189E02D1995DC01ED91FC910190F081E1
:1050B000E02D6C2FCF911994CF93DF93EC018E816B
:1050C0009F810196D9F4288539858A859B85820F31
:1050D000931F81159041A0F4E881F9810284F38542
:1050E000E02DCE011995813291056CF3E881F981AB
:1050F0000684F785E02D682FCE01199581E001C067
:1051000080E0DF91CF910895062E000C770BFC0113
:10511000778366830895CF93DF93EC018E819F811F
:10512000019611F5E881F9810088F189E02DCE0121
:105130001995DC01ED91FC910084F185E02D199524
:10514000892BA1F0E881F9810284F385E02DCE015D
:1051500019958132910534F3E881F9810684F78548
:10516000E02D682FCE01199581E001C080E0DF912C
:10517000CF91089508958EBD00000DB407FEFDCFB8
:105180008EB508958CBD9DBD0895CF93DF93EC013E
:10519000898D9A8D892B41F0E881F9810284F3850C
:1051A000E02DCE011995F4CFDF91CF910895FC0148
:1051B0002085318582859385AC014F5F5F4F538792
:1051C0004287820F931F0E94008B81E090E0089538
:1051D000FC01868197818F3F2FEF920729F02FEFF7
:1051E0003FEF378326830895208531858285938517
:1051F000AC014F5F5F4F53874287820F931F0E941E
:10520000F88A082E000C990B0895FC01868197817D
:105210008F3F2FEF920729F02FEF3FEF3783268341
:105220000895808591850C949884CF92DF92EF92B7
:10523000FF92CF93DF93EC018E819F818F3F2FEF01
:10524000920759F02FEF3FEF3F832E83DF91CF91ED
:10525000FF90EF90DF90CF9008950E94C5736B018F
:105260007C01A4EFCA0EA1E0DA1EE11CF11CE8816A
:10527000F9810088F189E02DCE011995DC01ED91CD
:10528000FC910084F185E02D1995892B39F40E9459
:10529000C5736C157D058E059F0548F3E881F9817E
:1052A0000088F189E02DCE011995DC01ED91FC918A
:1052B0000284F385E02DDF91CF91FF90EF90DF9096
:1052C000CF901994EF92FF920F931F93CF93DF9398
:1052D000009719F48FEF9FEF82C0FC01E484F584FE
:1052E000D7010D911C91D801ED91FC910688F789A9
:1052F000E02DC8011995882369F3D801ED91FC913F
:105300000084F185E02DC8011995D801ED91FC913B
:10531000892B61F30284F385E02DC8011995EC0116
:105320000196C1F2F8018589882339F04AE050E0FE
:105330006C2F84EA98E00E94F374D70112968C9146
:10534000882309F44BC0C532D10509F047C0D80104
:10535000ED91FC910084F185E02DC801199502972B
:105360005CF0D801ED91FC910688F789E02DC80129
:1053700019958111ECCFAECFD1E0C0E0D801ED910D
:10538000FC910284F385E02DC80119958F3FBFEF92
:105390009B0709F49FCF9C01215431092A31310523
:1053A00030F09C01215631092A31310538F48D2F16
:1053B0008295807F829FC00D11240AC0C0978A30D9
:1053C000910530F49D2F9295907F989FC00D1124E8
:1053D000D150A0F68C2FCC0F990B01C0CE01DF91DC
:1053E000CF911F910F91FF90EF90089561E0809110
:1053F00049090C94446460E0809149090C94446428
:105400000F931F93CF93DF93182F092FD62FC42FFD
:1054100080914709909148090E94C2280E94FB2967
:10542000802F0E94BB28812F0E94BB288D2F0E94B5
:10543000BB288C2F0E94BB280E94F62981E0DF91B7
:10544000CF911F910F910895CF93DF931F92CDB706
:10545000DEB7FC01218D328D232B61F021E041E08C
:1054600050E0BE016F5F7F4F84850E944F3E89816F
:1054700090E002C08FEF9FEF0F90DF91CF910895E2
:10548000AF92BF92CF92DF92FF920F931F93CF9371
:10549000DF938C015B01EA01FC01C788D08CF484A6
:1054A0008F2D0E94536E8C179D0720F48F2D0E9424
:1054B000536EEC019E01A501B6018F2D0E94146E62
:1054C000F8018789908D8C0F9D1F908F878BCE015F
:1054D000DF91CF911F910F91FF90DF90CF90BF9000
:1054E000AF900895EF92FF920F931F93CF93DF93A6
:1054F0008C017B01DC01ED91FC910284F385E02DB0
:105500001995829709F078C084E0F701808786E0DA
:1055100090E00E94CF80EC01892B09F46DC0EAE68F
:10552000F6E0F983E88380E091E0DF019C011D92C1
:1055300021503040E1F79B838A831D821C82D80171
:10554000ED91FC910284F385E02DC80119958F3F00
:10555000BFEF9B0709F44DC08232910509F44FC09B
:10556000803291050CF44BC08C35910511F0BE01D1
:105570003DC0D801ED91FC910284F385E02DC80176
:1055800019958F3FBFEF9B07A1F18236910531F14D
:105590005CF48F329105F9F08C359105C9F0829752
:1055A00071F6BE0182E222C08E369105D1F034F44C
:1055B0008636910521F6BE018CE018C08237910530
:1055C00099F08437910509F0BACFBE0189E00EC089
:1055D000BE018CE50BC0BE018FE208C0BE0188E0B1
:1055E00005C0BE018AE002C0BE018DE00E94BA7C07
:1055F000A6CFCE010E9467818FEF9FEF24C08C81E0
:105600009D81009749F0E881F9818E0F9F1FFC0171
:1056100031978081882321F0BE0180E00E94BA7C0E
:105620008C819D810E94CF808C01009739F06AE6C1
:1056300076E00E94DF8FCE010E946781F70112871A
:10564000018780E090E0DF91CF911F910F91FF9053
:10565000EF9008958DE090E00E94CF80009729F0B0
:105660002DE0FC0111922A95E9F708950F931F93FD
:10567000CF93DF930097E1F0EC010C851D850115B8
:10568000110579F0D8018D919C91009739F0DC01DA
:10569000ED91FC910488F589E02D1995C8010E94CF
:1056A0006781CE01DF91CF911F910F910C943684C9
:1056B000DF91CF911F910F910895AF92BF92CF923A
:1056C000DF92EF92FF920F931F93CF93DF9300D05F
:1056D0001F92CDB7DEB76115710509F496C06B0155
:1056E000182FDB011C96AD90BC901D97F501E08052
:1056F000F180D701ED91FC910688F789E02DC70173
:105700001995811104C0C6010E94362B7EC0F50197
:105710009281911114C0D701ED91FC910190F0811B
:10572000E02D612FC7011995F7018589882309F4B8
:1057300069C0612F84EA98E00E941B7463C0812FC6
:105740008F7D81548A3138F380ED810F8A3018F3D0
:1057500083ED810F8230F8F21F35E9F21E37D9F25E
:105760001132B1F086EC810F823090F08AED810F1A
:10577000873070F01D3361F0812F8F7E8F3241F0C2
:105780008DED810F823020F01B3511F01D3511F4A5
:1057900091FFC1CF19821A821B821C82812F012E98
:1057A000000C990B9F931F9382EA94E09F938F9331
:1057B0008E010F5F1F4F1F930F930E945B906E012E
:1057C000F4E0CF0ED11C0F900F900F900F900F9020
:1057D0000F90D701ED91FC910190F081E02DD8015F
:1057E0006C91C7011995F7018589882331F0D8019B
:1057F0006C9184EA98E00E941B740F5F1F4F0C1598
:105800001D0539F780E090E002C08FEF9FEF0F9009
:105810000F900F900F90DF91CF911F910F91FF90FC
:10582000EF90DF90CF90BF90AF900895DF92EF920E
:10583000FF920F931F93CF93DF934115510529F1E9
:105840008901EA01F62ED92EE82E80914709909120
:1058500048090E94C2280E94FB298D2D0E94BB2866
:105860008E2D0E94BB288F2D0E94BB287E01E00E4A
:10587000F11ECE15DF0529F080E00E94BB28899338
:10588000F8CF0E94F629C80102C080E090E0DF91C5
:10589000CF911F910F91FF90EF90DF9008951F938C
:1058A000CF93DF93D82F192FC62F8091470990915E
:1058B00048090E94C2280E94FB29812F0E94BB2810
:1058C0008D2F0E94BB288C2F0E94BB2880E00E9455
:1058D000BB28C82F0E94F6298C2FDF91CF911F91F2
:1058E0000895CF93DF931092060260ED77E080E099
:1058F00090E00E94976561E0809149090E9473647D
:10590000CFB7F89480916906811127C0E4E7F1E1EF
:105910008491EAEBF1E19491E82FF0E0EE0FFF1FA4
:10592000E55FFE4EA591B491EC91E92321F461E08D
:1059300085E30E94446461E085E30E9473648CB552
:1059400080618CBD8CB580648CBD61E084E30E9475
:10595000736461E083E30E947364809169068F5FE2
:1059600080936906CFBF60E080E090E00E944F2CFA
:10597000482F406864E080E090E00E94002AC0E088
:10598000DC2FD295DD0FD07ED45F42E06D2F8EE10B
:1059900090E00E94002A42E06D2F8FE190E00E948B
:1059A000002ACF5FC83061F7DF91CF910895DF9271
:1059B000EF92FF920F931F93CF93DF93D82FD92E9F
:1059C000C62F7A01890180914709909148090E9468
:1059D000C2280E94FB298D2D0E94BB288D2F0E947A
:1059E000BB288C2F0E94BB28E701E00EF11ECE15CC
:1059F000DF0521F089910E94BB28F9CF0E94F6298A
:105A0000C801DF91CF911F910F91FF90EF90DF9030
:105A100008951F93CF93DF93182F66E270E00E94E2
:105A20006059C82FD0E0DC2FCC2767E270E0812FCF
:105A30000E9460599E01280F311DC901DF91CF914D
:105A40001F9108951F93CF93DF93182F60E270E0AA
:105A50000E946059C82FD0E0DC2FCC2761E270E0B3
:105A6000812F0E9460599E01280F311DC901DF91CD
:105A7000CF911F910895CF92DF92EF92FF921F93E3
:105A8000CF93DF93182F6B017A010E948E3EEC01B9
:105A9000009799F463E070E0812F0E94605984318F
:105AA000F1F08823E1F0C1E0D0E08C3111F4C0E0E6
:105AB000D0E0D195C195D10912C0E816F9060CF4D1
:105AC000E7011C161D065CF420E0AE01B601812F33
:105AD0000E944F3E60E470E0812F0E94133BCE0194
:105AE000DF91CF911F91FF90EF90DF90CF900895BD
:105AF000CF93DF93FC01218D328D2115310519F4EF
:105B00008FEF9FEF11C0EC014217530708F0A90176
:105B10008C850E943B2D1816190694F7298D3A8D15
:105B2000281B390B3A8F298FDF91CF9108950F935E
:105B30001F93CF93DF931F92CDB7DEB7FC01218D6A
:105B4000328D232B61F08C0141E050E0BE016F5F8C
:105B50007F4F84850E943B2D181619061CF08FEF8D
:105B60009FEF08C0F801818D928D0197928F818FF0
:105B7000898190E00F90DF91CF911F910F9108954F
:105B80000F931F93CF93DF93CDB7DEB728970FB650
:105B9000F894DEBF0FBECDBF8C01DC01ED91FC910E
:105BA0000680F781E02D1995F80184850E948E3ECC
:105BB000892B51F148E050E0BE016F5F7F4FD80163
:105BC0001C968C910E943B2D18161906FCF4D801E6
:105BD000519684E0FE01319601900D928A95E1F78D
:105BE0008D8190E0982F88272E81820F911DF801DA
:105BF000968B858B8F8190E0982F88272885820F40
:105C0000911D928F818F02C080E090E028960FB6A0
:105C1000F894DEBF0FBECDBFDF91CF911F910F91E2
:105C200008959B018295880F807E6CE0680FC90102
:105C30000C94002ACF93C82F60E170E00E94133BC0
:105C40004FEF62E070E08C2FCF910C94112EFC018D
:105C5000848195810895089580E090E00895AF9241
:105C6000BF92CF92DF92EF92FF920F931F93CF9349
:105C7000DF93CDB7DEB7C154D1090FB6F894DEBFBC
:105C80000FBECDBF5C016B018A0168EE7BE084EA48
:105C900098E00E942274B50184EA98E00E94497558
:105CA00065EE7BE084EA98E00E942274C114D1047E
:105CB00009F4A1C00C0D1D1DF80110820E94105D99
:105CC0006A3F71051CF460EE7BE04DC07601E01682
:105CD000F10641F0F70161917F0184EA98E00E94AA
:105CE0001B74F5CF84EA98E00E94457580916B079C
:105CF00090916C079E012F5F3F4F790120E030E0CB
:105D0000039719F443E050E019C042E050E061E429
:105D1000C7010E94225CF70101900020E9F731974A
:105D20008F010E191F09A801B701C5010E94F68F46
:105D30000097A9F020E030E041E050E061E4C701C5
:105D40000E94225CF70101900020E9F731978F0152
:105D50000E191F09A801B701C5010E94F68F892BF2
:105D600039F065ED7BE084EA98E00E94227443C03C
:105D70000A0D1B1D68EA74E0C8010E94D68F892BAA
:105D800069F4F60101900020E9F73197EC19FD095B
:105D9000329720F0C6010E94FA7B2DC06FE270E0BE
:105DA000C8010E94CB8F5C01009741F0FC0110827A
:105DB0008181843201F1FFEFAF1ABF0AF8018081BF
:105DC0008432C9F0B801C7010E940740C7010E9490
:105DD0003B23882369F041E080916B0790916C0729
:105DE000039709F440E09501B601C7010E94212103
:105DF000C7010E949740CF5BDF4F0FB6F894DEBF1C
:105E00000FBECDBFDF91CF911F910F91FF90EF900B
:105E1000DF90CF90BF90AF900895CF93DF93EC01C8
:105E200067EF7AE084EA98E00E94227460E074E010
:105E3000CE01DF91CF910C94FE236F927F928F92CF
:105E40009F92AF92BF92CF92DF92EF92FF920F9309
:105E50001F93CF93DF93CDB7DEB72C970FB6F8948F
:105E6000DEBF0FBECDBF4C01762E672E6A015901F1
:105E700081E090E090937D0780937C0726E240E8E4
:105E800055E260E070E087E098E00E94B7447092CD
:105E9000FA0987E098E09093F9098093F809109245
:105EA000050B1092070B1092060B0115110541F01E
:105EB0000130110539F4FE2CEE24EE24EA9402C0E0
:105EC000FF24FA94C701A0E0B0E089839A83AB83F2
:105ED000BC8380E190E09E838D83A60160E070E04A
:105EE0004F83588769877A879C878B874AE050E081
:105EF000672D762D84EA98E00E94EC7460EA7BE0DE
:105F000084EA98E00E942274BE01695F7F4F84EAB0
:105F100098E00E9485248C016CE97BE00E94227449
:105F20004AE050E0B501C8010E94EC7469E97BE0E9
:105F3000C8010E942274BE016F5F7F4FC8010E949A
:105F400085240E944575A114B10491F082E0A81641
:105F5000B10409F5D092800AC0927F0A1092820A99
:105F60001092810AF092840AE092830A86E010C0BF
:105F7000D092800AC0927F0AE11003C080E090E0D6
:105F800002C080E09FEF9093820A8093810A85E0AF
:105F90000E94004207C061E87BE084EA98E00E942A
:105FA000227480E010927D0710927C07882331F0E4
:105FB000C4010E940D2F80E090E002C081E090E0DB
:105FC0002C960FB6F894DEBF0FBECDBFDF91CF91F8
:105FD0001F910F91FF90EF90DF90CF90BF90AF9007
:105FE0009F908F907F906F900895DF92EF92FF9235
:105FF0000F931F93CF93DF9300D000D0CDB7DEB7C0
:106000006DEE7BE084EA98E00E9422740EE91BE0CA
:10601000D12C80E1E82EF12CF8018081803130F420
:1060200061EB74E084EA98E00E944975F801808190
:10603000F5E090E0A0E0B0E089839A83AB83BC8375
:10604000FE82ED82BE016F5F7F4F84EA98E0DF162B
:1060500039F00E9485246BEE7BE00E94227404C01C
:106060000E9485240E944575D3940F5F1F4F86E0E0
:10607000D812D2CF26960FB6F894DEBF0FBECDBF92
:10608000DF91CF911F910F91FF90EF90DF900895D6
:10609000CF92DF92EF92FF928091880790918907CB
:1060A000892B09F46BC060EC7BE084EA98E00E94E5
:1060B000227480916E07882389F00E94737C0E946D
:1060C000422780916B0790916C07039711F00E9413
:1060D000464D0E9417600E940447EBCF10927F0745
:1060E00010927E070E94105D6B017C0168EA7BE0E4
:1060F00084EA98E00E9422742AE0B701A60184EAAB
:1061000098E00E945B7480918807909189070E94B3
:10611000BD3A109289071092880710927307109267
:1061200072071092700710926F0710928D071092ED
:106130008C071092B70B1092B60B1092BB0B1092FB
:10614000BA0B1092B90B1092B80B0E94105D6B0144
:106150007C0163EA7BE084EA98E00E9422742AE0F2
:10616000B701A60184EA98E00E945B7484EA98E093
:10617000FF90EF90DF90CF900C944575FF90EF90DB
:10618000DF90CF9008958F929F92BF92CF92DF922F
:10619000EF92FF920F931F93CF93DF93CDB7DEB7AC
:1061A000C854D1090FB6F894DEBF0FBECDBF7C0135
:1061B0008B010E947824B82E4801882428E092227E
:1061C00013FD06C080916B0790916C07039781F4D3
:1061D000B80166277370C7010E94FE2360E77BE069
:1061E00084EA98E00E94227488248A94982CF7C14B
:1061F00060E073E0C7010E943624082B192B1AAA0D
:1062000019AAFE01F3968EE0DF011D928A95E9F747
:1062100023961FAE1EAE2397709686E0DF011D9277
:106220008A95E9F711FF63C0F7018385948500978C
:1062300019F4C284D12C08C0DC01ED91FC91028CD0
:10624000F38DE02D19956C01C7010E948023B6E003
:10625000CB16D104B1F19E012F5C3F4FE7E0CE1683
:10626000D10444F4F1E0CF1AD10842E0C416D104BD
:1062700038F029C0A7E0CA16D10429F597FF13C04A
:106280001F926F931F927F939F779F938F9383EBC0
:1062900094E09F938F931F9280E18F933F932F936E
:1062A0000E941E901FC01F926F9389EB94E09F93F2
:1062B0008F931F9280E18F933F932F930E941E90A4
:1062C00011C01D7F14C09F938F937F936F9389EBB1
:1062D00094E09F938F931F9280E18F933F932F932E
:1062E0000E941E900FB6F894DEBF0FBECDBF10FF08
:1062F0001EC08B2D90E08D30910590F4FC01882715
:10630000EE53FF4F8F4F0C94818B6DE67BE002C004
:1063100069E67BE0CE018F5B9F4F0E94CF8307C071
:106320006BE57BE084EA98E00E9422741E7F20E007
:1063300030E043E050E060E3CE0101960E94225C31
:10634000D7011296ED91FC911397608171814FE214
:1063500050E0CE0101960E94E68F0E94C06C882317
:1063600009F439C180916D07811135C16801CC24D0
:10637000B2E0DB2211FF2DC08B2D90E08230910521
:1063800041F1059731F1BE016F5C7F4FCE0101965F
:106390000E94FA3E65E57BE084EA98E00E94227460
:1063A000BE016F5F7F4F84EA98E00E94497562E505
:1063B0007BE084EA98E00E942274BE016F5C7F4F0C
:1063C00084EA98E00E94497584EA98E00E94457545
:1063D0002AC010FF25C0BE016F5B7F4FCE01019622
:1063E0000E94FA3E6CE47BE084EA98E00E9422740A
:1063F000BE016F5F7F4F84EA98E00E94497569E4AF
:106400007BE084EA98E00E942274BE016F5B7F4FBC
:1064100084EA98E00E94497584EA98E00E944575F4
:10642000CD2809F457C020E030E043E050E060E3BD
:10643000CE0101960E94225CD7011296ED91FC914B
:106440001397608171814FE250E0CE0101960E9466
:10645000E68F60E474E0CE0101960E94C08F40E3B5
:1064600050E065E47BE0CE0101960E94D6836FE3A5
:106470007BE084EA98E00E942274BE016F5F7F4F48
:1064800084EA98E00E9449756CE37BE084EA98E036
:106490000E942274BE016F5C7F4F84EA98E00E94E4
:1064A000497584EA98E00E9445750E94C06C882373
:1064B00009F491C080916D0781118DC0BE016F5CA0
:1064C0007F4FCE0101960E94FA3E60E072E0C70164
:1064D0000E94C42310FF7BC0BAE0BB1681F0BB153D
:1064E00038F0E1E0BE1689F0F6E0BF1671F019C091
:1064F0002BE0B21639F04CE0B41661F012C062E342
:106500007BE00AC06DE27BE007C0D7011A968C9150
:10651000853039F467E37BE0CE018F5B9F4F0E94AB
:10652000CF8320E030E043E050E060E3CE0101960D
:106530000E94225CD7011296ED91FC911397608125
:1065400071814FE250E0CE0101960E94E68F60E437
:1065500074E0CE0101960E94C08F40E350E069E2F2
:106560007BE0CE0101960E94D68363E27BE084EA61
:1065700098E00E942274BE016F5F7F4F84EA98E02A
:106580000E94497560E27BE084EA98E00E942274F0
:10659000BE016F5B7F4F84EA98E00E94497584EAF0
:1065A00098E00E9445750E94C06C8823A1F08091FC
:1065B0006D07811110C0BE016F5B7F4FCE01019648
:1065C0000E94FA3E60E071E0C7010E94C423882463
:1065D0008394912C04C0B801C7010E94FE23C4011A
:1065E000C85BDF4F0FB6F894DEBF0FBECDBFDF91A3
:1065F000CF911F910F91FF90EF90DF90CF90BF90C0
:106600009F908F9008958F929F92AF92BF92EF923A
:10661000FF920F931F93CF93DF93CDB7DEB76997A8
:106620000FB6F894DEBF0FBECDBFDC011496ED911E
:10663000FC9115972085243009F0D7C0942EA62E02
:106640007C0161857285CE0101960E940740CE01D2
:1066500001960E943B23882309F454C08B8589301E
:1066600009F050C060E070E0CE0101960E949A23CC
:10667000B82E192F67E17BE084EA98E00E9422742B
:106680004AE050E06B2D712F84EA98E00E94EC7490
:1066900065E17BE084EA98E00E9422744AE050E0E1
:1066A0006A2D0A2C000C770B84EA98E00E94EC74A7
:1066B0006FE07BE084EA98E00E9422744AE050E0B8
:1066C000692D092C000C770B84EA98E00E94EC7489
:1066D00084EA98E00E94457500917C0710917D073F
:1066E0000115110591F0692DC7010E944D244A2D15
:1066F000AA0C550B660B770BC7010E944823C701F4
:106700000E940D2F00E010E06BC081E090E09093BC
:106710007D0780937C0726E040E855E260E070E06A
:1067200087E098E00E94B744B092FA0987E098E0C9
:106730009093F9098093F8091092050B1092070BBA
:106740001092060BB2E09B1609F457C085E098162C
:1067500009F453C06A2DAA0C770B880B990B0E9481
:10676000BB8C22E538EB42E152E40E94A08B20E092
:1067700030E040E251E40E94708D2DEE3EE94CE3A2
:106780005EE30E94118C4B015C0120E030E0A90126
:106790000E946B8D20E030E040E05FE387FD28C081
:1067A000C501B4010E94A08B0E94838C83ED97E009
:1067B0009093800A80937F0A1092820A1092810A35
:1067C0007093840A6093830A86E00E9400421092CC
:1067D0007D0710927C07882399F0C7010E940D2F36
:1067E000CE0101960E9497400EC000E010E00BC061
:1067F000C501B4010E949F8BD7CF60E070E0D6CF77
:1068000001E010E0EDCFC80169960FB6F894DEBF45
:106810000FBECDBFDF91CF911F910F91FF90EF90F1
:10682000BF90AF909F908F900895DF92EF92FF926C
:106830000F931F93CF93DF93EC01E62ED42E60E0ED
:1068400070E00E949A23F82E192F6BE07BE084EA17
:1068500098E00E9422744AE050E06F2D712F84EA84
:1068600098E00E94EC7469E07BE084EA98E00E9482
:1068700022746E2D0E2C000C770B4AE050E084EA57
:1068800098E00E94EC7484EA98E00E9445750091BB
:106890007C0710917D070115110591F06D2DCE013A
:1068A0000E944D244E2DEE0C550B660B770BCE013E
:1068B0000E944823CE010E940D2F00E010E05FC02F
:1068C00081E090E090937D0780937C0726E040E88C
:1068D00055E260E070E087E098E00E94B744F092F3
:1068E000FA0987E098E09093F9098093F8091092EB
:1068F000050B1092070B1092060B80ED97E090931A
:10690000800A80937F0A1092820A1092810AEE20F8
:1069100039F085E090E09093840A8093830A04C064
:106920001092840A1092830A86E00E94004262E379
:1069300070E080E090E00E94976582ED97E0909390
:10694000800A80937F0A1092820A1092810A8E2D0B
:1069500094E68902A00111245093840A4093830A8B
:1069600086E00E94004210927D0710927C078823E7
:1069700021F0CE010E940D2F02C001E010E0C801FD
:10698000DF91CF911F910F91FF90EF90DF900895CD
:106990002F923F924F925F926F927F928F929F922F
:1069A000AF92BF92CF92DF92EF92FF920F931F931D
:1069B000CF93DF9300D01F92CDB7DEB76C013B01C0
:1069C0000E947824823011F0853011F4612C712CF2
:1069D000F6010480F581E02DFC83EB838085853012
:1069E00009F076C0CF010E948A3FE82EF12CF2E038
:1069F000EF16F1040CF46CC060E08B819C810E9466
:106A0000263FFC014184528461E08B819C810E947D
:106A1000263FFC0181849284A384B48480917C0706
:106A200090917D079A83898392E0E916F10409F435
:106A30004CC062E08B819C810E94263FFC01018555
:106A40001285F3E0EF16F10409F443C063E08B8193
:106A50009C810E94263FFC0121843284F4E0EF16E1
:106A6000F10449F064E08B819C810E94263FFC0187
:106A70008185928502C082E090E09C838B83211403
:106A80003104B1F0E981FA81EF2B31F0C6010E94A7
:106A90000D2F80E090E025C09301D1010E94988BDA
:106AA00024E630E040E050E00E94408B790105C0D0
:106AB00089819A81892B51F773012B813C81A40133
:106AC000B201C6010E941D2F0CC00FEF1FEF01C0C5
:106AD00008C08FE3282E312CE2E0F0E0FC83EB834A
:106AE000D1CF0F900F900F900F90DF91CF911F910A
:106AF0000F91FF90EF90DF90CF90BF90AF909F905D
:106B00008F907F906F905F904F903F902F9008955F
:106B1000EF92FF920F931F93CF93DF93CDB7DEB722
:106B200069970FB6F894DEBF0FBECDBF7C01DC01C4
:106B30001296ED91FC9113976081718184EA98E03F
:106B40000E944975C7010E943B2381110DC06EEE62
:106B50007AE084EA98E00E94227484EA98E00E9435
:106B600045758FEF9FEFAFC0C7010E947824F701F2
:106B700012851730F1F0853099F028F4813049F012
:106B8000823071F016C0863021F0E6EFE80FE33076
:106B900080F465EE7AE084EA98E00E94227491C065
:106BA0006AED7AE084EA98E00E94227480E090E046
:106BB0008AC0D7011B968D919C911C97009741F03C
:106BC000DC01ED91FC910688F789E02D19957BC0D9
:106BD000C7010E948023812F90E08A30910508F040
:106BE00054C0FC018827E153FF4F8F4F0C94818BD9
:106BF000D7011496ED91FC9115978085853009F0A9
:106C000047C064ED7AE084EA98E00E942274D701DC
:106C10001496ED91FC9115970681178101151105C8
:106C200061F1F8018085843011F561857285CE01AE
:106C300001960E940740CE0101960E943B238823C3
:106C400091F0CE0101960E948835181619065CF461
:106C50006BEC7AE084EA98E00E942274CE010196FF
:106C60000E9497402EC0CE0101960E949740D80105
:106C700012960D911C911397D1CF60EC7AE092CFD0
:106C8000062F10E007C08B0105C066EB7AE08ACFC3
:106C900000E010E06BEA7AE084EA98E00E94227457
:106CA0004AE050E0B80184EA98E00E94EC7484EA7B
:106CB00098E00E94457581E090E0012B21F480E08E
:106CC00002C081E074CF69960FB6F894DEBF0FBEA4
:106CD000CDBFDF91CF911F910F91FF90EF9008955D
:106CE0002F923F924F925F926F927F928F929F92DC
:106CF000AF92BF92CF92DF92EF92FF920F931F93CA
:106D0000CF93DF93CDB7DEB728970FB6F894DEBFE9
:106D10000FBECDBF8C016B010E94ED7D019609F481
:106D2000D3C2D801ED91FC910284F385E02DC80116
:106D300019957C018F3FBFEF9B0709F4C5C2D801AD
:106D4000ED91FC910684F785E02D682FC801199517
:106D5000B2E2EB16F10429F4B601C8010E94722ACE
:106D6000B5C2EDE2EE16F10429F0C701C0970A970B
:106D700008F044C1D801ED91FC910284F385E02D27
:106D8000C80119957C018F3FBFEF9B0709F49CC296
:106D90008D9789F4D801ED91FC910284F385E02D63
:106DA000C80119957C01019609F48EC2EFEFFFEF3F
:106DB000F887EF8304C021E030E038872F83C701D4
:106DC000C097A12CB12C0A97C8F49AE0992E9A9CEE
:106DD000C0019B9C900D1124B701605371095B01A8
:106DE000A80EB91ED801ED91FC910284F385E02D27
:106DF000C80119957C01C0970A9748F3BEE2EB16CB
:106E0000F104D1F0C7018F7D85349105A9F0EF81A0
:106E1000F885AE9EC001AF9E900DBE9E900D1124D0
:106E2000092E000CAA0BBB0BF60181879287A38762
:106E3000B48782E08087D8C0B501BB0C880B990B62
:106E40000E94BB8C2B013C01FEE2EF16F104A1F580
:106E5000D801ED91FC910284F385E02DC8011995CC
:106E60007C01212C312C20E030E040E251E4C301D0
:106E7000B2010E94708D4B015C01B7016053710932
:106E8000072E000C880B990B0E94BB8CA501940166
:106E90000E94A08B2B013C01B1E02B1A3108D801D4
:106EA000ED91FC910284F385E02DC80119957C01D8
:106EB000C0970A97C0F202C0212C312CC7018F7DE8
:106EC0008534910509F042C0D801ED91FC9102840E
:106ED000F385E02DC80119957C018B32910559F499
:106EE000D801ED91FC910284F385E02DC80119953C
:106EF0007C01B1E00CC08D9761F4D801ED91FC915B
:106F00000284F385E02DC80119957C01BFEFBE8393
:106F100002C0E1E0EE83A12CB12C8AE0982EC701DB
:106F2000C0978A309105B0F49A9C90019B9C300DDB
:106F300011245C01A20EB31ED801ED91FC910284D4
:106F4000F385E02DC80119957C01E9CFB1E0BE833E
:106F5000A12CB12CEF81F885BF01FF0F880B990B95
:106F60000E94BB8CA30192010E94708D2B013C01F9
:106F7000B501BB0C880B990B0E94BB8C4B015C01CB
:106F8000FE816F2FFF0F770B880B990B0E94BB8C34
:106F90009B01AC01C501B4010E94708D4B015C01E5
:106FA000B101330C880B990B0E94BB8C9B01AC0187
:106FB000C501B4010E94A08B9B01AC0160E070E0B0
:106FC00080E291E40E94DD8D9B01AC01C301B2011E
:106FD0000E94708DD60119966D937D938D939C932D
:106FE0001C9783E018968C93D801ED91FC91068450
:106FF000F785E02D6E2DC801199522C0BBE5EB1673
:10700000F10409F060C0D801ED91FC910284F38590
:10701000E02DC80119958B35910509F055C185E022
:10702000F6018087C8010E94ED7DD801ED91FC91A9
:107030000284F385E02DC80119958D35910519F469
:1070400080E090E043C1D801ED91FC910684F78582
:10705000E02D682FC8011995BB24BA940E942A2BF1
:107060007C01009709F430C1BB2021F0F601978321
:10707000868308C0D40113969C938E931297FC01CB
:1070800095828482C8010E94ED7DB701C8010E94EB
:107090007036892B09F018C1C8010E94ED7DD80116
:1070A000ED91FC910284F385E02DC8011995B12C76
:1070B00047018C32910591F221E030E08D35910548
:1070C00009F089C086C0BBE7EB16F10409F088C05F
:1070D000D801ED91FC910284F385E02DC80119954A
:1070E0008B37910509F0F0C086E0F6018087C80172
:1070F0000E94ED7DD801ED91FC910284F385E02D95
:10710000C80119958D37910509F49ACFD801ED91F1
:10711000FC910684F785E02D682FC8011995992404
:107120009A940E942A2B7C01009709F4CDC09920E3
:1071300021F0F6019783868308C0D50113969C93AE
:107140008E931297FC01B582A482C8010E94ED7D46
:10715000B701C8010E94722A019609F4B5C0C8019E
:107160000E94ED7DD70119968D919C911A971196E9
:107170009C938E931A961C921E921997D801ED91AA
:10718000FC910284F385E02DC8011995CA9709F096
:107190009BC0C8010E94ED7DB701C8010E947036F6
:1071A000019609F491C0C8010E94ED7DD801ED91CE
:1071B000FC910284F385E02DC8011995912C5701AB
:1071C0008C32910509F4ADCF21E030E08D37910587
:1071D00011F420E030E088279927821B930B76C0BA
:1071E000BEE6EB16F10411F519821A821B821C828D
:1071F000D801ED91FC910484F585E02D44E050E048
:10720000BE016F5F7F4FC8011995049709F05CC0FC
:1072100044E050E06CEB74E0CE0101960E94F68FE2
:10722000009709F051C0F601108650C0F6E6EF163F
:10723000F10421F59E012F5F3F4F790185E0D901CF
:107240001D928A95E9F7D801ED91FC910484F585AA
:10725000E02D45E050E0B901C80119950597A1F569
:1072600045E050E061EC74E0C7010E94F68F0097A2
:1072700059F521E0F6012087118628C0F4E7EF16C2
:10728000F10411F519821A821B821C82D801ED913A
:10729000FC910484F585E02D44E050E0BE016F5F71
:1072A0007F4FC8011995049779F444E050E067ECEA
:1072B00074E0CE0101960E94F68F009729F421E038
:1072C000F6012087218702C08FEF9FEF28960FB627
:1072D000F894DEBF0FBECDBFDF91CF911F910F910C
:1072E000FF90EF90DF90CF90BF90AF909F908F90E6
:1072F0007F906F905F904F903F902F900895CF9226
:10730000DF92EF92FF92CF93DF93EC010E94C5735F
:107310006B017C0180915B0990915C09DC01ED912E
:10732000FC910084F185E02D1995892B79F40E9458
:10733000C573DC01CB018C199D09AE09BF098839E1
:107340009A43A105B10530F380E00DC080915B093F
:1073500090915C09DC01ED91FC910284F385E02DB4
:107360001995888381E0DF91CF91FF90EF90DF90B6
:10737000CF900895AF92BF92CF92DF92EF92FF929B
:107380000F931F93CF93DF938C01EB0162E070E0CA
:107390000E949A237C0197FF03C080E090E076C0B2
:1073A00063E070E0C8010E949A23AC011816190628
:1073B00014F04FE350E081E0E816F10421F4CD2F02
:1073C000DD0FDD0B04C082E0E816F1040CF4DD27CC
:1073D00024E630E0DE010E94988B9A01550F440BA1
:1073E000550B0E94408B69017A015901C8010E9426
:1073F0007824C82FD0E0C8010E9480230D2C000CF7
:10740000EE08FF086C157D058E059F0549F4AB2835
:10741000E9F1C230D10561F0C530D105B9F508C038
:10742000AB28E1F0C630D10539F0C130D10521F0EB
:1074300061E0C8010E944D24B701A601C8010E9465
:107440004823C230D10511F0259729F460E071E09E
:10745000C8010E94C33060E072E00BC0C530D105A6
:10746000A9F0229799F062E0C8010E944D2460E0E3
:1074700071E0C801DF91CF911F910F91FF90EF90C4
:10748000DF90CF90BF90AF900C94C330DF91CF913D
:107490001F910F91FF90EF90DF90CF90BF90AF9032
:1074A0000895CF93DF93EC0160E073E00E943624EF
:1074B000009791F020916B0730916C0724303105D3
:1074C00059F4BC01CE010E94C33060E073E0CE01EC
:1074D000DF91CF910C94C423DF91CF9108958F92C7
:1074E0009F92AF92BF92EF92FF920F931F93CF9311
:1074F000DF938C017B0149015A010E942A2BEC0188
:10750000892BF9F083E0888789869A86AB86BC86CA
:1075100088819981009711F00E946781C7010E94BC
:10752000748F99838883BE01C801DF91CF911F9129
:107530000F91FF90EF90BF90AF909F908F900C9421
:10754000333FDF91CF911F910F91FF90EF90BF904C
:10755000AF909F908F9008956115710549F0FB01E0
:1075600001900020E9F73197AF01461B570B02C08D
:1075700040E050E020E00C94AA3E0F931F93CF937D
:10758000DF93EC012097F9F00A811B81888587FD44
:1075900006C08E819F81009711F00E94BD3A8885B8
:1075A000843031F489859A85009711F00E946781B3
:1075B00088819981009711F00E946781CE010E9415
:1075C0006781E801DFCFDF91CF911F910F9108957F
:1075D0000F931F93CF93DF93009791F08C010E943C
:1075E0002A2BEC01892B61F0C8010E94ED7DBE01C0
:1075F000C8010E947036019631F4CE010E94BD3A56
:1076000080E090E001C0CE01DF91CF911F910F91FA
:107610000895FC018485883021F063E070E00C94CB
:10762000605980E00895CF93C82F462F61E070E045
:107630000E94112E61E070E08C2F0E946059811130
:10764000F9CFCF9108950F931F93CF93DF93EC0160
:107650000E9446748C01CE010E944575800F911FD7
:10766000DF91CF911F910F9108952F923F924F92EA
:107670005F926F927F928F929F92AF92BF92CF92C2
:10768000DF92EF92FF920F931F93CF93DF9300D07F
:1076900000D0CDB7DEB71C018DE599E00E947F399F
:1076A00081113BC036C07801CE0101960E947F391E
:1076B000882379F187010F5F1F4FE981D601ED9390
:1076C0006D01AE2FAF77B0E0A50194010E945F8BF2
:1076D000460E571E681E791E47E0880C991CAA1C8E
:1076E000BB1C4A95D1F7E7FF2BC005301105D9F631
:1076F0008FEF9FEF9093F7098093F60980915B09D4
:1077000090915C09DC01ED91FC910488F589E02DF4
:10771000199560E070E0CB01B0C0F0915D09FA838B
:1077200019828EE5C82E89E0D82EEE24E394F12C40
:10773000412C512C3201812C912C54018394B4CFD3
:10774000BA81B07FBA838FEF800FF1018083B033AD
:1077500021F5C801835A964F0E947F398823C9F2C8
:10776000C701815A964F0E947F39882391F20E5F9C
:107770001F4FD101EC91F0E0E95AF64FC780D12CB0
:10778000DC2CCC248085C80ED11C80915D0981FF42
:1077900008C0B2E0CB0ED11C04C080E0C12CD12CBB
:1077A00001C082E090E0A0E0B0E04801A12CB12C43
:1077B0009C01AD01281939094A095B092B833C83D7
:1077C0004D835E83E12CF12C8B819C81AD81BE8148
:1077D000880D991DAA1DBB1D84159505A605B70525
:1077E000D8F5CE0101960E947F39882309F491CF04
:1077F0008091F4099091F5090097F1F03A813033C6
:10780000D9F4D1012C914EEF5FEF6FEF7FEF421B68
:10781000510961097109480D591D6A1D7B1DC41666
:10782000D506E606F70640F4DC01ED91FC910190E7
:10783000F081E02D698119950038110538F4F801BF
:10784000E95AF64F898186830F5F1F4FBFEF8B1A6E
:107850009B0AAB0ABB0AB8CF8091F4099091F50955
:10786000892B41F4E1E88E169104A104B10410F0D3
:1078700000E010E0B80180E090E026960FB6F894A2
:10788000DEBF0FBECDBFDF91CF911F910F91FF9053
:10789000EF90DF90CF90BF90AF909F908F907F90B0
:1078A0006F905F904F903F902F9008952F923F924E
:1078B0004F925F926F927F928F929F92AF92BF9200
:1078C000CF92DF92EF92FF920F931F93CF93DF93AC
:1078D00000D0CDB7DEB70E94C06C382E882309F4E3
:1078E00028C10E94C5734B015C018091E30990910E
:1078F000E409A091E509B091E609A5019401281BCE
:10790000390B4A0B5B0BDA01C90189399A43A1058E
:10791000B105A8F48091DF099091E009A091E109F7
:10792000B091E209A5019401281B390B4A0B5B0BAE
:10793000DA01C90189399A43A105B105C8F120913D
:10794000E70980915B0990915C09222371F02CEF8B
:107950003FEF3093F7092093F609DC01ED91FC919C
:107960000488F589E02D1995E3C020EC20935D098A
:1079700010925E09DC01ED91FC910280F381E02D13
:1079800042E050E06DE579E019958092DF09909230
:10799000E009A092E109B092E2098092E309909295
:1079A000E409A092E509B092E60981E08093E70935
:1079B00080915B0990915C09DC01ED91FC91008460
:1079C000F185E02D1995892B09F4B3C0CE010196FC
:1079D0000E94353B2B013C01672B09F4A5C0809226
:1079E000E3099092E409A092E509B092E60980913A
:1079F0005D09807F803309F07BC08091E809909118
:107A0000E909892B09F495C0E980F12CF701E95ABD
:107A1000F64F078110E0102F00278085080F111DF9
:107A20009701215A364F6901B701605A764FA80174
:107A3000C9010E949B8FB8016E0D7F1DDB01A95A01
:107A4000B64F18961C92189780915D098670282E63
:107A5000E091E809F091E90932E083133CC01996FE
:107A60008C91199790E0982F88271A962C91AC0149
:107A7000420F511D5B834A834BEF5FEF4E195F0945
:107A8000401B510B440D551D6E59764FC60119957B
:107A900080E480935D0920925E095B8150935F09C9
:107AA0008A818093600980915B0990915C09DC0177
:107AB000ED91FC910280F381E02D44E050E06DE512
:107AC00079E019958092DF099092E009A092E1098E
:107AD000B092E2092EC04DEF5FEF4E195F09401BD7
:107AE000510B440D551D605A764FC601199521C0A2
:107AF000803CA9F480ED80935D0910925E0980912D
:107B00005B0990915C09DC01ED91FC910280F381AD
:107B1000E02D42E050E06DE579E019950AC0803D26
:107B200041F41092E70905C00E94C06C811101C0A8
:107B3000312C832D0F900F900F90DF91CF911F91DB
:107B40000F91FF90EF90DF90CF90BF90AF909F90FC
:107B50008F907F906F905F904F903F902F900895FF
:107B6000AF92BF92CF92DF92EF92FF921F93CF938B
:107B7000DF9300D000D0CDB7DEB76C017C0110E000
:107B80008AE0A82EB12C1330A9F0F701828190E091
:107B9000A0E0B0E089839A83AB83BC83BE82AD82D0
:107BA000BE016F5F7F4F84EA98E00E94852465EFF5
:107BB0007BE014C0F601858190E0A0E0B0E089830D
:107BC0009A83AB83BC83BE82AD82BE016F5F7F4F61
:107BD00084EA98E00E94852462EF7BE00E94227490
:107BE0001F5FFFEFEF1AFF0A143069F626960FB6F3
:107BF000F894DEBF0FBECDBFDF91CF911F91FF90F4
:107C0000EF90DF90CF90BF90AF90089524E030E0E8
:107C1000AC0160E08FE090E00C94162CCF93DF93E2
:107C2000C7E5D9E080EE8E831F828C819D81DC01C7
:107C3000ED91FC910280F381E02D42E050E06DE592
:107C400079E019958FEF9FEF9093F7098093F609EC
:107C50008C819D81DC01ED91FC910680F781E02D06
:107C600019958C819D81DC01ED91FC910488F58949
:107C7000E02D19950E94C5736093DF097093E009A8
:107C80008093E1099093E2096093E3097093E4091A
:107C90008093E5099093E609DF91CF910895CF9203
:107CA000DF92EF92FF920F931F93CF93DF93D82E23
:107CB0007B018A01C22E68E270E00E946059D82FD1
:107CC00069E270E08D2D0E946059CD2FD0E0DC2F4D
:107CD000CC27C80FD11D6D2D6295660F607E685E42
:107CE0009801A701CE010E94162CC1100EC0C00F32
:107CF000D11F4D2F68E270E08D2D0E94112E4C2F68
:107D000069E270E08D2D0E94112EDF91CF911F91BD
:107D10000F91FF90EF90DF90CF900895FF920F9317
:107D20001F93CF93DF93F82E00E010E08F2D0E9479
:107D3000092DEC01892B21F08F2D0E94092D8C013A
:107D4000C017D10799F7CE01DF91CF911F910F9105
:107D5000FF900895DF92EF92FF920F931F93CF93BE
:107D6000DF938C01D62EE72EEA01F22E0E94C06C22
:107D70008823B9F1F80101900020E9F73197E01B61
:107D8000F10BCE010796E80FF91FE138F10548F530
:107D900045E050E06DE579E0C8010E94376CAC0128
:107DA000ED2DFE2DDC01A35AB64F9F012C0F3D1F78
:107DB000E217F30719F081918D93FACF2597FF20F1
:107DC00011F081E301C080E34C0F5D1F6DE579E0A8
:107DD000DF91CF911F910F91FF90EF90DF900C9466
:107DE000576C80E0DF91CF911F910F91FF90EF9042
:107DF000DF9008956115710549F0FB0101900020A5
:107E0000E9F73197AF01461B570B02C040E050E045
:107E100021E00C94AA3E0F931F93CF93DF938B0125
:107E2000FC01C681D781209759F0B80188819981DA
:107E30000E94AD8F892B21F00A80DB81C02DF3CF0A
:107E4000CE01DF91CF911F910F910895FC018681A2
:107E50009781009739F0662329F06150FC018281F7
:107E60009381F7CF0895DC011696ED91FC91179759
:107E700061157105A1F0309729F417967C936E93E4
:107E80001697089582819381009711F0FC01FACF33
:107E900073836283DB011596FC93EE931497089528
:107EA000CF92DF92EF92FF920F931F93CF93DF93C6
:107EB0008C017B016A010E942A2BEC01892B09F1BC
:107EC00082E08887A601DD0C660B770B49875A870D
:107ED0006B877C8788819981009711F00E94678168
:107EE000C7010E94748F99838883BE01C801DF9106
:107EF000CF911F910F91FF90EF90DF90CF900C9456
:107F0000333FDF91CF911F910F91FF90EF90DF9062
:107F1000CF900895DC011696ED91FC91179780E0C3
:107F2000309729F08F5F0280F381E02DF9CF08951B
:107F3000BF92CF92DF92EF92FF920F931F93CF9356
:107F4000DF93EC018A819B810E948A3F082F10E019
:107F5000C801880F991F9C0125563D4F790132E0D9
:107F6000B32E04301105D4F4F701C190D1907F01F4
:107F70000E942A2B009751F0FC01B086A601DD0C6F
:107F8000660B770B4187528763877487BC018A81B0
:107F90009B810E94333F0F5F1F4FE3CF0A811B81FC
:107FA00060E0C8010E94263FFC01F184FA8661E08E
:107FB000C8010E94263F9D838C8362E0C8010E9415
:107FC000263F9F838E8364E0C8010E94263F9987E5
:107FD0008887FCE0FF1211C08DE090E00E94CF8006
:107FE0008C01FC01D383C28387E492E09183808378
:107FF000C8010E94825F1C870B87DF91CF911F9180
:108000000F91FF90EF90DF90CF90BF9008958F92E7
:108010009F92AF92BF92CF92DF92EF92FF920F9317
:108020001F93CF93DF93CDB7DEB767970FB6F89462
:10803000DEBF0FBECDBF8C017B018FE392E0F80164
:10804000918380834801FDE08F0E911C9F8A8E8A68
:10805000F801148613861586108E178A672B09F48B
:1080600048C0A0906F07B0907007A114B10409F444
:1080700040C06FE270E0C7010E94CB8F6C01892B7A
:1080800081F1D701FE01319680E090E0BF012D9192
:10809000222341F02F3231F08431910519F02193E0
:1080A0000196F5CFFB01E80FF91F1082C5010E9470
:1080B0000B3FF80193838283B6016F5F7F4F4AE0E5
:1080C00050E0C4010E940490CE0146960E94EB202D
:1080D000F801908F878B8E899F89892B69F415868B
:1080E0000BC0B701C5010E940B3FF8019383828347
:1080F00003C0F80113821282C8010E943B23882327
:1081000019F0C8010E94983F67960FB6F894DEBF39
:108110000FBECDBFDF91CF911F910F91FF90EF90D8
:10812000DF90CF90BF90AF909F908F9008952FE3F6
:1081300032E0DC0111963C932E931B968D919C911D
:108140001C97009739F0DC01ED91FC910280F381DE
:10815000E02D199408953F924F925F926F927F9213
:108160008F929F92AF92BF92CF92DF92EF92FF9247
:108170000F931F93CF93DF93CDB7DEB7C054D109D0
:108180000FB6F894DEBF0FBECDBF6115710509F4BF
:108190001DC1342E8B012C01FB018085853019F027
:1081A0008630D9F013C180916E078F5F80936E0780
:1081B000FB01068117810115110549F0432DB80116
:1081C000C2010E94AB40F80102811381F4CF80917B
:1081D0006E07815080936E07F9C062E474E0C801B5
:1081E0000E940B3F7C016CEC74E0C8010E940B3FC5
:1081F0005C0161ED74E0C8010E940B3F4C0166ED2B
:1082000074E0C8010E940B3F3C016BED74E0C801B3
:108210000E940B3F6C0167E474E0C8010E940B3FB1
:108220008C018114910461F0332051F0F4018085B8
:10823000843031F4A184B284C114D10491F415C006
:10824000A114B10439F0F5018085843019F4A184BA
:10825000B28402C0A12CB12CC114D10431F033205E
:1082600021F0F6018085843039F06114710439F011
:10827000F3018085843019F4C184D28402C0C12CFA
:10828000D12CF201938061E17CE084EA98E00E94C5
:1082900022744AE050E0692D84EA98E00E94F37469
:1082A0006DE07CE084EA98E00E94227484EA98E021
:1082B0000E944575E114F104F1F0F70161857285C2
:1082C00084EA98E00E94497568E07CE084EA98E0DE
:1082D0000E942274B50184EA98E00E94497584EAFC
:1082E00098E00E9445750115110549F4A114B104E7
:1082F00009F04EC069C00115110509F465C0F80107
:108300006185728584EA98E00E94497563E07CE0AB
:1083100084EA98E00E942274B60184EA98E00E9400
:10832000497584EA98E00E944575C114D10459F159
:10833000F8018085843039F56185728540E450E02C
:10834000CE0101960E9404900E94C06C8823D9F04F
:1083500080916D07811117C06FE270E0CE01019628
:108360000E94CB8F892B51F4F8012185328543E09F
:1083700050E060E4CE0101960E94225CB601CE017D
:1083800001960E94FA3EE114F10409F0AFCF1CC03F
:10839000F70180858430C1F461857285CE01019634
:1083A0000E940740CE0101960E943B23882341F0A2
:1083B00020E030E041E0B501CE0101960E9421218C
:1083C000CE0101960E94974081E001C080E0C05C30
:1083D000DF4F0FB6F894DEBF0FBECDBFDF91CF9158
:1083E0001F910F91FF90EF90DF90CF90BF90AF90D3
:1083F0009F908F907F906F905F904F903F900895E7
:108400008F929F92AF92BF92CF92DF92EF92FF92A4
:108410000F931F93CF93DF93CDB7DEB7DA950FB6E7
:10842000F894DEBF0FBECDBFC82E8091FA098983B4
:10843000CA8221E0C216A0F074E07C1518F487E12E
:10844000C8120EC08091FB099091FC099B838C831C
:108450008091FD099091FE099D838E8386E001C085
:1084600082E08E010F5F1F4F90E19C1528F0AFE076
:10847000CA1630F49BEF01C09AEE9C0D923078F44E
:1084800020917F0A9091800AF801E80FF11D9083F6
:1084900091E0980FF801E90FF11D8E5F2083BFE096
:1084A000CB1641F1BC1558F0E5E0CE16A1F0F6E090
:1084B000CF12B6C02091830A9091840A10C026E1A1
:1084C000C21609F48EC077E1C71609F459C090E1CD
:1084D000C912A6C055C02091810A9091820AF80164
:1084E000E80FF11D908391E0980FF801E90FF11D5D
:1084F0008E5F95C02091810A3091820AF801E80FC1
:10850000F11D308342E0480F91E0980FF801E90F28
:10851000F11D2083B90167707727A3E03695279571
:10852000AA95E1F7672B19F091E0920F01C0922F05
:10853000B3E0B80FF801E40FF11D90838C5F60E0A9
:1085400070E0A0E04FEF480F9A1303C08B2F890F04
:1085500067C050E09B0135952795400F511F220FB2
:10856000331FF901ED57F54FA0FD02C0208101C076
:108570002181FA012083AF5F6F5F7F4F8F5FE2CF72
:108580002091810A3091820AF801E80FF11D3083B1
:1085900091E0980FF801E90FF11D208392E0980F08
:1085A000F801E90FF11D8D5F922F990F908390E0F4
:1085B0003327E92FF0E0E217F30794F5EE0FFF1FE2
:1085C000ED57F54F50814181F801E80FF11D4083CF
:1085D00041E0480FF801E40FF11D8E5F50839F5F6B
:1085E000E8CF9091830A2091840AF801E80FF11DE9
:1085F000208321E0280FF801E20FF11D90832091E4
:10860000850A9091860A32E0380FF801E30FF11DD8
:10861000908393E0980FF801E90FF11D8C5F2083A0
:108620007801F8012FEF3FEFD02E9E2F901B981767
:10863000A0F49191292748E050E0B901769567951B
:1086400020FF06C09B0191E0292790EA392701C04D
:108650009B014150510989F7E8CFF801E80FF11D5E
:108660002083B2E0BB2EB80E8F5FF801E80FF11D3A
:108670003083F801EB0DF11D10828091F809909183
:10868000F909DC01ED91FC910284F385E02D199547
:10869000019699F7E0910E0BF0910F0B309709F0CE
:1086A00019958091F8099091F9092E2D2D192B1506
:1086B00058F4F70161917F01DC01ED91FC9101908B
:1086C000F081E02D1995EDCFDC01ED91FC91068054
:1086D000F781E02D1995E091100BF091110B309777
:1086E00009F019950E94C5734B015C01A8E0EA2EC0
:1086F000F12CD12C8091F8099091F909DC01ED91D0
:10870000FC910084F185E02D1995892BC1F08091B1
:10871000F8099091F909DC01ED91FC910284F3854F
:10872000E02D19959091FA09891711F0FF2099F120
:10873000F801EF0DF11D8083EA94F39407C0E091F6
:108740000C0BF0910D0B309709F01995B5E0FB1269
:1087500022C0EA818E2F8F7790E08C159D0509F05D
:10876000A2C0E7FF04C08B81882381F181C08E2FD6
:1087700090E0FC013197E731F10568F48827E75272
:10878000FF4F8F4F0C94818BF3E0EF2E04C0EB80F2
:1087900002C0E5E0EE2E0E94C573DC01CB01881912
:1087A0009909AA09BB09813D9740A105B10538F493
:1087B00080E0EE2031F0882309F49CCF59C082EE8E
:1087C000F8CF811155C0F4E0FF15C0F58FEF9FEF92
:1087D00060E0EF2DF0E09F0122503109462F50E07C
:1087E000D80142175307BCF4A40FB51F4C9184273E
:1087F00048E050E0DC01B695A79580FF06C0CD01AA
:1088000071E0872770EA972701C0CD0141505109D7
:1088100089F76F5FE3CFA20FB31F2C9130E0AC015B
:1088200055274217530709F040C0892F9927EC0FAD
:10883000FD1F208130E082179307B9F58A818530CA
:10884000B0F58330B0F5813090F05B81652F70E03A
:108850007595679520910B0B40E0842F90E086176B
:1088600097070CF452C020930B0B50FD6CC080E0B6
:108870001092050B1092070B1092060B10920A0B28
:10888000D3950FB6F894DEBF0FBECDBFDF91CF9169
:108890001F910F91FF90EF90DF90CF90BF90AF901E
:1088A0009F908F90089581EEE3CF83EEE1CF8731E3
:1088B000F1F66B8170E07595679520910B0B40E0A8
:1088C000842F90E0861797071CF020930B0BCFCFD7
:1088D0004034C0F49C012E5F3F4F220F331F880F9E
:1088E000991FFC01E850F64FDE01A20FB31F8C91D7
:1088F00090E0982F8827D801A20FB31F2C91822BCC
:1089000090878783242F4F5FDBCF4034C8F4880FD4
:10891000991FFC01E850F64FA5E0B0E0AC0FBD1F79
:10892000A80FB91F2C9130E0322F2227A4E0B0E02D
:10893000AC0FBD1FA80FB91F8C91282B3087278340
:10894000242F4F5F8ACF403468F4880F991FFC01B1
:10895000E850F64FDE01A80FB91F14968C9190E0F5
:108960009087878381E0840F80930B0B80CFCF9219
:10897000DF92EF92FF921F93CF93DF93EC016A0196
:108980007B01122FE889F98982E080834115514EDD
:1089900061057105B1F060E079E08DE390E0A70139
:1089A00096010E941E8BDA01C9010197A109B10944
:1089B000B695A795979587959C01211580E1380775
:1089C000A8F0E889F989108260E874E88EE190E007
:1089D000A70196010E941E8BDA01C9010197A10926
:1089E000B109B695A795979587959C01EC85FD856E
:1089F0003083EE85FF852083188EEC89FD891083F6
:108A0000EA89FB89808180618083EA89FB89808192
:108A100088608083EA89FB89808180688083EA8915
:108A2000FB8980818F7D8083DF91CF911F91FF90A3
:108A3000EF90DF90CF9008954F925F926F927F9268
:108A40008F929F92AF92BF92EF92FF920F931F93DC
:108A50004B015C0129013A016E0D7F1D801F911FA2
:108A60002FEF3FEF40E050E00E941E8B641575052C
:108A70008605970570F4481459046A047B0410F4C1
:108A800021E013C021E086169706A806B90668F013
:108A90000BC086169706A806B90630F421E04814E4
:108AA00059046A047B0408F020E0822F1F910F9183
:108AB000FF90EF90BF90AF909F908F907F906F90BE
:108AC0005F904F9008957F928F929F92AF92BF9246
:108AD000CF92DF92EF92FF920F931F93CF93DF938A
:108AE0008C016A017B01722E9A01AB01C701B601AC
:108AF0000E942D8E882319F060EE74E027C0460195
:108B00005701E894B7F82FEF3FEF4FE75FE7C50154
:108B1000B4010E942D8E81110DC02FEF3FEF4FE762
:108B20005FE7C501B4010E940C8C18161CF464EEBA
:108B300074E00CC02FEF3FEF4FE75FE4C701B601D1
:108B40000E946B8D181694F468EE74E0C801DF91F2
:108B5000CF911F910F91FF90EF90DF90CF90BF903A
:108B6000AF909F908F907F900C9446742FEF3FEFC3
:108B70004FE75FECC701B6010E940C8C87FDE4CF84
:108B800020E030E0A901C701B6010E940C8C87FFEC
:108B90000AC06DE2C8010E941B74EC01F7FAF09460
:108BA000F7F8F09402C0C0E0D0E0B12C60E070E0D3
:108BB00080E09FE37B1441F020E030E040E251E4AC
:108BC0000E94118CB394F6CFA70196010E94A08B4E
:108BD0006B017C010E948A8C4B015C012AE0AB0195
:108BE000BC01C8010E945B74C80FD91F7720C1F176
:108BF000C501B4010E94B98C9B01AC01C701B6014B
:108C00000E949F8B6B017C016EE2C8010E941B7465
:108C1000C80FD91F20E030E040E251E4C701B6019F
:108C20000E94708D4B015C010E948A8C6B01E12CCB
:108C3000F12C2AE0B701A601C8010E945B74C80F9D
:108C4000D91FC701B6010E94B98C9B01AC01C501B7
:108C5000B4010E949F8B6B017C017A947110DACF72
:108C6000CE01DF91CF911F910F91FF90EF90DF9098
:108C7000CF90BF90AF909F908F907F9008950F936B
:108C80001F93CF93DF93FC01838594850097C9F0F0
:108C90008B01EF01DC01ED91FC910484F585E02D61
:108CA0001995892B71F08B859C85DC01ED91FC91E8
:108CB0000480F581E02DB801DF91CF911F910F91D4
:108CC000199484E690E0DF91CF911F910F91089560
:108CD000FC0180859185009789F0FC012085223078
:108CE00041F0253059F460E00E94263F009731F0B2
:108CF000FC016185728583859485089560E070E04C
:108D0000CB010895BF92CF92DF92EF92FF920F9323
:108D10001F93CF93DF93EC016A017B0188859985CE
:108D2000892B21F58A819B810E948A3F082F10E0C0
:108D300082E0B82E0530110594F40E942A2B00978A
:108D400031F0FC01B0861186128613861486BC01B0
:108D50008A819B810E94333F0F5F1F4FEBCF64E0FE
:108D60008A819B810E94263F99878887E885F985BB
:108D700080858230F9F4C186D286E386F48667EF77
:108D80007BE084EA98E00E9422742AE030E0B70198
:108D9000A60184EA98E00E94A47484EA98E0DF9136
:108DA000CF911F910F91FF90EF90DF90CF90BF90E8
:108DB0000C944575DF91CF911F910F91FF90EF902B
:108DC000DF90CF90BF900895CF93DF93EC018FE3B6
:108DD00092E0998388837B836A831C861B86CE01FD
:108DE0000E943B23882329F0CE01DF91CF910C9480
:108DF000983FDF91CF91089560E08DE00C9444643A
:108E000061E08DE00C9444642F923F924F925F9208
:108E10006F927F928F929F92AF92BF92CF92DF928A
:108E2000EF92FF920F931F93CF93DF93CDB7DEB7EF
:108E3000C156D1090FB6F894DEBF0FBECDBF009169
:108E40007207109173070115110509F454C580913B
:108E50006E078F5F80936E070E94C57380907807BE
:108E600090907907A0907A07B0907B0786169706B6
:108E7000A806B90608F052C0D80116962D903C906D
:108E8000179721143104D9F1F1018085863089F5D5
:108E900063963FAE2EAE6397CE018F5A9F4F0E94CE
:108EA000D6266596FFAC6597FF2019F167968EADC3
:108EB0009FAD6797892B09F06FC01BC00E94C573D7
:108EC000F8017383628364968FAD649780FF6FC3EC
:108ED0008A149B0471F46796EEADFFAD67976081CD
:108EE00068606083617070E0CE018F5A9F4F0E946E
:108EF0009524D10112962D903C901397C2CF0E94D9
:108F0000C573DC01CB010F96A11DB11D80937807BD
:108F100090937907A0937A07B0937B070E94C5735B
:108F200000917407109175072091760730917707AB
:108F3000061717072807390748F5E0917207F091DF
:108F40007307068117810115110581F0F8018085ED
:108F5000863031F41A830983CE0101960E94D62609
:108F6000D80112960D911C911397EDCF0E94C573F5
:108F7000DC01CB0188579C4EAF4FBF4F80937407E5
:108F800090937507A0937607B093770780916E074B
:108F9000815080936E07AFC464968FAD6497803420
:108FA00009F017C16CEE74E063968EAD9FAD6397C8
:108FB0000E940B3F8C018F2D0E9478655C0101158A
:108FC000110509F4F2C0F8018085853009F0EDC083
:108FD000C8010E948A3F68968FAF6897843008F472
:108FE00079C063E0C8010E94263FDC0119968D918B
:108FF0009C911A974AE0742E789E4001799E900CBD
:10900000112462E0C8010E94263FFC0181859285FF
:10901000789E6001799ED00C1124A296DFAECEAE70
:10902000A2972601DD0C6608770861E0C8010E945E
:10903000263F6C0160E0C8010E94263FDC011996C2
:109040002D913D914D915C911C976C962CAF3DAF4D
:109050004EAF5FAF6C9795010B2C000C440B550B7A
:109060006C968CAD9DADAEADBFAD6C97281B390B2A
:109070004A0B5B0BC401092C000CAA0BBB0BBC01F7
:10908000CD0164197509860997090E940E8BD601D6
:1090900019962D913D914D915C911C976C96CCAC9D
:1090A000DDACEEACFFAC6C972C193D094E095F09A5
:1090B0006C962CAF3DAF4EAF5FAF6C970E94408B6C
:1090C000420E531E641E751E68962FAD689725309C
:1090D00091F414C08AE08A9D20018B9D500C1124CC
:1090E000052C000C66087708A2961FAE1EAEA2974C
:1090F000812C38E2932E81E090E009C064E0C80141
:109100000E94263FDC0119968D919C911A97A4012B
:10911000092C000C660B770B441555056605770581
:1091200034F42A013B01AA24AA9423E0B22EA29689
:10913000CEACDFACA297A601DD0C660B770B441614
:1091400055066606770624F42A013B01A12CB12CB2
:1091500068962FAD6897223009F0BEC24501BB0C5E
:10916000AA08BB0860E0C8010E94263FFC01818577
:109170009285A385B48588169906AA06BB060CF4C9
:109180008BC261E0C8010E94263FFC018185928567
:10919000A385B48588159905AA05BB050CF0A9CE51
:1091A000812C912C540183947AC28AE08A9D2001FB
:1091B0008B9D500C1124052C000C66087708A29694
:1091C0001FAE1EAEA297812C98E2992E81E090E00E
:1091D00083C2813408F044C2843008F08ACE42E071
:1091E00050E06FEFCE018F5A9F4F0E94AC256496DE
:1091F0001FAD64971695117065962FAD659730E099
:10920000F901E553FE4E8491F901EB57FE4E0491AE
:10921000F901E15CFE4EF490FF20A1F081110E9463
:10922000EE63EF2DF0E0EE0FFF1FE956F24FA59130
:10923000B491EC910E2391E080E009F490E0A92E26
:10924000B82E02C0A12CB12C812E912CDD24D394F8
:109250008A149B0409F0D12C6796EEADFFAD679799
:109260008181E82FEF708E2F90E0FC013197EC3078
:10927000F10508F086C18827E051FF4F8F4F0C940D
:10928000818B0E94C5739B01AC01442755276796CB
:10929000EEADFFAD679782819381BC0180E090E0E5
:1092A00018EEE12E13E0F12E00E010E00E941C45C4
:1092B000882309F466C163960EAD1FAD639767E717
:1092C00074E0C8010E940B3F892B09F0CDC16CE707
:1092D00074E0C8010E940B3F892B09F0C5C1D4C0BE
:1092E0000E94C5739B01AC01442755276796EEADDC
:1092F000FFAD679782819381BC0180E090E01CE222
:10930000E12EFF24F39400E010E00E941C45882326
:1093100009F437C142E050E064E0D7C00E94C57351
:109320009B01AC01442755276796EEADFFAD6797CB
:1093300082819381BC0180E090E016E9E12EF12C5E
:1093400000E010E00E941C45882309F41AC142E0A5
:1093500050E064E0E6C00E94C5739B01AC01442765
:1093600055276796EEADFFAD679782819381BC016B
:1093700080E090E018EEE12E13E0F12E00E010E026
:109380000E941C45882309F4FCC063960EAD1FADF6
:10939000639762E874E0C8010E940B3F892B09F0D3
:1093A00067C168E874E0C8010E940B3F892B09F08F
:1093B0005FC16AC00E94C5739B01AC014427552759
:1093C0006796EEADFFAD679782819381BC0180E027
:1093D00090E01CE2E12EFF24F39400E010E00E94F4
:1093E0001C45882309F4CDC042E050E069E06DC01F
:1093F0000E94C5739B01AC01442755276796EEADCB
:10940000FFAD679782819381BC0180E090E016E90F
:10941000E12EF12C00E010E00E941C45882309F4A5
:10942000B0C042E050E069E07CC00E94C5739B017F
:10943000AC01442755276796EEADFFAD6797828153
:109440009381BC0180E090E018EEE12E13E0F12E54
:1094500000E010E00E941C45882309F492C0639646
:109460000EAD1FAD63976FE874E0C8010E940B3F1B
:10947000892B09F001C165E974E0C8010E940B3F26
:10948000892B09F0F9C0FCC042E050E06DE074C0E7
:109490000E94C5739B01AC01442755276796EEAD2A
:1094A000FFAD679782819381BC0180E090E01CE270
:1094B000E12EFF24F39400E010E00E941C45882375
:1094C00009F45FC042E050E06CE0CE018F5A9F4F3C
:1094D0000E94AC2567960EAD1FAD67970E94C573BD
:1094E000D80113967C936E9312974BC00E94C5735C
:1094F0009B01AC01442755276796EEADFFAD6797FA
:1095000082819381BC0180E090E016E9E12EF12C8C
:1095100000E010E00E941C45882399F142E050E0F1
:109520006CE0CE018F5A9F4F0E94AC2567960EAD1E
:109530001FAD67970E94C573F8017383628321C0D2
:109540000E94C5739B01AC01442755276796EEAD79
:10955000FFAD679782819381BC0180E090E018E5C0
:10956000E12E12E0F12E00E010E00E941C4588235D
:1095700041F042E050E060E0CE018F5A9F4F0E94E0
:10958000AC2567960EAD1FAD6797D8018C9183FB14
:10959000992790F9D91609F45EC0982F907E09F4A6
:1095A0008DCC982F907E90528F71892B57C06D2D46
:1095B00070E0CE018F5A9F4F0E9495246796EEADC2
:1095C000FFAD679781818A149B04B1F48F7082305C
:1095D00079F030F4811136C042E050E061E02AC0F9
:1095E000853031F0873071F542E050E06AE022C00A
:1095F00042E050E066E01EC0E82FEF708E2F90E052
:10960000FC013197ED30F105E8F48827E450FF4F75
:109610008F4F0C94818B42E050E062E00BC042E03F
:1096200050E065E007C042E050E067E003C042E080
:1096300050E060E0CE018F5A9F4F0E94AC258823F6
:1096400009F457CC6796EEADFFAD67978081D0FAED
:1096500083F980834ECC8F718066D8018C9349CC7E
:10966000823409F49FCC45CC42E050E063E084CFE3
:1096700042E050E068E080CF42E050E06BE07CCF19
:1096800061E774E0C8010E940B3F892B09F0FCCE12
:1096900042E050E066E070CF812C912C5401679637
:1096A000EEADFFAD679782819381092E000CAA0B66
:1096B000BB0B88159905AA05BB0509F41ACCB401A2
:1096C000CE018F5A9F4F0E9495246796EEADFFAD55
:1096D0006797938282820DCC6796EEADFFAD679758
:1096E000428153819501241B350B37FF03C031950F
:1096F000219531098217930724F480818F7180832B
:1097000012C03081232F229526952770822F90E05A
:1097100006974CF42F5F822F8295880F807E232F2F
:109720002F71282B2083808182958695877090E009
:109730000597BCF0A296CEACDFACA297C601DD0CBB
:10974000AA0BBB0B84159505A605B70551F0C401FE
:10975000990CAA0BBB0B84159505A605B70509F056
:10976000C8CB4A155B0509F4C4CBC301B2010E9402
:10977000BB8C20E030E040E251E40E94118C2B01D0
:109780003C0165961FAD659763EB7DE084EA98E048
:109790000E9422744AE050E0612F84EA98E00E941F
:1097A000F37461EB7DE084EA98E00E94227422E089
:1097B000B301A20184EA98E00E94634584EA98E03C
:1097C0000E9445756396EEACFFAC639762E474E06B
:1097D000C7010E940B3F8C0167E474E0C7010E943F
:1097E0000B3F7C01009791F1DC0118968C91189742
:1097F000843061F519966D917C911A9740E450E0A0
:10980000CE0101960E9404906FE270E0CE010196B5
:109810000E94CB8F892B51F4F7012185328543E0DB
:1098200050E060E4CE0101960E94225CAE014F5BE5
:109830005F4FC301B2010E94B95C0E94C06C8823D3
:1098400029F080916D07882309F44DC00115110599
:1098500009F442C0D80118968C918430E9F520E0D3
:1098600030E0A901C301B2010E946B8D20E030E01D
:1098700040E05FE387FD05C0C301B2010E94A08BF9
:1098800004C0C301B2010E949F8B0E94838C239667
:109890007FAF6EAF2397F80161857285CE01019687
:1098A0000E940740CE0101960E943B23882381F04D
:1098B000C12CD12CE12CF12C01E09E012F5B3F4FFC
:1098C00041E050E060E070E0CE0101960E948B0A1A
:1098D000CE0101960E9497406796EEADFFAD679767
:1098E000B382A28206CBBE016F5B7F4FCE01019691
:1098F0000E94FA3EABCFCF59DF4F0FB6F894DEBFD0
:109900000FBECDBFDF91CF911F910F91FF90EF90D0
:10991000DF90CF90BF90AF909F908F907F906F908F
:109920005F904F903F902F900895A8950E941E142D
:10993000029724F00E94563C0E9404470C94422750
:1099400080916D078F5F80936D07A8950E940447F3
:1099500080916D07815080936D07089565E77DE0E4
:1099600084EA98E00E94227462E67DE084EA98E04E
:109970000E94227464E57DE084EA98E00E942274EB
:109980006CE47DE084EA98E00E94227484EA98E026
:109990000E9445756FE37DE084EA98E00E9422749E
:1099A0006FE27DE084EA98E00E94227463E27DE049
:1099B00084EA98E00E9422746CE07DE084EA98E0FA
:1099C0000E9422746AEF7CE084EA98E00E9422748C
:1099D00065EE7CE084EA98E00E94227466ED7CE00B
:1099E00084EA98E00E94227467EC7CE084EA98E0C4
:1099F0000E9422746FEB7CE084EA98E00E9422745B
:109A000064EB7CE084EA98E00E9422746AEA7CE0DD
:109A100084EA98E00E94227462EA7CE084EA98E09A
:109A20000E94227466E97CE084EA98E00E94227435
:109A30006CE77CE084EA98E00E9422746DE57CE0AB
:109A400084EA98E00E94227468E47CE084EA98E06A
:109A50000E9422746BE37CE084EA98E00E94227406
:109A60006DE27CE084EA98E00E94227461E27CE08E
:109A700084EA98E00E94227465E17CE084EA98E040
:109A80000E94227484EA98E00C9445752F923F92CC
:109A90004F925F926F927F928F929F92AF92BF92FE
:109AA000CF92DF92EF92FF920F931F93CF93DF93AA
:109AB000CDB7DEB7C555D1090FB6F894DEBF0FBEDE
:109AC000CDBF80916E078F5F80936E07E0916F0727
:109AD000F09170073097B1F0E680F780C0906F0783
:109AE000D0907007C114D10469F0E114F10451F071
:109AF000F70180858530B1F7C7010E948A3F823027
:109B000088F3B8C180916E07815080936E07809171
:109B10006B0790916C07039709F4E3C40E94C57327
:109B2000C0908007D0908107E0908207F090830773
:109B3000C616D706E806F90608F0D3C466961FAE27
:109B4000669766246394712C60917E0770917F07FD
:109B50006115710509F4C5C46696FFAD6697F111EC
:109B6000C0C4FB018085853009F069C1CE01CA9669
:109B70000E94E44625968FAD2597883009F40AC1E6
:109B8000893009F4DBC0843009F030C180917C0752
:109B900090917D07892B09F0CAC060E074E0CE0186
:109BA000CA960E943624892BC1F0CE01CA960E9423
:109BB00080236B017C0162E27EE084EA98E00E94EF
:109BC000227460E074E0CE01CA960E94C423B601FC
:109BD000CE01CA960E94C834AAC0CEACDFACF60152
:109BE0008085853009F05FC1C6010E948A3F882EBA
:109BF000912CF2E08F1691040CF455C170927D0700
:109C000060927C0760E070E0CE01CA960E949A23C1
:109C10005C0161E070E0CE01CA960E949A237C014B
:109C2000F5E08F1691040CF4ACC164E0C6010E940B
:109C3000263FFC01C184D28426E240E855E260E080
:109C400070E087E098E00E94B744A092FA0987E0AC
:109C500098E09093F9098093F8091092050B1092FF
:109C6000070B1092060BF1E0CF16D10409F43CC1AA
:109C70000CF420C192E0C916D10409F027C1F0927A
:109C8000FC09E092FB097092FE096092FD0983E0F5
:109C90000E940042182F111158C1C090FF09D090A6
:109CA000000AC6010D2C000CAA0BBB0B89839A83FA
:109CB000AB83BC8380E190E09E838D83ECADFDADF2
:109CC0008080918064E57EE084EA98E00E942274BE
:109CD000B40184EA98E00E9449756DE47EE084EA6C
:109CE00098E00E942274BE016F5F7F4F84EA98E083
:109CF0000E9485240E944575B601CE01CA960E9435
:109D0000BA3980907E0790907F07F4016281738159
:109D1000CE0101960E94E446892809F0F6C0CE01E2
:109D200001960E94974010927D0710927C07CE0109
:109D3000CA960E94513A80ED97E062C080917C07FC
:109D400090917D07892B99F7CE01CA960E947824BD
:109D5000E82E60E074E0CE01CA960E943624892B7A
:109D600009F430C1CE01CA960E948023F62E61E12B
:109D70007EE084EA98E00E94227460E074E0CE0104
:109D8000CA960E94C4234E2D6F2DCE01CA960E9402
:109D90001534CDCF80917C0790917D07892B39F6C2
:109DA000CE01CA960E947824E82E60E074E0CE01CD
:109DB000CA960E943624892B09F4B9CFCE01CA96DF
:109DC0000E948023F62E67EB7DE084EA98E00E94F3
:109DD000227460E074E0CE01CA960E94C4234E2D26
:109DE0006F2DCE01CA960E940333A1CFCE01CA9631
:109DF0000E94513A61E070E0CE01CA960E943F464F
:109E00006C01990FEE08FF08C114D104E104F104BC
:109E100091F00E94C573C60ED71EE81EF91EC092AF
:109E20008007D0928107E0928207F0928307F1E0E9
:109E30006696FFAF6697CE01CA960E949740E09162
:109E40007E07F0917F07309709F44BC3828193819D
:109E500090937F0780937E07892B09F075CEE09160
:109E60006F07F09170078681978190937F078093A9
:109E70007E0737C3B701CE0101960E94E446CE01AA
:109E800001960E943B23882331F062E070E0CE010E
:109E900001960E943F46F701E280F380CE010196D1
:109EA0000E9497401BCE61E77EE084EA98E00E9422
:109EB00022743DCFCD2811F5F092FC09E092FB0908
:109EC0007092FE096092FD0981E0E2CEE3E0CE16D9
:109ED000D104A1F4F092FC09E092FB097092FE0912
:109EE0006092FD0984E0D4CEF092FC09E092FB0977
:109EF000D092FE09C092FD0982E0CACE69E57EE0FB
:109F000084EA98E00E942274C6CECE0101960E9497
:109F10003B23882309F403CF8B85843009F0FFCEDF
:109F200060E070E0CE0101960E949A23A816B9065F
:109F300009F0F5CE61E070E0CE0101960E949A230F
:109F4000E816F90609F0EBCE20C0812F90E0A0E0E2
:109F5000B0E089839A83AB83BC8380E190E09E83E9
:109F60008D8367E37EE084EA98E00E942274BE015C
:109F70006F5F7F4F84EA98E00E9485240E944575B8
:109F8000D2CE82E0C82ED12C57CEB601CE0101969A
:109F90000E94BA39E0917E07F0917F078281938118
:109FA00090937F0780937E07892B09F0B8CEE091CC
:109FB0006F07F09170078681978190937F07809358
:109FC0007E07ADCE70927D0760927C070E942A2B9F
:109FD0005C01892B19F086E0F501808720E030E0F4
:109FE00043E050E060E2CE0101960E94225CECADBD
:109FF000FDAD608171814FE150E0CE0101960E947C
:10A00000E68F60EF74E0CE0101960E94C08F26E0DB
:10A0100040E855E260E070E087E098E00E94B744D5
:10A0200060E070E0CE01CA960E949A238093FA09FC
:10A0300087E098E09093F9098093F8091092050B56
:10A040001092070B1092060B84E398E09093FC09A2
:10A050008093FB09EAE0F0E0F093FE09E093FD094C
:10A0600083E00E9400428111C5C067E07EE084EA7F
:10A0700098E00E9422743FEF832E39E0932E43E153
:10A08000E42E4AE0F42E50E1C52ED12CF40181914A
:10A0900091914F01092E000CAA0BBB0B89A39AA327
:10A0A000ABA3BCA3DEA2CDA2BE016F5D7F4F84EA4D
:10A0B00098E00E94852465E07EE00E942274E81406
:10A0C000F90421F784EA98E00E9445756091030A3B
:10A0D0007091040A072E000C880B990B0E94BB8C10
:10A0E00020E030E048EC52E40E94118C9B01AC016E
:10A0F00066EF74E0C5010E946F3AE090070AF090A5
:10A10000080AA70168EF74E0C5010E94503F609102
:10A11000090A70910A0A072E000C880B990B0E94FD
:10A12000BB8C20E030E048EC52E40E94118C9B0193
:10A13000AC016CEF74E0C5010E946F3A60910B0AAC
:10A1400070910C0A072E000C880B990B0E94BB8C97
:10A1500020E030E040E251E40E94118C9B01AC0110
:10A160006AEF74E0C5010E946F3A4091FF09509177
:10A17000000A6EEF74E0C5010E94503FEF2809F419
:10A1800053C08EAD9FADFC012085253009F04CC039
:10A1900061E00E94263F009709F446C0FC0120853B
:10A1A000243009F041C024E630E065963FAF2EAF81
:10A1B000659761857285CE0181960E940740CE0128
:10A1C00081960E943B23882381F0C12CD12CE12C65
:10A1D000F12C01E09E012D5A3F4F41E050E060E03C
:10A1E00070E0CE0181960E948B0ACE0181960E947A
:10A1F00097401AC090E0A0E0B0E089A39AA3ABA377
:10A20000BCA380E190E09EA38DA36FEE7DE084EA85
:10A2100098E00E942274BE016F5D7F4F84EA98E04F
:10A220000E9485240E9445758091FF0983FF37C0F5
:10A230008EE398E09093FC098093FB097092FE09ED
:10A240006092FD0983E00E940042811109C04091A3
:10A25000FF095091000A61E075E0C5010E94503F7E
:10A2600010927D0710927C07CE01CA960E94883515
:10A27000181619067CF4C12CD12CE12CF12C01E02C
:10A2800020E030E040E050E062E070E0CE01CA96AD
:10A290000E948B0A70927D0760927C0707C040E0A5
:10A2A00050E061E075E0C5010E94503F62E370E05C
:10A2B00080E090E00E94976583E190E09093FC0934
:10A2C0008093FB09E4E0F0E0F093FE09E093FD09E0
:10A2D00083E00E9400428111ACC065EE7DE084EA1B
:10A2E00098E00E9422749FEFE92E99E0F92E27E072
:10A2F000C22E2AE0D22EF701619171917F014AE0CE
:10A3000050E084EA98E00E94EC7463EE7DE084EA19
:10A3100098E00E942274CE14DF0469F784EA98E082
:10A320000E944575E090FF09F090000AE114F104E5
:10A33000D1F0B7010F2C000C880B990B0E94BB8C3D
:10A340002DEE3EE94CE35EE30E94708D22E538EB92
:10A3500042E152E40E949F8B9B01AC0165E075E0F5
:10A36000C5010E946F3A6091010A7091020A072E9E
:10A37000000C880B990B0E94BB8C2DEE3EE94CE340
:10A380005EE30E94708D22E538EB42E152E40E94C8
:10A390009F8B1B012C019B01AC0164EF74E0C50194
:10A3A0000E946F3A6091050A7091060A1616170608
:10A3B000A4F4072E000C880B990B0E94BB8C20E0A4
:10A3C00030E040E251E40E94118C9B01AC0169E055
:10A3D00075E0C5010E946F3A07C040E050E069E0B7
:10A3E00075E0C5010E94503F20E030E040E252E4B9
:10A3F000C201B1010E946B8D18169CF5EF2889F1FE
:10A400000E94C06C882329F080916D07882309F48D
:10A4100059C0C12CD12CE12CF12C01E020E030E01E
:10A4200040E050E062E070E0CE01CA960E948B0AE4
:10A4300018C090E0A0E0B0E089A39AA3ABA3BCA3AE
:10A4400080E190E09EA38DA36DEC7DE084EA98E02E
:10A450000E942274BE016F5D7F4F84EA98E00E94E3
:10A46000852480E091E00E94CF807C01892BD9F087
:10A470001CA21BA21EA21DA28FEF9FEF98A78FA365
:10A48000E7EAF2E0FAA3E9A31AA619A6FCA6EBA64E
:10A4900080E091E098AB8FA71EA61DA6B501CE0166
:10A4A00081960E94CF7C0E94C06C882321F080910D
:10A4B0006D07882381F0C7010E946781C5010E9452
:10A4C000BD3A31CCECADFDAD608171818DE095E0A0
:10A4D0000E94AC3A9ECFB701CE0101960E94AC3AE1
:10A4E000EACFCB5ADF4F0FB6F894DEBF0FBECDBF19
:10A4F000DF91CF911F910F91FF90EF90DF90CF9060
:10A50000BF90AF909F908F907F906F905F904F9093
:10A510003F902F900895CF92DF92EF92FF920F938A
:10A520001F93CF93DF936C01EB0109900020E9F7B3
:10A530002197C61BD70BC032D10514F0CFE1D0E074
:10A540008B01E12CF12CEC16FD0664F4F80161910D
:10A550008F01C7018C0D9D1D0E94008BFFEFEF1A2C
:10A56000FF0AF1CF60E0C6018C0F9D1FDF91CF91F4
:10A570001F910F91FF90EF90DF90CF900C94008B84
:10A58000CF93DF931F92CDB7DEB71982892B21F0CD
:10A59000FB016281738103C0BE016F5F7F4F86E361
:10A5A00090E00E948B5269E27FE084EA98E00E948A
:10A5B00022740F90DF91CF910895CF93DF93C0E085
:10A5C000D0E060E0CE010E94008B2196C11582E0B0
:10A5D000D807B9F769E17FE084EA98E0DF91CF918D
:10A5E0000C942274EF92FF920F931F93CF93DF93FB
:10A5F0001F92CDB7DEB78B01CE0101969F938F934B
:10A6000083EA9BE09F938F9382EA9BE09F938F93D3
:10A6100081EA9BE09F938F9380EA9BE09F938F93C7
:10A620008FE99BE09F938F938EE99BE09F938F939D
:10A630008AE195E09F938F93FB0183818F938281C1
:10A640008F930E948A900FB6F894DEBF0FBECDBFE5
:10A6500006977CF4F801028113816BE37FE084EAC2
:10A6600098E00E942274B80184EA98E00E9449753B
:10A6700019C00E94F52F8EE9E82E8BE0F82E00E03D
:10A6800010E0F70161917F01C8010E94008B0F5F0C
:10A690001F4F06301105A9F76DE47FE084EA98E0CA
:10A6A0000E9422740F90DF91CF911F910F91FF9024
:10A6B000EF900895EF92FF920F931F93CF93DF9344
:10A6C000CDB7DEB72C970FB6F894DEBF0FBECDBF67
:10A6D0008C017B0186EC93E09A8389831B821C8228
:10A6E0001D821E8298878F8319861A861B861C8678
:10A6F000053011055CF0BE01695F7F4FF701808571
:10A7000091850E94E863892B09F052C0BE016F5FFA
:10A710007F4F82E190E00E94C963043011050CF480
:10A720004FC0BE01695F7F4FF701868197810E940C
:10A73000E863892B09F444C0BE01695F7F4F8EE056
:10A7400090E00E94C963BE01695F7F4FF701848179
:10A7500095810E94E863892BF1F1BE01695F7F4F0B
:10A760008AE090E00E94C963BE01695F7F4FF701F4
:10A77000828193810E94E863892BC1F1BE01695FE8
:10A780007F4F86E090E00E94C96362E07FE084EA48
:10A7900098E00E9422742C960FB6F894DEBF0FBE8C
:10A7A000CDBFDF91CF911F910F91FF90EF90089552
:10A7B000BE01695F7F4F82E190E00E94C963B1CF23
:10A7C000BE016F5F7F4F8EE090E00E94C96303304F
:10A7D00011050CF0B8CFBE016F5F7F4F8AE090E0AB
:10A7E0000E94C963023011050CF0BECFBE016F5F3D
:10A7F0007F4F86E090E00E94C9630130110529F681
:10A80000BE016F5F7F4F86E090E00E94C96369E000
:10A810007FE084EA98E00E942274B7CFCF93DF9361
:10A82000CDB7DEB72C970FB6F894DEBF0FBECDBF05
:10A830001C821B821E821D828FEF9FEF98878F8361
:10A8400084EE92E09A83898388E490E09A878987EE
:10A850001C861B8668EE7EE084EA98E00E942274E3
:10A860006091880770918907CE0101960E94CF7C84
:10A870006FEFCE0101960E94D72868ED7EE084EA52
:10A8800098E00E9422742C960FB6F894DEBF0FBE9B
:10A89000CDBFDF91CF9108950F931F93CF93DF9397
:10A8A000CDB7DEB769970FB6F894DEBF0FBECDBF48
:10A8B0008FE290E09A838983FE01339687E1DF017E
:10A8C0001D928A95E9F763EC7EE084EA98E00E94A5
:10A8D00022742EE93BE0DE011196AE01435F5F4F2B
:10A8E0008D01F90161919F01862F90E074E09595AB
:10A8F00087957A95E1F781539D4FFC0180811196F0
:10A900008C931197E62FEF70F0E0E153FD4F8081BB
:10A9100012968C9312971296A417B50711F71E86FC
:10A920006EE275E0C8010E94C08FB80184EA98E029
:10A930000E944975C8010E94A26E1E8666E375E0FA
:10A94000C8010E94C08FB80184EA98E00E9449754E
:10A9500060E475E0C8010E94AC3A69960FB6F894BD
:10A96000DEBF0FBECDBFDF91CF911F910F91089534
:10A97000AF92BF92CF92DF92EF92FF920F931F930D
:10A98000CF93DF936C017B018A010E94F88A81508A
:10A990008E3FA0F45701C0E0D0E001501109C0176C
:10A9A000D1077CF4C6018C0F9D1F0E94F88AF50127
:10A9B00081935F01882329F02196F1CF80E090E018
:10A9C00005C0CE0DDF1D188281E090E0DF91CF91B0
:10A9D0001F910F91FF90EF90DF90CF90BF90AF90BD
:10A9E0000895882319F066E57FE002C068E57FE0FE
:10A9F00084EA98E00C942274CF93DF93CDB7DEB74E
:10AA00002C970FB6F894DEBF0FBECDBF68EA7EE08C
:10AA100084EA98E00E94227484EA98E00E944575D6
:10AA200088E490E00E94F88A8B37A1F51C821B8293
:10AA30001E821D828FEF9FEF98878F8384EE92E0B6
:10AA40009A83898388E490E09A8789871C861B868D
:10AA50000E944830CE0101960E94E83A90938907FF
:10AA600080938807892B19F46BE87EE015C064E8B1
:10AA70007EE084EA98E00E94227484EA98E00E94D2
:10AA800045750E948F7682E19BE00E94686981E0B3
:10AA900090E00CC067E97EE084EA98E00E942274AE
:10AAA00084EA98E00E94457580E090E02C960FB60D
:10AAB000F894DEBF0FBECDBFDF91CF910895AF9266
:10AAC000BF92CF92DF92EF92FF920F931F93CF939B
:10AAD000DF93CDB7DEB7C058D1090FB6F894DEBF0B
:10AAE0000FBECDBF8E010F5B1F4FD8011D921C9270
:10AAF000FE01ED5BFF4F2EE1DF011D922A95E9F784
:10AB00000297CCF0FB01628173814FE150E0C801F4
:10AB10000E940490B80186E190E00E948B52B80137
:10AB200084EA98E00E94497566E470E184EA98E05E
:10AB30000E9422741BC040E250E0B80186E190E020
:10AB40000E94B854892BB1F440E250E06AE370E10E
:10AB5000C8010E94F4836CE170E184EA98E00E94ED
:10AB60002274B80184EA98E00E94497584EA98E06A
:10AB70000E9445758091A30B1F928F938091A20B29
:10AB80001F928F938091A10B1F928F938091A00BA6
:10AB90001F928F9380919F0B1F928F9380919E0B9A
:10ABA0001F928F9382E495E09F938F931F9280E48E
:10ABB0008F93CE0101966C019F938F930E941E90FC
:10ABC00068E070E184EA98E00E942274B80184EAA7
:10ABD00098E00E944975B60184EA98E00E944975A0
:10ABE00084EA98E00E9445750FB6F894A895809184
:10ABF0006000886180936000109260000FBE7E014B
:10AC000091E6E90EF11CD70113961C921E92129741
:10AC100088EE93E0A0E0B0E0F70184839583A683FB
:10AC2000B78388E0848784EA93E0918380831687E2
:10AC30000587108A178680E590E0928B818B158AB4
:10AC400062E679E28DE59BE20E944D848C010FB6AD
:10AC5000F894DEBF0FBECDBF892BE1F183E090E019
:10AC60000E94CF80D8011D969C938E931C97FC0167
:10AC7000F182E0821282C7010E944469882319F0A0
:10AC8000C7010E946869D7011F966D917C9150970A
:10AC90005196AD90BC9052976115710569F0CE0147
:10ACA00089589F4F0E944B75A501BE0169587F4F7F
:10ACB000C7010E94646A07C0F70165857685A50112
:10ACC000C7010E942D5D181619060CF498C0C80122
:10ACD0000E94362B00E010E0F701E388F48899E247
:10ACE00088E10FB6F894A895809360000FBE90930A
:10ACF00060000115110509F469C0F8ECEF16F104C4
:10AD000009F056C06CEF7FE084EA98E00E9422745C
:10AD1000EB961FAE1EAEEB97ED961FAE1EAEED97F7
:10AD20008FEF9FEFEF969FAF8EAFEF978AEF92E096
:10AD3000E9969FAF8EAFE997C158DF4F198308831B
:10AD4000CF57D040F8940E944830CE0189589F4F89
:10AD50000E94E83A90938907809388077894C80105
:10AD60000E94362B8091880790918907892B79F46E
:10AD700065EE7FE084EA98E00E9422740E94C57329
:10AD8000DC01CB018856954CAF4FBF4F2DC06AED0B
:10AD90007FE084EA98E00E9422740E948F7663ED3F
:10ADA0007FE084EA98E00E94227482E090E0C7C0CD
:10ADB0006BEB7FE084EA98E00E9422744AE050E066
:10ADC000B70184EA98E00E94EC7406C068EA7FE06C
:10ADD00084EA98E00E9422740E94C573DC01CB01D2
:10ADE00088579C4EAF4FBF4F809384079093850741
:10ADF000A0938607B093870785EF9FEFA0C0D70188
:10AE00001D96BC901D971E96AC90DF92CF9284EA5F
:10AE10009FE09F938F931F930F930E94D684DF929E
:10AE2000CF928FE99FE09F938F931F930F930E9480
:10AE3000D684D8011C96ED91FC911D9781E0828308
:10AE4000DF92CF928CE99FE09F938F931F930F9394
:10AE50000E94D684D8011C96ED91FC911D97128218
:10AE6000AF92BF9286E69FE09F938F931F930F93BD
:10AE70000E94D68481EA9FE09F938F931F930F9344
:10AE80000E94D684F701148A138AD8011C96ED918A
:10AE9000FC911D97A080B1800FB6F894DEBF0FBE65
:10AEA000CDBF83E3C82ED12CD501ED91FC91008458
:10AEB000F185E02DC501199541975CF4B1E0CB1AFD
:10AEC000D10839F064E170E080E090E00E9497657D
:10AED000EBCF6E01F7E7CF0ED11CDF92CF928AE560
:10AEE0009FE09F938F931F930F930E94F3840F9083
:10AEF0000F900F900F900F900F90019709F0ECCEEC
:10AF0000F60180819181D70154969C938E9353973B
:10AF1000D12C80E08A3039F4BAE0DB1609F4DCCEBB
:10AF20009AE0D92E03C08D3009F0D82EC8010E94B6
:10AF300098848F3F79F7C8010E94362BCDCEC05838
:10AF4000DF4F0FB6F894DEBF0FBECDBFDF91CF91BC
:10AF50001F910F91FF90EF90DF90CF90BF90AF9037
:10AF600008950E945F5590936C0780936B0782E170
:10AF70009BE00C946869DC01ED91FC91028CF38DEF
:10AF8000E02D199591E089270895CF93DF931F92C3
:10AF9000CDB7DEB789832091FA073981E091FB07AD
:10AFA000F091FC07822F90E080959095F8940080B6
:10AFB000082200824BE000C05DE000005A95E9F7EE
:10AFC000008008220894379508F4022A00824A95E6
:10AFD00099F778940F90DF91CF91089585ED809344
:10AFE000BC008091BC0084FDFCCF1092D407089572
:10AFF0004091B007262F30E0240F311D213231055A
:10B00000DCF42091D4072430C9F4FC0180E090E006
:10B01000861758F43091B0072191DC01A057B84F42
:10B02000A30FB11D2C930196F3CF8091B007680F49
:10B030006093B00780E0089581E0089582E008956C
:10B0400008958FEF9FEF08958FEF9FEF0895809100
:10B050008F0790E09195819591090895CF93DF93A3
:10B06000CB01EA01642F0E94F857CE01DF91CF9106
:10B070000895CF93DF931F92CDB7DEB7698361E068
:10B08000CE0101960E94F85781E090E00F90DF9189
:10B09000CF91089583E090E008950C9467816F92BA
:10B0A0007F928F929F92AF92BF92CF92DF92EF9258
:10B0B000FF920F93CF93DF93EC016B014A0159018B
:10B0C0008A819B810E9488353C011C141D0434F444
:10B0D000E114F10419F4EE24E394F12C60E070E142
:10B0E0008A819B810E94FE2381E0E816F10409F425
:10B0F00040C0E2E0EE16F10451F0E114F10409F071
:10B10000C5C062E870E184EA98E00E942274A1144C
:10B11000B10409F4C5C0892809F4C2C0F5018080D2
:10B120009180092C000CAA08BB08B501A4018A81F2
:10B130009B810E9448238A819B81EF28A9F41614E1
:10B14000170434F489288A288B2859F462E007C050
:10B15000672839F489288A288B2819F061E00E9431
:10B160004D2460E07BE071C060E07AE00E94C33073
:10B170008AC06C2D8A819B810E944D24F1E0CF16FC
:10B18000D10431F082E0C816D10409F45AC07EC05F
:10B19000AA80BB80C5010E9480236B017C016115E0
:10B1A00071058105910561F0693171058105910590
:10B1B0003CF4002329F088E2C82ED12CE12CF12C9C
:10B1C000B701A601C5010E944823C114D104E104BE
:10B1D000F104D9F0002331F060E073E08A819B81B3
:10B1E0000E94C33067E770E184EA98E00E9422740D
:10B1F0002AE030E0B701A60184EA98E00E94A47436
:10B2000084EA98E00E94457524C02AE030E040E0DE
:10B2100050E0BA0184EA98E00E94A47469E570E104
:10B2200084EA98E00E94227444E650E060E070E016
:10B230008A819B810E944823002359F060E073E0DB
:10B2400004C0002331F060E071E08A819B810E949C
:10B25000C3308A819B810E946846672B682B692BCB
:10B2600091F00E94C5734F8158856A01550FEE0811
:10B27000FF08AB01BC014C0D5D1D6E1D7F1D8A8159
:10B280009B810E94824681E090E00CC06DE470E1F9
:10B2900084EA98E00E94227484EA98E00E9445754E
:10B2A00080E090E0DF91CF910F91FF90EF90DF90E1
:10B2B000CF90BF90AF909F908F907F906F900895A8
:10B2C0009B018295880F807E68E0680FC9010C940D
:10B2D0004F2C24E030E0AC0164E08FE090E00C946F
:10B2E000D72C24E030E0AC0164E085E090E00C94E1
:10B2F000D72C24E030E0AC0164E081E090E00C94D5
:10B30000D72C78941F920F920FB60F9211240BB680
:10B310000F92CF92DF92EF92FF920F931F932F9392
:10B320003F934F935F936F937F938F939F93AF93CD
:10B33000BF93CF93DF93EF93FF93809170008E7F45
:10B34000809370000FE310E08BE1E82EF12C9BE27C
:10B35000C92ED12CC091FD07D091FE072097F9F49A
:10B360000332110508F43BC003521109E091FB07B9
:10B37000F091FC0790812091FA07822F8095982305
:10B3800090839BE0D7011197F1F79150D9F7808115
:10B39000822B8083C6010197F1F780E00DC00B304E
:10B3A0001105E8F00B501109E091FF07F09100083A
:10B3B000EC0FFD1F319780810E94C5572196D093D5
:10B3C000FE07C093FD0780910102909102028C1745
:10B3D0009D0708F0BFCF1092FE071092FD078091E5
:10B3E0007000816080937000FF91EF91DF91CF91A9
:10B3F000BF91AF919F918F917F916F915F914F918D
:10B400003F912F911F910F91FF90EF90DF90CF9080
:10B410000F900BBE0F900FBE0F901F90189581E0FC
:10B4200080938E0780910002282F30E0F901E15CC3
:10B43000FE4EE491F0E0EE0FFF1FEB5DFE4E4591F6
:10B4400054915093FC074093FB07F901EB57FE4ED4
:10B45000E491E093FA0761E00E94736483E08093D3
:10B46000B100E0E7F0E08081816080830895CF93B0
:10B47000DF931816190644F0809170008E7F809338
:10B48000700010928E0719C0EC018091FF07909117
:10B4900000080E946781CE01C130D24014F080E0E4
:10B4A00092E090930202809301020E94CF809093D9
:10B4B00000088093FF07892B29F410920202109252
:10B4C000010208C080918E07811104C0DF91CF91E5
:10B4D0000C940F5ADF91CF910895FF920F931F9311
:10B4E000CF93DF938C01F62E80918E07811102C0DD
:10B4F0000E940F5AE8012197C11582E0D80798F4FD
:10B5000080910102909102028017910718F4C801FE
:10B510000E94375A8091FF0790910008009719F018
:10B52000C80FD91FF882DF91CF911F910F91FF9023
:10B5300008951F920F920FB60F9211240BB60F921F
:10B540002F933F934F935F936F937F938F939F932B
:10B55000AF93BF93EF93FF938091B900887F8036BC
:10B5600009F49CC068F5883209F45BC090F480311E
:10B5700009F454C038F4882309F4F2C0883009F47F
:10B580004DC0F2C0883109F44CC0803209F45DC06E
:10B59000EBC0803409F468C048F4803309F455C026
:10B5A000883309F0E1C08093D307D4C0803509F413
:10B5B0004FC0883509F45DC0883409F0D5C0D2C0C9
:10B5C000883909F4C3C0A8F4883709F467C038F48F
:10B5D000883609F463C0803709F460C0C5C0883874
:10B5E00009F4B4C0803909F45FC0803809F0BCC0E8
:10B5F0005BC0803B09F484C038F4803A09F466C02B
:10B60000883A09F47DC0B0C0803C09F4A3C0883CEE
:10B6100009F4A0C0883B09F486C0A6C08091F90750
:10B6200010C09091F8078091F707981770F5E09196
:10B63000F80781E08E0F8093F807F0E0E952F84FA9
:10B6400080818093BB0085EC82C08093D3078AC041
:10B65000E091F80781E08E0F8093F8078091BB009E
:10B66000F0E0E952F84F80839091F8078091F70756
:10B670006AC0E091F80781E08E0F8093F80780910F
:10B68000BB00F0E0E952F84F80838091D60781112A
:10B6900069C081E08093D50784EA5DC083E0809330
:10B6A000D4071092D207CFCF8091D207803208F012
:10B6B0004DC0E091D20781E08E0F8093D207809138
:10B6C000BB00F0E0EE54F84F8083BDCF85EC809353
:10B6D000BC001092D4078091D207803230F4E09100
:10B6E000D207F0E0EE54F84F10826091D20770E07C
:10B6F00082EB97E0E0E0F0E019951092D20734C0B9
:10B7000084E08093D4071092B1071092B007E0E074
:10B71000F0E019958091B007811105C081E0809318
:10B72000B00710929007E091B10781E08E0F8093EF
:10B73000B107F0E0E057F84F80818093BB00909113
:10B74000B1078091B007981708F47DCF85E8809302
:10B75000BC000AC085EC8093BC001092D40704C0E2
:10B760001092D3070E94EE57FF91EF91BF91AF91D6
:10B770009F918F917F916F915F914F913F912F9109
:10B780000F900BBE0F900FBE0F901F9018958F92C9
:10B790009F92AF92BF92CF92DF92EF92FF920F9360
:10B7A0001F93CF93DF93CDB7DEB72B970FB6F894E7
:10B7B000DEBF0FBECDBF8C01CE0101967C016C01B6
:10B7C0008AE0882E912CA12CB12CC6018E199F09DC
:10B7D000411551056105710581F0CB01BA01A50143
:10B7E00094010E941E8B942F852F605DF60161935A
:10B7F0006F01A901692F782FE8CFFC013197EE0D79
:10B80000FF1DD8019E012150310940814D93319790
:10B81000E217F307D1F7F801E80FF91F10822B9612
:10B820000FB6F894DEBF0FBECDBFDF91CF911F9151
:10B830000F91FF90EF90DF90CF90BF90AF909F90CF
:10B840008F9008958F929F92AF92BF92CF92DF9286
:10B85000EF92FF920F931F93CF93DF938C014A01D6
:10B860005901E0908C07F0908D07C62F660FDD0B15
:10B87000E114F10461F1F7018085863041F561E75B
:10B8800075E0C7010E940B3F6C01F2E08F16910436
:10B8900039F083E08816910451F46AEE75E002C035
:10B8A00066E775E0C7010E940B3F7C0102C0E12CF6
:10B8B000F12CC114D10469F0F6018085843049F47B
:10B8C00061857285AE01C8010E94049008C0E12C18
:10B8D000F12CAE016CE970E1C8010E94F483AE0165
:10B8E00060E474E0C8010E94E68FE114F10439F0CD
:10B8F000F7018085843019F4618572850FC0F2E00C
:10B900008F169104A1F083E08816910461F08A9467
:10B91000892899F460918A0770918B07AE01C8015C
:10B920000E94E68F0AC0AE0166E970E103C0AE0175
:10B9300063E970E1C8010E94D683AE0160E474E05F
:10B94000C8010E94E68FA114B10429F0AE01B5012F
:10B95000C8010E94E68FC801DF91CF911F910F911E
:10B96000FF90EF90DF90CF90BF90AF909F908F901F
:10B970000895CF92DF92EF92FF920F931F93CF9390
:10B98000DF936B017C01EA010E94838C8B011F9382
:10B990006F9389EB94E09F938F93DF93CF930E94F3
:10B9A0005B900F900F900F900F900F900F9020E0F2
:10B9B00030E0A901C701B6010E946B8D181624F072
:10B9C000F7FAF094F7F8F09409900020E9F721973E
:10B9D0008EE28883B80117FF03C0719561957109E4
:10B9E000072E000C880B990B0E94BB8C9B01AC01AD
:10B9F000C701B6010E949F8B20E030E040E251E495
:10BA00000E94708D0E94838C605D69831A82DF9131
:10BA1000CF911F910F91FF90EF90DF90CF900895FD
:10BA2000CF93DF931F921F92CDB7DEB780910F0C9B
:10BA30009091100C009711F48BE19CE0BE016F5FB8
:10BA40007F4F681B790B072E000C880B990B0F900A
:10BA50000F90DF91CF9108950895AF92BF92CF924A
:10BA6000DF92EF92FF920F931F93CF93DF93CDB7A7
:10BA7000DEB7AF970FB6F894DEBF0FBECDBF7C0127
:10BA80005B016A0106EC13E01A8309831B821C82A6
:10BA90001D821E82CE0109960E94B26B1BA70AA7C7
:10BAA0001CA61DA61EA61FA680914C0990914D09AB
:10BAB000A0914E09B0914F098EA39FA3A8A7B9A743
:10BAC0008B839C83AD83BE8318861F82AE01465D47
:10BAD0005F4FB501CE0101960E94D165813091057D
:10BAE000B1F4D701ED91FC910684F785E02D1DA3FB
:10BAF0000CA38CA59DA5AEA5BFA58EA39FA3A8A7AB
:10BB0000B9A7A601BE016C5D7F4FC7011995AF961D
:10BB10000FB6F894DEBF0FBECDBFDF91CF911F915E
:10BB20000F91FF90EF90DF90CF90BF90AF9008956E
:10BB300080910508909106080895CF93DF93EC015A
:10BB40006BE775E084EA98E00E94233B60E08C811B
:10BB50000E94446460E08D810E94446440E050E0B3
:10BB6000BA018A819B810E94824610920608109237
:10BB7000050881E090E0DF91CF910895FC0182817A
:10BB800093810E948023CB0108954F925F926F9220
:10BB90007F928F929F92AF92BF92CF92DF92EF925D
:10BBA000FF920F931F93CF93DF93EC010A811B81C8
:10BBB00060E070E1C8010E943624892B09F48FC12E
:10BBC00060E070E2C8010E943624892B79F48091EC
:10BBD0000302882309F483C160E070E2C8010E9477
:10BBE000FE23809103028150809303020A811B810E
:10BBF000C8010E9468466B017C01C8010E9478243C
:10BC0000823049F018F4813049F00DC0853019F0C8
:10BC1000863021F008C000E010E007C0C8010E9493
:10BC200080238B0102C00FEF1FEF8E819AEC980FDB
:10BC3000903158F549845A84612C712C8B849C84F2
:10BC4000A12CB12C0E947865092E000CAA0BBB0B0D
:10BC50009C01AD01281939094A095B09A4E6B0E045
:10BC60000E945F8BA3019201281939094A095B09D7
:10BC70000E94408B590137FD27C1253631050CF450
:10BC800025C184E6A82EB12C21C1C114D104E10440
:10BC9000F104D1F0AA24AA94BA2C0E94C573C61646
:10BCA000D706E806F90658F46DEF70E184EA98E0EB
:10BCB0000E94227484EA98E00E944575DEC08FEFEE
:10BCC000A816B80609F008C1025311090E3F8FEFFC
:10BCD00018070CF05DC060E08D810E9444648A8189
:10BCE0009B810E946846672B682B692B91F40E9408
:10BCF000C5734F8158856A01550FEE08FF08AB01E7
:10BD0000BC014C0D5D1D6E1D7F1D8A819B810E94B3
:10BD10008246FC808EEF8F0D8C3020F084ED8F0DED
:10BD2000833038F4AA27BB27A01BB10B2FEF30E0DC
:10BD30005DC08D819EEF980F61E09C3020F08C52A9
:10BD4000833008F096C08F2D0E9444642227332749
:10BD5000201B310BA1E0BFEF0E94908B2AE030E066
:10BD600040E050E00E94408BDA01C90181509F4FB2
:10BD7000AF4FBF4FBC018F3F910509F02CF497FFE7
:10BD800005C060E070E002C06FEF70E08D816EC0B2
:10BD9000033011050CF471C060E08C810E94446492
:10BDA0008A819B810E946846672B682B692B91F4DE
:10BDB0000E94C5734F8158856A01550FEE08FF0830
:10BDC000AB01BC014C0D5D1D6E1D7F1D8A819B81E9
:10BDD0000E948246FD808EEF8F0D8C3020F084ED26
:10BDE0008F0D8330C8F42FEF30E0D8010E94988B7C
:10BDF0002AE030E040E050E00E94408BB9012F3F44
:10BE0000310509F02CF437FF05C060E070E002C096
:10BE10006FEF70E08F2D2AC08C819EEF980F61E04C
:10BE20009C3018F08C52833020F58F2D0E94446492
:10BE30009801A1E0BFEF0E94908B2AE030E040E043
:10BE400050E00E94408BDA01C90181509F4FAF4FF3
:10BE5000BF4FBC018F3F910509F02CF497FF05C03F
:10BE600060E070E002C06FEF70E08C810E94AF6410
:10BE700036C08F2D0E94446432C069E875E084EAC0
:10BE800098E00E94233B60E08C810E94446460E063
:10BE90008D810E94446440E050E0BA018A819B8118
:10BEA0000E94824660E070E18A819B810E94C423E7
:10BEB00060E070E28A819B810E94C423809103022A
:10BEC0008F5F809303020BC0A12CB12CC114D1044D
:10BED000E104F10409F0E1CE0A191B09F7CE80E074
:10BEE00090E0DF91CF911F910F91FF90EF90DF9045
:10BEF000CF90BF90AF909F908F907F906F905F900A
:10BF00004F9008950F931F93CF93DF93EC010A8115
:10BF10001B8160E070E0C8010E949A239FEF980F98
:10BF2000953408F080E28C8361E070E0C8010E94E3
:10BF30009A239FEF980F953408F081E28D8362E099
:10BF400070E0C8010E949A23863410F48E8301C0E9
:10BF50001E8263E070E0C8010E949A239C01215078
:10BF600031092115344018F49A87898702C01A864E
:10BF7000198664E070E0C8010E949A23813024E0B1
:10BF8000920710F080E094E09C878B8765E070E07A
:10BF9000C8010E949A231816190614F080E197E24E
:10BFA00098878F83DF91CF911F910F910895CF9341
:10BFB000DF93EC010E94825F60E975E084EA98E01B
:10BFC0000E94233B61E08C810E94736461E08D815B
:10BFD0000E94736460E08C810E94446460E08D8103
:10BFE0000E94446460E08E810E94736440E050E0EF
:10BFF000BA018A819B810E94824660E070E18A8159
:10C000009B810E94C42360E070E28A819B810E9430
:10C01000C42381E090E0909306088093050882E0B5
:10C020008093030281E090E0DF91CF9108952F92F9
:10C030003F924F925F926F927F928F929F92AF92B8
:10C04000BF92CF92DF92FF920F931F93CF93DF9314
:10C05000CDB7DEB7C855D1090FB6F894DEBF0FBE15
:10C06000CDBF0E94C5730091010810910208209174
:10C07000030830910408601771078207930708F4DA
:10C0800028C2E0916F07F0917007309709F421C240
:10C0900080916E078F5F80936E0706811781F12C68
:10C0A0000115110541F1F8018085853001F560E049
:10C0B000C8010E94263FFC0181859285A385B48535
:10C0C0000597A105B10599F4C8010E948A3F90E047
:10C0D00005976CF064E0C8010E94263F6C01892B33
:10C0E00031F0C6010E948A3F823008F05CC0F8013E
:10C0F00002811381D5CF80916E07815080936E07A6
:10C100000E94C573DC01CB01805D9A48AF4FBF4FE1
:10C110008093010890930208A0930308B093040849
:10C120000E94105D2B013C010E94C5734B015C0114
:10C130000E94C06C882329F080916D07882309F440
:10C1400065C1FF20C1F00E94105D4B015C016EEBE8
:10C1500070E184EA98E00E9422742AE0B501A4010B
:10C1600084EA98E00E945B7464EC75E084EA98E0ED
:10C170000E944975AEC10E94105D4B015C016CEBE1
:10C1800070E184EA98E00E9422742AE0B501A401DB
:10C1900084EA98E00E945B746AEB70E184EA98E0BC
:10C1A0000E94227496C161E0C8010E94263FFC01F2
:10C1B000F184328462E0C8010E94263FFC01418480
:10C1C00052846384748463E0C8010E94263FFC01AA
:10C1D000218532854385548567962CAF3DAF4EAFA0
:10C1E0005FAF679760E0C6010E94263FFC01818433
:10C1F0009284A384B48461E0C6010E94263FFC01BE
:10C200004185528563857485411551056105710528
:10C2100071F4F8016081718184EA98E00E944975A7
:10C2200063EF70E184EA98E00E94227414C04150E8
:10C23000510961097109FC0141875287638774873D
:10C24000452B462B472B39F4F801608171818BE92E
:10C2500095E00E94AC3A20E030E048E152E4C501AC
:10C26000B4010E946B8D18163CF4F8016081718155
:10C270008DE095E00E94AC3A6296FFAE62976396BD
:10C280003FAE6397C301B2010E94BB8C2B013C01FE
:10C2900065962EAC3FAC6597F8010190F081E02DDA
:10C2A0006996FFAFEEAF699784EA98E00E94457502
:10C2B00069966EAD7FAD699784EA98E00E944975F2
:10C2C0006DEE70E184EA98E00E94227422E0B301EE
:10C2D000A20184EA98E00E94634567EE70E184EA77
:10C2E00098E00E94227422E0B501A40184EA98E05B
:10C2F0000E94634561EE70E184EA98E00E94227436
:10C300004AE050E065966EAD7FAD659784EA98E0AF
:10C310000E94EC7463962EAD3FAD639761E08F2D64
:10C3200037FD81950E94736461E0C6010E94263F3B
:10C33000FC0181859285A385B485892B8A2B8B2B63
:10C3400089F0F6E02F163104F1F024F42A94232822
:10C3500049F419C04AE024163104A9F05CE025161E
:10C36000310489F063962EAD3FAD639737FF04C06B
:10C3700060E08F2D819502C060E08F2D0E944464A3
:10C380006CED70E11DC020E030E040E85FE3C301E8
:10C39000B2010E949F8B9B01AC01C501B4010E94B8
:10C3A0000C8C87FF17C063968EAD9FAD639797FF88
:10C3B0000EC060E08F2D81950E94446468ED70E1AD
:10C3C00084EA98E00E942274FF24F39490CE61E006
:10C3D0008F2DF2CFA5019401C301B2010E940C8CF4
:10C3E00018168CF06396EEADFFAD6397F7FF04C0AF
:10C3F00061E08F2D819502C060E08F2D0E94446422
:10C4000063ED70E1DDCF64EC70E1DACF20E030E085
:10C4100041E050E060E4CE0101960E94225C40E4DD
:10C4200050E063EB70E1CE0101960E94D68360E498
:10C4300074E0CE0101960E94C08F40E450E06AEAA9
:10C4400070E1CE0101960E94D683B301A201CE0114
:10C450008F5B9F4F0E94C75BBE016F5B7F4FCE011A
:10C4600001960E94FA3E20E030E041E050E060E4B6
:10C47000CE0101960E94225C40E450E063EB70E143
:10C48000CE0101960E94D68360E474E0CE0101964D
:10C490000E94C08F40E450E063EA70E1CE01019653
:10C4A0000E94D683C501B40128EE33E040E050E09D
:10C4B0000E941E8BBA01A901CE018F5B9F4F0E9483
:10C4C000C75BBE016F5B7F4FCE0101960E94FA3EB3
:10C4D00038CEC85ADF4F0FB6F894DEBF0FBECDBFBF
:10C4E000DF91CF911F910F91FF90DF90CF90BF9080
:10C4F000AF909F908F907F906F905F904F903F9004
:10C500002F900895FC0140E050E020E030E08AE008
:10C510009191992301F1243031055CF59E3271F43B
:10C520004F3F510509F02CF5DB01A20FB31F129606
:10C530004C932F5F3F4F40E050E0EACF849FD00103
:10C54000859FB00D1124492F990F550B4053510968
:10C550004A0F5B1FDDCF4F3F510509F054F42430E3
:10C5600031053CF4FB01E20FF31F428381E090E0D0
:10C57000089580E090E00895CF92DF92EF92FF92CD
:10C58000CF93DF93CDB7DEB768970FB6F894DEBFD1
:10C590000FBECDBFFA0126EC33E03A8329835FEF6B
:10C5A0005B835C835D831E8238872F83C280D38048
:10C5B000E480F580C986DA86EB86FC863E872D8787
:10C5C000FB0142815381648175814F87588B698B50
:10C5D0007A8B3C8B2B8BFC0182819381A481B5816A
:10C5E0008D8B9E8BAF8BB88F9E012F5F3F4FAE011F
:10C5F000495F5F4FBE01635F7F4FCE0143960E944C
:10C60000E26E68960FB6F894DEBF0FBECDBFDF9125
:10C61000CF91FF90EF90DF90CF9008950F931F93ED
:10C62000CF93DF93CDB7DEB768970FB6F894DEBF30
:10C630000FBECDBFFB01DC0112964D915D916D9156
:10C640007C9115974D8B5E8B6F8B788F86EC93E08A
:10C650009A83898321E0288F0D891E892F89388D3F
:10C660000B831C832D833E8398878F8302811381E4
:10C670002481358109871A872B873C879E878D8780
:10C680004F87588B698B7A8BAE014F5F5F4FBE012E
:10C69000695F7F4FCE010D960E94BC6268960FB60F
:10C6A000F894DEBF0FBECDBFDF91CF911F910F91E8
:10C6B0000895CF93DF93CDB7DEB762970FB6F894A6
:10C6C000DEBF0FBECDBFFC0182819381A481B58105
:10C6D0008F87988BA98BBA8B26EC33E03A8329831A
:10C6E00041E04A8B4F85588969897A894B835C83FD
:10C6F0006D837E8338872F8389879A87AB87BC8732
:10C70000BE016F5F7F4FCE0107960E940E63629657
:10C710000FB6F894DEBF0FBECDBFDF91CF91089565
:10C72000CF92DF92EF92FF920F931F93CF93DF93FD
:10C730006C01EB017B0182E0E80EF11C00E010E0EF
:10C74000C601800F911F0E94F88AF70181937F0133
:10C750000F5F1F4F0430110599F78A81882361F01C
:10C760008F3F61F48B818F3F49F48C818F3F31F48F
:10C7700081E09D819F3F19F480E001C081E090E05D
:10C78000DF91CF911F910F91FF90EF90DF90CF90AD
:10C790000895EF92FF920F931F93CF93DF937C0145
:10C7A0008B010E5F1F4FC0E0D0E0F80161918F0157
:10C7B000C7018C0F9D1F0E94008B2196C430D105AC
:10C7C000A1F7DF91CF911F910F91FF90EF90089506
:10C7D000FC0121912111FDCF0C94826290E0FC01BB
:10C7E0003197E231F10508F04EC08827E75FFE4F30
:10C7F0008F4F0C94818B809180008F7703C0809144
:10C8000080008F7D80938000089580918000877FD5
:10C81000F9CF84B58F7702C084B58F7D84BD08952C
:10C820008091B0008F7703C08091B0008F7D80939E
:10C83000B0000895809190008F7707C0809190009C
:10C840008F7D03C080919000877F80939000089532
:10C850008091A0008F7707C08091A0008F7D03C0DA
:10C860008091A000877F8093A0000895809120018F
:10C870008F7707C0809120018F7D03C080912001B8
:10C88000877F8093200108951F93CF93DF93282FF4
:10C8900030E0F901E553FE4E8491F901EB57FE4E6D
:10C8A000D491F901E15CFE4EC491CC23C1F0162F66
:10C8B00081110E94EE63EC2FF0E0EE0FFF1FEB5DA5
:10C8C000FE4EA591B4919FB7F894111104C08C91BC
:10C8D000D095D82302C0EC91DE2BDC939FBFDF9173
:10C8E000CF911F910895CF93DF9390E0FC01EB5718
:10C8F000FE4E2491FC01E15CFE4E8491882361F19F
:10C9000090E0880F991FFC01E55FFE4EC591D49120
:10C91000FC01EB5DFE4EA591B491611109C09FB77A
:10C92000F8948881209582238883EC912E230BC074
:10C93000623061F49FB7F8948881322F3095832359
:10C940008883EC912E2B2C939FBF06C08FB7F89451
:10C95000E8812E2B28838FBFDF91CF9108951F93FD
:10C96000CF93DF93182FEB0161E00E94736420974F
:10C9700011F460E004C0CF3FD10539F461E0812FAC
:10C98000DF91CF911F910C944464E12FF0E0E553C7
:10C99000FE4EE4918E2F90E0FC013197E231F105DB
:10C9A00008F09DC08827E55EFE4F8F4F0C94818B69
:10C9B00084B5806884BDC7BD97C084B5806284BDDE
:10C9C000C8BD92C080918000806880938000D09321
:10C9D0008900C093880088C0809180008062809325
:10C9E0008000D0938B00C0938A007EC0809180002D
:10C9F000886080938000D0938D00C0938C0074C0B9
:10CA00008091B00080688093B000C093B3006CC088
:10CA10008091B00080628093B000C093B40064C085
:10CA200080919000806880939000D0939900C0938B
:10CA300098005AC080919000806280939000D093BB
:10CA40009B00C0939A0050C08091900088608093B2
:10CA50009000D0939D00C0939C0046C08091A000A0
:10CA600080688093A0008091A0008F7B8093A000BD
:10CA7000D093A900C093A80037C08091A000806225
:10CA80008093A000D093AB00C093AA002DC08091EA
:10CA9000A00088608093A000D093AD00C093AC004C
:10CAA00023C080912001806880932001D0932901C8
:10CAB000C093280119C080912001806280932001D9
:10CAC000D0932B01C0932A010FC080912001886070
:10CAD00080932001D0932D01C0932C0105C0C03854
:10CAE000D1050CF04BCF45CFDF91CF911F91089529
:10CAF000863308F0865390917B00282F2870977F0B
:10CB0000922B90937B008770806480937C0080914F
:10CB10007A00806480937A0080917A0086FDFCCF51
:10CB2000809178002091790090E0922B08958F9267
:10CB30009F92AF92BF92CF92DF92EF92FF926B01E2
:10CB40007C010E94A0734B015C01C114D104E1047B
:10CB5000F104F1F00E94A073DC01CB01881999095E
:10CB6000AA09BB09883E9340A105B10570F321E0F5
:10CB7000C21AD108E108F10888EE880E83E0981EF9
:10CB8000A11CB11CC114D104E104F10419F7DDCFDB
:10CB9000FF90EF90DF90CF90BF90AF909F908F90DD
:10CBA00008954F925F926F927F928F929F92AF9271
:10CBB000BF92CF92DF92EF92FF920F931F93CF938A
:10CBC000DF93CDB7DEB763970FB6F894DEBF0FBE25
:10CBD000CDBF7C015B012A01FB0181918111FDCF59
:10CBE000B201C5010E948262892B09F04DC1F70193
:10CBF00042815381648175818091430990914409F8
:10CC0000A0914509B0914609481759076A077B0763
:10CC100009F43DC10E94C5738701085F1F4F6F7003
:10CC200077277C5FC8010E941669813009F017C11F
:10CC300086EC93E09A838983F70182819381A481B2
:10CC4000B5818B839C83AD83BE8345E350E0BE01F9
:10CC50006F5F7F4FC8010E94C968892B19F4C12CEE
:10CC6000D12CF9C00E94C573F7017783668342E037
:10CC700050E0B7016A5F7F4FC8010E94402A81E0FF
:10CC800090E09A83898342E050E0BE016F5F7F4F5E
:10CC9000C8010E94402A80E091E09A83898342E0A3
:10CCA00050E0BE016F5F7F4FC8010E94402A1A8288
:10CCB000198242E050E0BE016F5F7F4FC8010E94C1
:10CCC000402A42E050E0BE016F5F7F4FC8010E94E2
:10CCD000402A42E050E0BE016F5F7F4FC8010E94D2
:10CCE000402A4501F5018081882301F16401560144
:10CCF000F60181913F01882321F08E3211F063010A
:10CD0000F6CFC818D9081C141D0474F4CD8641E070
:10CD100050E0BE01635F7F4FC8010E94402AA60118
:10CD2000B401C8010E94402A4301DCCF1D8641E0C6
:10CD300050E0BE01635F7F4FC8010E94402AC12CB2
:10CD4000DD24D394DA82C98242E050E0BE016F5FF5
:10CD50007F4FC8010E94402ADA82C98242E050E037
:10CD6000BE016F5F7F4FC8010E94402AC8010E9428
:10CD7000A068892B09F473CFE3E0AE2EB12C22E03A
:10CD8000420E511C0E94C5733B014C01C8010E9418
:10CD9000C02D18161906B4F00E94C573DC01CB0132
:10CDA00086199709A809B90989389341A105B105E0
:10CDB000E0F462E370E080E090E00E9497650E94FA
:10CDC000A04CE4CFF7014281538164817581818D4C
:10CDD000928DA38DB48D481759076A077B0749F4D4
:10CDE000858D968DC59729F409C0CC24CA94DC2C76
:10CDF00029C09EEFC92EDD24DA9424C0F70181A159
:10CE000092A10C970CF41FC14CE050E0BE016F5F83
:10CE10007F4FC8010E94782D8B819C81982789279C
:10CE200098279A8B898BF7014681578129813A810E
:10CE30004217530779F1C8010E94C5287CEFC72E1D
:10CE4000DD24DA9481E0A81AB10829F0FFEFCF16AB
:10CE5000DF0609F497CFC8010E94086902C0C12CFF
:10CE6000D12C67EA75E084EA98E00E9449754AE0AF
:10CE700050E0B60184EA98E00E94EC7484EA98E0FD
:10CE80000E944575C601E4C081E090E0E1C08EEFEC
:10CE90009FEFDEC097FFCFCF8F709270892B41F04C
:10CEA000C8010E94C5286BEFC62EDD24DA94CACFD4
:10CEB0006F8078847624672476246114710419F0D5
:10CEC000C12CD12C25C0C8010E94C5285AEFC52EFF
:10CED000DD24DA94B7CF41E050E0BE01635F7F4FBD
:10CEE000C8010E94782D8D8581111BC08D8581110F
:10CEF000F2CFC8010E94972DC8010E94972DC8014A
:10CF00000E94972DC8010E94972DFFEFCF1ADF0ACC
:10CF10008D819E81982789279827C816D906D8F22F
:10CF20000AC08D859FEF980F9D878823F9F2C8016D
:10CF30000E94972DF6CF812C912C41E050E0BE014C
:10CF40006D5E7F4FC8010E94782D8B89982F907C51
:10CF500061F4882389F08B899FEF980F9B8B88233E
:10CF600041F0C8010E94972DF6CFC8010E94972D6D
:10CF70001B8A8B898111E1CF42E050E0BE01615FE5
:10CF80007F4FC8010E94782D42E050E0BE01635FF0
:10CF90007F4FC8010E94782DC8010E94972DC801BB
:10CFA0000E94972DC8010E94972DC8010E94972DBD
:10CFB00042E050E0BE016F5E7F4FC8010E94782DB5
:10CFC0008F8598898115914049F4CD84DE84DC24D5
:10CFD000CD24DC2481E0C816D10419F0C12CD12C59
:10CFE00014C089899A898115944041F0C8010E9432
:10CFF000C52847EFC42EDD24DA9424CF44E050E066
:10D00000B201C8010E94782D1DCF89899A8998277D
:10D0100089279827C816D90638F4C8010E94972D89
:10D02000FFEFCF1ADF0AF1CF2FEF821A920A6814AE
:10D03000790409F082CFC8010E94C52836EFC32EBB
:10D04000DD24DA94FFCE8DEFC82EDD24DA94FACEFB
:10D0500063960FB6F894DEBF0FBECDBFDF91CF91C0
:10D060001F910F91FF90EF90DF90CF90BF90AF9006
:10D070009F908F907F906F905F904F900895CF9387
:10D08000DF931F92CDB7DEB76983DC01ED91FC9190
:10D090000280F381E02D41E050E0BE016F5F7F4FE1
:10D0A00019950F90DF91CF910895FC01818D928D9C
:10D0B0000895FC0185899689089526EC33E0FC01EA
:10D0C00031832083FB014189528963897489FC0182
:10D0D00042835383648375830895DC01ED91FC9151
:10D0E000048CF58DE02D199480E00895FC01948561
:10D0F000FB018485981303C081E0983009F480E037
:10D10000089521E0FC018485883009F420E0822F15
:10D1100008950895CF93DF931F92CDB7DEB769834B
:10D12000DC01ED91FC910280F381E02D41E050E0C3
:10D13000BE016F5F7F4F19950F90DF91CF910895DA
:10D14000CF93FC01C48560E270E08C2F0E94133BFA
:10D1500062E070E08C2F0E94605984FD10C062E094
:10D1600070E08C2F0E94605983FFF2CF48E162E0AB
:10D1700070E08C2F0E94112E80E090E008C040E10A
:10D1800062E070E08C2F0E94112E81E090E0CF9140
:10D1900008951F93CF93DF93FB01DC0158961C92F7
:10D1A0001E9257972281211109C02381211106C0A7
:10D1B0002481211103C02581222321F1411551052C
:10D1C00009F1EA01DC011C961C91AF014E5F5F4F33
:10D1D000612F6295660F607E645F24E030E08CE032
:10D1E00090E00E94D72C4D2F60E170E0812F0E94CB
:10D1F000112E4C2F61E170E0812F0E94112E81E0F1
:10D2000090E002C080E090E0DF91CF911F910895FF
:10D21000CF93DF93FC018485883029F0EF010E94D1
:10D220001A2E88E08C87DF91CF910895EF92FF92BC
:10D230001F93CF93DF93FC012485283011F080E009
:10D240001DC07B01EC0110E063E070E0812F0E94C3
:10D250006059811102C01C8705C08831E1F31F5F4E
:10D26000183091F78C85883051F3FE86ED861A8E42
:10D27000198EA70162E00E946F6E81E0DF91CF916D
:10D280001F91FF90EF900895CF93DF93FC012485C9
:10D290002830D1F0EC010E94093B843181F08823D1
:10D2A00071F0883161F08C3161F4E881F98100849A
:10D2B000F185E02DCE01199521E0892B19F420E0AC
:10D2C00001C021E0822F01C080E0DF91CF9108955D
:10D2D000CF92DF92EF92FF92CF93DF93EC018C8598
:10D2E0008830B9F168E070E00E94133B0E94C5737A
:10D2F0006B017C01CE010E94093B8823A1F00E94B2
:10D30000C573DC01CB018C199D09AE09BF09883EAC
:10D310009340A105B10538F461E070E080E090E051
:10D320000E949765E7CFCE010E94093B882319F040
:10D330008C850E941A2E88E08C876CEA75E084EA5E
:10D3400098E0DF91CF91FF90EF90DF90CF900C9419
:10D35000233BDF91CF91FF90EF90DF90CF90089526
:10D360000F931F93CF93DF931F92CDB7DEB78C013E
:10D37000DC01ED91FC910084F185E02D1995892B5C
:10D3800069F021E041E050E0BE016F5F7F4FF8019E
:10D3900084850E944F3E898190E002C08FEF9FEF0D
:10D3A0000F90DF91CF911F910F910895FC0184851B
:10D3B0000C943B2DCF93DF931F92CDB7DEB741E0A6
:10D3C00050E0BE016F5F7F4FFC0184850E943B2DC2
:10D3D000181619061CF4898190E002C08FEF9FEFA8
:10D3E0000F90DF91CF910895FC018485883011F072
:10D3F0000C948E3E80E090E008958F929F92AF92C1
:10D40000BF92CF92DF92EF92FF920F931F93CF9331
:10D410006C015B017A01FC01C485C83041F481E0F4
:10D4200090E0F6019383828380E090E041C08A011E
:10D430004130584010F000E018E08C2F0E94536EED
:10D440004C0163E070E08C2F0E946059873111F02D
:10D450008C3121F48016910680F302C000E010E0C8
:10D460009801A50160E070E08C2F0E94146E60E2CC
:10D4700070E08C2F0E94133B62E070E08C2F0E94C2
:10D48000605984FD0BC063E070E08C2F0E946059EE
:10D490008111F2CF8C2F0E941A2EC1CF40E162E0A1
:10D4A00070E08C2F0E94112E012B09F4B8CFC70118
:10D4B000CF911F910F91FF90EF90DF90CF90BF9091
:10D4C000AF909F908F9008958F929F92AF92BF924E
:10D4D000CF92DF92EF92FF920F931F93CF93DF9340
:10D4E000EC018B017A016C85683069F04AE050E00C
:10D4F00084EA98E00E94F37463EB75E084EA98E0B4
:10D500000E94233B12C184EA98E00E944575C12C19
:10D51000D12CAC2C63E070E08C2D0E946059B82EA9
:10D5200062EC75E084EA98E00E94497540E150E0C1
:10D53000B60184EA98E00E94EC7466EC75E084EA37
:10D5400098E00E94497540E150E06B2D84EA98E034
:10D550000E94F37484EA98E00E944575B11013C0EC
:10D56000AC866FEC75E084EA98E00E94497540E172
:10D5700050E06C8584EA98E00E94F37484EA98E0B5
:10D580000E9445750CC08B2D8B7F883149F38FEF3E
:10D59000C81AD80AE8E0CE16D10409F0BACF8C85B3
:10D5A000883009F4C2C0C0900402D0900502FFEF99
:10D5B000CF1ADF0A0E94C573DC01CB019927AA2785
:10D5C000BB27B601680F791F611584E0780728F042
:10D5D000709305026093040206C080E094E090938B
:10D5E000050280930402409104025091050261E01B
:10D5F0008C850E946F6E6801E2E0CE0ED11C460160
:10D600005801F6E0AF0EB11CF40161914F014AE000
:10D6100050E084EA98E00E94F37468ED75E084EAD3
:10D6200098E00E944975A814B90471F784EA98E05B
:10D630000E944575F80182818F3F51F483818F3FAD
:10D64000A1F484818F3F89F485818F3F71F46BC091
:10D6500081110BC0F8018381811107C08481811180
:10D6600004C08581882309F45EC0E114F10409F443
:10D670005AC01C85612F6295660F607E645F24E04E
:10D6800030E0A6018CE090E00E94D72C4F2D60E1A5
:10D6900070E0812F0E94112E4E2D61E170E0812FEC
:10D6A0000E94112E64E070E0812F0E94133B0E94C3
:10D6B000C5734B015C016B017C01F8E9CF0EFAE305
:10D6C000DF1EE11CF11CCE010E94093B873129F0CD
:10D6D0008C149D04AE04BF0420F00E94C57397FD16
:10D6E00015C00E94C5736C157D058E059F0570F0F1
:10D6F00066EE75E084EA98E00E94233BE881F981B8
:10D700000488F589E02DCE0119950FC06AE070E01C
:10D7100080E090E00E9497650E94A04CCE010E949C
:10D72000093B811105C088E08C8780E090E00DC046
:10D73000CE010E94093B873131F66AED75E084EA3B
:10D7400098E00E94233B81E090E0DF91CF911F9110
:10D750000F91FF90EF90DF90CF90BF90AF909F9090
:10D760008F900895FC011382128288EE93E0A0E06E
:10D77000B0E084839583A683B78380E193E09183AF
:10D78000808388E0848786EC93E0908B8787118A7A
:10D79000128A138A148A0895AF92BF92CF92DF92B1
:10D7A000EF92FF920F931F93CF93DF93CDB7DEB726
:10D7B000AF970FB6F894DEBF0FBECDBF7C015B0103
:10D7C0006A0106EC13E01A8309831B821C821D8206
:10D7D0001E82CE0109960E94B26B1BA70AA71CA647
:10D7E0001DA61EA61FA680914C0990914D09A091DF
:10D7F0004E09B0914F098EA39FA3A8A7B9A78B8309
:10D800009C83AD83BE8318861F82AE01465D5F4F49
:10D81000B501CE0101960E94D16581309105B1F428
:10D82000D701ED91FC910488F589E02D1DA30CA38F
:10D830008CA59DA5AEA5BFA58EA39FA3A8A7B9A79C
:10D84000A601BE016C5D7F4FC7011995AF960FB65B
:10D85000F894DEBF0FBECDBFDF91CF911F910F9126
:10D86000FF90EF90DF90CF90BF90AF900895CF934F
:10D87000DF93EC01FA013296E60FF71FDC01AD01F0
:10D880004C1B5D0BCF01861B970B2D91222311F0B2
:10D890002193F5CF9C01241B350B620F731FFB01F5
:10D8A0003297508331964083DF91CF910895EF9264
:10D8B000FF920F931F93CF93DF9300D01F92CDB7AA
:10D8C000DEB77B01BA0130E0962F9F77660F672F96
:10D8D000661F770B71956115710509F0906821E05D
:10D8E000230FE1E0F0E0EC0FFD1FE30FF11D90834B
:10D8F0006115710511F0322FE7CF30E0B701621BDF
:10D90000730B6C5F7F4FDB018C93DE011196F70187
:10D91000E21BF30B359685E0E80EF11CEE16FF06D0
:10D9200019F08D918193FACF80915B0990915C09F8
:10D930002F5F3F4F8901040F151FDC01ED91FC9112
:10D940000280F381E02DA80119957C010E94C57326
:10D950006093DF097093E0098093E1099093E209F5
:10D9600081E00E151F0509F080E00F900F900F90D9
:10D970000F90DF91CF911F910F91FF90EF9008953D
:10D9800080915B0990915C09009779F1DC01ED9140
:10D99000FC910688F789E02D19952091F6093091C0
:10D9A000F70981111FC0232B01F58DEF9FEF909395
:10D9B000F7098093F60980915B0990915C09DC017D
:10D9C000ED91FC910680F781E02D199580915B091E
:10D9D00090915C09DC01ED91FC910488F589E02DC2
:10D9E000199503C081E0232B09F080E0089520E31E
:10D9F000FC0120833296862F82958F7090E1899F5B
:10DA0000601911246A3014F4605D01C0695C62938E
:10DA1000682F8111F0CF08957F928F929F92AF92DD
:10DA2000BF92CF92DF92EF92FF920F931F93CF930B
:10DA3000DF93CDB7DEB7A6970FB6F894DEBF0FBE63
:10DA4000CDBF8C01762E942E852E20E2B22ECE01F3
:10DA500001967C01FC012B2D11922A95E9F786ECA9
:10DA600093E09AA389A38FEF8BA38CA38DA38EA39E
:10DA700068018BE4C80ED11C43E450E0BE016F5D29
:10DA80007F4FC6010E94C968019609F4B9C081E0C0
:10DA900089838A8386E0A82EAB821C82F801648188
:10DAA0007581868197810E94898B6D837E838F83A8
:10DAB000988789869A8680E890E09C878B874CE1DE
:10DAC00050E0B701C6010E94402AF7012B2D1192A8
:10DAD0002A95E9F7480188E0880E911CF401D701E6
:10DAE00001900D92AA94E1F740E150E0B701C60120
:10DAF0000E94402AF7011192BA94E9F796E0A92E04
:10DB0000B12C40E250E0B701C6010E94402AF1E08A
:10DB1000AF1AB108B1F783E6898392E89A8393E557
:10DB20009B838C8385E38D8381E08E837F829DE35D
:10DB3000988797E099878A8786E0F401DE011B9633
:10DB400001900D928A95E1F78CE0898B8A8B6EEEBD
:10DB500075E0CE0143960E94DF8FF8016385CE0108
:10DB600049960E94F76CF8016485CE014B960E949D
:10DB7000F76CF8016585CE014D960E94F76C4EE179
:10DB800050E0B701C6010E94402AF3E07F121EC098
:10DB900082E3898384E08A83F80196859B83978555
:10DBA0009C8390899D8391899E8396E39F83888738
:10DBB000868D8987878D8A8780A18B8781A18C87B5
:10DBC0004CE050E0B701C6010E94402A87E38983F8
:10DBD00086E08A8391E09B8393E09C838D838FE032
:10DBE0008E838AE38F838BE388878FEF898749E071
:10DBF00050E0B701C6010E94402AC6010E94A068F9
:10DC0000A6960FB6F894DEBF0FBECDBFDF91CF91C1
:10DC10001F910F91FF90EF90DF90CF90BF90AF904A
:10DC20009F908F907F900895AF92BF92CF92DF9296
:10DC3000FF920F931F93CF93DF93F82E8B015A011E
:10DC4000690164E270E00E946059C82F65E270E0EB
:10DC50008F2D0E946059D0E0DC2FCC27080F111DBA
:10DC6000C00FD11F6F2D6295660F607E6C5E9601AE
:10DC7000A501CE010E94D72CCC0DDD1D4D2F64E2F5
:10DC800070E08F2D0E94112E4C2F65E270E08F2DD9
:10DC9000DF91CF911F910F91FF90DF90CF90BF90B8
:10DCA000AF900C94112EFF920F931F93CF93DF939D
:10DCB000F82E00E010E08F2D0E94222DEC01892B20
:10DCC00021F08F2D0E94222D8C01C017D10799F7CA
:10DCD000CE01DF91CF911F910F91FF9008950F9387
:10DCE0001F93CF93DF93C82FD62F8A010E941A2E3D
:10DCF0004D2F60E070E08C2F0E94112E0115110550
:10DD000051F40091A40B1091A50B0F5F1F4F1093BE
:10DD1000A50B0093A40B412F64E070E08C2F0E94B0
:10DD2000112E402F65E070E08C2F0E94112E61E0D3
:10DD300070E08C2F0E94133B81E0DF91CF911F9107
:10DD40000F910895CF93DF93FC0101900020E9F734
:10DD50009F01281B390B285F3F4F2138310570F593
:10DD6000EC010E94C06C882349F18091DD099091FB
:10DD7000DE09019611F481E090E09093DE09809332
:10DD8000DD098091DD099091DE099093620980930D
:10DD9000630947E050E06DE579E0CE010E94376C01
:10DDA000FC01E95AF64F1682AC01445051096DE569
:10DDB00079E082E8DF91CF910C94576C80E0DF919D
:10DDC000CF910895CF92DF92EF92FF920F931F931E
:10DDD000CF93DF936C01EB017A01890180915609A1
:10DDE0008093490980910602882319F00E94712CC2
:10DDF00006C06DE274E084EA98E00E94233B26E0CE
:10DE000030E04EE95BE064E089E090E00E94D72CCE
:10DE1000C60102960E946959C70102960E9479596B
:10DE2000C80102960E9471598A819B81AC81BD8193
:10DE300080934C0990934D09A0934E09B0934F09DC
:10DE4000DF91CF911F910F91FF90EF90DF90CF90D6
:10DE500008952F923F924F925F926F927F928F928E
:10DE60009F92AF92BF92CF92DF92EF92FF920F9369
:10DE70001F93CF93DF93CDB7DEB7E2970FB6F89439
:10DE8000DEBF0FBECDBF7C012A013B0169010E94AC
:10DE9000C5734B015C018701055B1F4FC8010E94E0
:10DEA000C02D18161906A4F00E94C573DC01CB0121
:10DEB00088199909AA09BB09481659066A067B06FA
:10DEC000F0F062E370E080E090E00E949765E6CFBA
:10DED00042E250E0BE016F5F7F4FC8010E94782D83
:10DEE0008981823031F4F8018589968983349105DE
:10DEF00041F0D12CC8010E94C5288D2D93C18FEF10
:10DF000091C16D817E818F8198850E94898B4B01A3
:10DF10005C01F601608371838283938346E050E065
:10DF2000B701685F7F4FCE014D960E948E8F892B7F
:10DF300099F4F70180819181A281B38188169906B5
:10DF4000AA06BB0648F084819581A681B781881511
:10DF50009905AA05BB0528F4C8010E94C52880E0E0
:10DF600061C189899A89AB89BC89F70186879787BE
:10DF7000A08BB18B8EECC82ED12CC8010E94972D9E
:10DF8000F1E0CF1AD108C9F7D12CC7014E963C0158
:10DF9000F701E45AFF4FFAA7E9A740969CA78BA781
:10DFA000F297FEA7EDA7089798AB8FA77097FAABEB
:10DFB000E9AB1701F2E22F0E311C270186E1480E72
:10DFC000511CF801818D928D181619060CF092CF14
:10DFD000C8010E94972D8F30910509F49AC06CF505
:10DFE0008330910509F45EC064F4009751F3019702
:10DFF00009F00CC1C8010E94972D44E050E0B20125
:10E00000B5C08630910509F469C00C9709F0FEC0CF
:10E01000C8010E94972D5C01BB24C50101960E9496
:10E02000CF80F701958B848BA501BC01C8010E94AC
:10E030006D68F7018489958980C08633910509F45C
:10E0400081C07CF48333910509F4C6C0C59709F0FB
:10E05000DDC0C8010E94972DC8010E94972DD82EBF
:10E06000B0CF8B33910509F4A1C08F3F910509F41E
:10E07000A8CFCA9709F0CAC0C8010E94972D44E0F2
:10E0800050E06DA57EA5C8010E94782DF70162A51C
:10E0900073A584A595A50E94898B62A773A784A701
:10E0A00095A78FCFC8010E94972D5C0144E050E0F6
:10E0B00069A97AA9C8010E94782D812C912CBB24D2
:10E0C000F4E0AF1AB1088A149B040CF07ACFC801AF
:10E0D0000E94972D8FEF881A980AF5CFC8010E94E9
:10E0E000972D5C0144E050E0B101C8010E94782DF9
:10E0F000812C912CBB2494E0A91AB1088A149B04AA
:10E100000CF05FCFC8010E94972DEFEF8E1A9E0A88
:10E11000F5CFC8010E94972D5C01BB24C501019673
:10E120000E94CF80F701938B828BA501BC01C801AF
:10E130000E946D68F70182899389FC01EA0DFB1D3D
:10E1400010823FCFC8010E94972DC82EF701868DFF
:10E15000811110C0878D81110DC080A181110AC06D
:10E1600081A1811107C044E050E0B301C8010E94C1
:10E17000782D27CFE9A5FAA580809180A280B38071
:10E18000B301CE0183960E944B758DA19EA1AFA1D4
:10E19000B8A588169906AA06BB0629F3CC2009F46F
:10E1A00010CFC8010E94972DCA94F8CFC8010E94D1
:10E1B000972D44E050E06BA57CA5C8010E94782D06
:10E1C000F70166A577A580A991A90E94898B66A70A
:10E1D00077A780AB91ABF5CEC8010E94972D44E0A4
:10E1E00050E06FA578A9C8010E94782DF70166A1BB
:10E1F00077A180A591A50E94898B66A377A380A7AC
:10E2000091A762AB73AB84AB95ABDBCEC8010E9428
:10E21000972DC82ECC2009F4D4CEC8010E94972D8A
:10E22000CA94F8CFE2960FB6F894DEBF0FBECDBF0A
:10E23000DF91CF911F910F91FF90EF90DF90CF90E2
:10E24000BF90AF909F908F907F906F905F904F9016
:10E250003F902F9008952F923F924F925F926F922E
:10E260007F928F929F92AF92BF92CF92DF92EF9266
:10E27000FF920F931F93CF93DF93CDB7DEB729970C
:10E280000FB6F894DEBF0FBECDBF8C010E943B825B
:10E290002FEC37E040E050E00E94408BDC01CB01E6
:10E2A0000196A11DB11DF80184839583A683B783D0
:10E2B00080839183A283B3835801FBE4AF0EB11C2A
:10E2C000C5010E94086964E470E0C5010E941669F6
:10E2D000882309F42EC10E94C5732B013C01812CB7
:10E2E000912CC801865B9F4F9E838D83180192E419
:10E2F000290E311C48EEC42E43E0D42EE12CF12C23
:10E30000D801DE96B987A887ED81FE8180818330B0
:10E3100009F4FEC0811120C0F80184819581A68195
:10E32000B7810196A11DB11D84839583A683B78310
:10E330000E94C5736419750986099709A70196019A
:10E340000E941E8BA90161E0C8010E940C6D81E052
:10E35000AD81BE818C93C3C08430E9F4F80184811F
:10E360009581A681B7810196A11DB11D84839583F6
:10E37000A683B7830E94C573641975098609970936
:10E38000A70196010E941E8BA90163E0C8010E94AB
:10E390000C6DE2E02AC0813061F5D1014D915D91B3
:10E3A0006D917C919E012F5F3F4FC8010E94296FA4
:10E3B0008F83823009F08DC089819A81AB81BC81C5
:10E3C000F80184839583A683B7830E94C57364197B
:10E3D000750986099709A70196010E941E8BA9015C
:10E3E00063E0C8010E940C6DEF81AD81BE81EC93AA
:10E3F00076C0823009F073C0D1014D915D916D916D
:10E400007C919E012F5F3F4FC8010E94296F8F832F
:10E41000853009F057C083E0ED81FE818083F801EB
:10E4200086A197A1A0A5B1A5892B8A2B8B2B41F49E
:10E4300084E893E0A0E0B0E086A397A3A0A7B1A7EB
:10E44000F80182A593A5A4A5B5A5892B8A2B8B2BB2
:10E4500061F486A197A1A0A5B1A5B695A7959795BA
:10E46000879582A793A7A4A7B5A7D8019E964D919B
:10E470005D916D917C91D1979A968D919D910D9022
:10E48000BC91A02D452B462B472B59F4AC01BD0167
:10E49000440F551F661F771FF80146A757A760ABAB
:10E4A00071ABF80182AB93ABA4ABB5AB86A597A5D6
:10E4B000A0A9B1A986AB97ABA0AFB1AF88248394D4
:10E4C000912C0DC0FF81F63021F4AD81BE811C92EC
:10E4D00006C0BF81BF3F19F4ED81FE811082F1E0DB
:10E4E0008F16910409F410CF0E94C573DC01CB0193
:10E4F00084199509A609B709E885F9852081318134
:10E5000042815381281739074A075B0708F0FCCE80
:10E51000C5010E940869F80184819581A681B781AF
:10E520000196A11DB11D84839583A683B783C40181
:10E5300002C080E090E029960FB6F894DEBF0FBECF
:10E54000CDBFDF91CF911F910F91FF90EF90DF90A2
:10E55000CF90BF90AF909F908F907F906F905F9083
:10E560004F903F902F900895CF92DF92EF92FF92BD
:10E570000F931F93CF93DF936C017A018B01C0E05F
:10E58000D0E0CE15DF0581F0D8016D918D01D60167
:10E59000ED91FC910190F081E02DC6011995892B38
:10E5A00011F02196EECF7E01C701DF91CF911F912F
:10E5B0000F91FF90EF90DF90CF900895FC01538D65
:10E5C000448D252F30E0842F90E0821B930B54174D
:10E5D00010F0CF96089501970895FC01918D828DDA
:10E5E000981761F0828DDF01A80FB11D5D968C91A7
:10E5F000928D9F5F9F73928F90E008958FEF9FEFB2
:10E600000895FC01918D828D981731F0828DE80F6D
:10E61000F11D858D90E008958FEF9FEF0895FC0127
:10E62000918D228D892F90E0805C9F4F821B9109F4
:10E630008F739927089587E098E00E940F7321E077
:10E64000892B09F420E0822F089584EA98E00E9443
:10E650000F7321E0892B09F420E0822F08950E9496
:10E66000678FEF92FF920F931F93CF93DF93EC018D
:10E6700081E0888F9B8D8C8D981305C0E889F9897E
:10E68000808185FD26C0F62E0B8D10E00F5F1F4F99
:10E690000F731127E02E8C8DE8120CC00FB607FC0B
:10E6A000FACFE889F989808185FFF5CFCE010E94F4
:10E6B000787AF1CF8B8DFE01E80FF11DE35AFF4F01
:10E6C000F0829FB7F8940B8FEA89FB898081806282
:10E6D0000AC09FB7F894EE89FF896083E889F989B9
:10E6E00080818370806480839FBF81E090E0DF91B0
:10E6F000CF911F910F91FF90EF900895CF93DF93EB
:10E70000EC01888D8823C9F0EA89FB89808185FD29
:10E7100005C0A889B9898C9186FD0FC00FB607FC8A
:10E72000F5CF808185FFF2CFA889B9898C9185FFCB
:10E73000EDCFCE010E94787AE7CFDF91CF91089597
:10E740003FB7F8948091AE0B9091AF0BA091B00BB6
:10E75000B091B10B26B5A89B05C02F3F19F00196CB
:10E76000A11DB11D3FBFBA2FA92F982F8827820F57
:10E77000911DA11DB11DBC01CD0142E0660F771FA7
:10E78000881F991F4A95D1F708952FB7F894609183
:10E79000AA0B7091AB0B8091AC0B9091AD0B2FBF7E
:10E7A00008951F920F920FB60F9211242F933F934B
:10E7B0008F939F93AF93BF938091AA0B9091AB0BD4
:10E7C000A091AC0BB091AD0B3091A90B23E0230FBE
:10E7D0002D3720F40196A11DB11D05C026E8230F99
:10E7E0000296A11DB11D2093A90B8093AA0B9093B3
:10E7F000AB0BA093AC0BB093AD0B8091AE0B909193
:10E80000AF0BA091B00BB091B10B0196A11DB11D42
:10E810008093AE0B9093AF0BA093B00BB093B10B62
:10E82000BF91AF919F918F913F912F910F900FBE0C
:10E830000F901F901895DC01ED91FC910190F081F3
:10E84000E02D1994EF92FF920F931F93CF93DF93D4
:10E850008C017B01C0E0D0E0F701EC0FFD1F64915B
:10E86000662361F0D801ED91FC910190F081E02DDB
:10E87000C8011995892B11F02196EECFCE01DF91B9
:10E88000CF911F910F91FF90EF9008956115710541
:10E8900079F0FB0101900020E9F73197AF01461BA9
:10E8A000570BDC01ED91FC910280F381E02D19946E
:10E8B00080E090E008958F929F92AF92BF92EF9286
:10E8C000FF920F931F93CF93DF93CDB7DEB7A1973E
:10E8D0000FB6F894DEBF0FBECDBF7C01FA01CB01AD
:10E8E00019A2223008F42AE08E010F5D1F4F822EFC
:10E8F000912CA12CB12CBF01A50194010E941E8B6B
:10E90000F901CA01015011096A3014F4605D01C0B7
:10E91000695CD8016C93232B242B252B61F7B8015C
:10E92000C7010E944674A1960FB6F894DEBF0FBED1
:10E93000CDBFDF91CF911F910F91FF90EF90BF90CE
:10E94000AF909F908F900895CF92DF92EF92FF92B9
:10E950000F931F93CF93DF932115310581F4DC01D1
:10E96000ED91FC910190F081E02D642FDF91CF912A
:10E970001F910F91FF90EF90DF90CF9019942A3064
:10E98000310501F577FF1DC06A017B01EC016DE2E5
:10E990000E941B748C0144275527BA014C195D094C
:10E9A0006E097F092AE0CE010E945B74800F911FDF
:10E9B000DF91CF911F910F91FF90EF90DF90CF905B
:10E9C00008952AE0DF91CF911F910F91FF90EF9072
:10E9D000DF90CF900C945B749A01AB01770F660BBC
:10E9E000770B0C94A4749A01452B39F4DC01ED915A
:10E9F000FC910190F081E02D1994462F50E060E0E9
:10EA000070E00C945B748F929F92AF92BF92CF9202
:10EA1000DF92EF92FF920F931F93CF93DF937C01CE
:10EA20008B014C0182E0880E911C5701E5E0AE0E8F
:10EA3000B11CC0E0D0E0F40161914F014AE050E028
:10EA4000C8010E94F3746C016EE2C8010E941B743D
:10EA50008C0D9D1DC80FD91F8A149B0461F74AE0D5
:10EA600050E0F7016581C8010E94F3748C0F9D1F6F
:10EA7000DF91CF911F910F91FF90EF90DF90CF909A
:10EA8000BF90AF909F908F90089567E376E00C94CD
:10EA900046740C944674DC0186EC93E08D939D9350
:10EAA00084E0FB0101900D928A95E1F708951F9291
:10EAB0000F920FB60F9211240BB60F922F933F9324
:10EAC0004F935F936F937F938F939F93AF93BF9376
:10EAD000EF93FF9387E098E00E94787AFF91EF919F
:10EAE000BF91AF919F918F917F916F915F914F9166
:10EAF0003F912F910F900BBE0F900FBE0F901F9064
:10EB000018951F920F920FB60F9211240BB60F9209
:10EB10002F938F939F93EF93FF93E0911708F091BA
:10EB200018088081E0911D08F0911E0882FD12C036
:10EB30009081809120088F5F8F7320912108821728
:10EB400051F0E0912008F0E0E95FF74F958F809356
:10EB5000200801C08081FF91EF919F918F912F91AB
:10EB60000F900BBE0F900FBE0F901F9018951F9225
:10EB70000F920FB60F9211240BB60F922F933F9363
:10EB80004F935F936F937F938F939F93AF93BF93B5
:10EB9000EF93FF9384EA98E00E94787AFF91EF91D7
:10EBA000BF91AF919F918F917F916F915F914F91A5
:10EBB0003F912F910F900BBE0F900FBE0F901F90A3
:10EBC00018951F920F920FB60F9211240BB60F9249
:10EBD0002F938F939F93EF93FF93E091B408F0915D
:10EBE000B5088081E091BA08F091BB0882FD12C09F
:10EBF00090818091BD088F5F8F732091BE0882172E
:10EC000051F0E091BD08F0E0EC55F74F958F8093FF
:10EC1000BD0801C08081FF91EF919F918F912F914D
:10EC20000F900BBE0F900FBE0F901F9018950C9475
:10EC3000FC5463EE73E184EA98E00E942274E0E001
:10EC4000F0E01994CF93C1E068EE73E080E090E0CB
:10EC50000E9497654AE050E06C2F84EA98E00E9499
:10EC6000F374CF5FC43181F7CF9108950F931F9351
:10EC7000CF93DF9300D000D0CDB7DEB70E94AE4C6B
:10EC80006CE372E184EA98E00E94227406EC13E0DF
:10EC90001A8309831B821C821D821E82CE01039669
:10ECA0000E94063ECE0101960E94B03D1A83098360
:10ECB0001B821C821D821E8224E030E0AE014D5F6B
:10ECC0005F4F60E081E090E00E94162CCE0101963B
:10ECD0000E94B03D1A8309831B821C821D821E8202
:10ECE00024E030E0AE014D5F5F4F60E085E090E0F2
:10ECF0000E94162CCE0101960E94B03D62E672E1A0
:10ED000084EA98E00E94227426960FB6F894DEBF3B
:10ED10000FBECDBFDF91CF911F910F9108959F92AC
:10ED2000AF92BF92CF92DF92EF92FF920F931F9319
:10ED3000CF93DF93CDB7DEB769970FB6F894DEBFF8
:10ED40000FBECDBF2091880730918907211531056D
:10ED500009F4D7C290916E079F5F90936E076AE3A4
:10ED600076E0C9010E940B3F9093BB0B8093BA0BD6
:10ED7000009709F4A9C00E948A3F082F10E00115EE
:10ED8000110509F4A1C0000F111F000F111F809180
:10ED9000B30B9091B40B892B09F085C0C8010E9478
:10EDA000CF809093B40B8093B30B1092CA0B109248
:10EDB000C90B1092BD0B1092BC0B1092C80B109295
:10EDC000CC0B1092CB0B7801013082E018071CF0BD
:10EDD000E12C22E0F22EC70101960E94CF80909391
:10EDE000CE0B8093CD0B9093C70B8093C60B8E0DEB
:10EDF0009F1D9093C10B8093C00B0E94C5736093BD
:10EE0000C20B7093C30B8093C40B9093C50B80E02F
:10EE100090E0E091CD0BF091CE0BE80FF91F10823E
:10EE20000196E816F906ACF782E090E09093CA0BE1
:10EE30008093C90B80E98093C9001092C80010929A
:10EE4000CD0083E08093CC008EE08093CA00F092E6
:10EE50000902E09208022091CD0B3091CE0B8091F7
:10EE6000080290910902820F931F9093C10B809327
:10EE7000C00B232B09F453C16CE074E184EA98E0E1
:10EE80000E9422744AE050E0B80184EA98E00E94AF
:10EE9000EC7484EA98E00E94457588E99FE19093BC
:10EEA000BF0B8093BE0B6FE774E184EA98E00E9489
:10EEB00022744AE050E0B80184EA98E00E94EC74C1
:10EEC00084EA98E00E94457560E476E080918807C6
:10EED000909189070E940B3F8C010097B1F00E942E
:10EEE0008A3F811123C111C063E674E184EA98E08E
:10EEF0000E9422744AE050E0B60184EA98E00E9441
:10EF0000EC7484EA98E00E944575E0908807F090E0
:10EF1000890764E476E0C7010E940B3F9093B90B28
:10EF20008093B80B6BE476E0C7010E940B3F8C0125
:10EF30009093700780936F0761E576E0C7010E94A8
:10EF40000B3F90938D0780938C0710927F07109250
:10EF50007E070115110501F1D8011696ED90FC9080
:10EF6000179700916F07109170070115110569F04F
:10EF7000E114F10451F0F70180858530B1F7C70144
:10EF80000E948A3F823088F301C1F801868197810F
:10EF900090937F0780937E07E0908807F090890721
:10EFA0006DE376E0C7010E940B3F8C0190937307DD
:10EFB0008093720768E576E0C7010E940B3F90934B
:10EFC000B70B8093B60B0115110509F443C080916E
:10EFD0006E078F5F80936E07D80116960D911C9176
:10EFE00017970115110589F1F8018085863039F5EB
:10EFF0001A830983CE0101960E94D6268C8188232C
:10F00000F1F0ED81FE813097D1F0809188079091E9
:10F010008907892BA1F010821182128213828B81C1
:10F02000843008F002C1823008F006C162E08C81B1
:10F030000E947364ED81FE818181807F8183D8018C
:10F0400012960D911C911397CCCF80916E07815031
:10F0500080936E076EE374E184EA98E00E94227464
:10F0600066E374E184EA98E00E94227481E02091D2
:10F070006F0730917007232B09F480E00E94F15450
:10F080006DE274E184EA98E00E94227481E02091AC
:10F09000720730917307232B09F480E00E94F1542A
:10F0A00064E274E184EA98E00E94227481E0209195
:10F0B000B80B3091B90B232B09F480E00E94F15476
:10F0C0006DE174E184EA98E00E94227481E020916D
:10F0D000B60B3091B70B232B09F480E00E94F1545A
:10F0E00084EA98E00E9445750E94105D6B017C01E6
:10F0F00068E174E184EA98E00E9422742AE0B70192
:10F10000A60184EA98E00E945B7484EA98E00E9479
:10F11000457580916E07815080936E07F2C065EF50
:10F1200073E184EA98E00E942274B3CE6FEF680F17
:10F13000C8010E94263FFC01C184D284E384F48488
:10F1400090918E07992359F0809170008E7F809363
:10F15000700010928E07109202021092010282E15A
:10F160008093000291110E940F5A5601C6010E941D
:10F17000375A01E010E0A016B1060CF4B5CE60E0FD
:10F18000C8010E946D5A0F5F1F4FF5CFB701CE0126
:10F1900001960E94E446CE0101960E943B238823FB
:10F1A000D1F18C859D850097E1F0DC01ED91FC911A
:10F1B0000484F585E02D1995892B49F08C859D8572
:10F1C000DC01ED91FC910284F385E02D19958C858D
:10F1D0009D85DC01ED91FC910680F781E02D19956C
:10F1E0001AC060E070E0CE0101960E949A238C0163
:10F1F00097FF84C0119501951109AA24A394B12CFD
:10F20000CE0101960E947824C82ED12C8B858530A2
:10F21000D1F08630E9F1D7011296ED90FC9013976A
:10F22000CE0101960E9497409CCE803439F0823402
:10F2300009F005CF60E003C060E0F9CE62E08C81A8
:10F240000E947364FCCECD2829F462E0CE010196C1
:10F250000E944D2461E0802F0E94736460E0802F43
:10F260000E9444646BE574E184EA98E00E94227491
:10F270004AE050E0B80184EA98E00E94EC7466E548
:10F2800074E184EA98E00E94227464E574E131C07C
:10F29000902E61E0802F0E94736461E0AB2821F022
:10F2A000CA94CD2829F403C0CA94CD2809F060E09F
:10F2B000C62ED12C892D0E9444646FE474E184EA47
:10F2C00098E00E9422744AE050E0B80184EA98E095
:10F2D0000E94EC746DE474E184EA98E00E94227468
:10F2E0004AE050E0B60184EA98E00E94EC746BE4D6
:10F2F00074E184EA98E00E9422748DCFA12CB12C95
:10F300007FCF69960FB6F894DEBF0FBECDBFDF91F9
:10F31000CF911F910F91FF90EF90DF90CF90BF9012
:10F32000AF909F900895009779F0FC0120852530DB
:10F3300059F40E94263F009739F0FC0120852430C3
:10F3400019F481859285089580E090E0089580E029
:10F3500090E0892B21F00E942573811121C080E06B
:10F3600090E0892B41F080E090E0892B21F00E9411
:10F370000000811118C080E090E0892B21F00E94EC
:10F380001B73811113C080E090E0892BA1F080E015
:10F3900090E0892B81F00E94000081110AC008953D
:10F3A0000E940000DCCF0E940000E5CF0E94000018
:10F3B000EACF0C9400000895CF93DF93EC01E8812D
:10F3C000F9810284F385E02DCE0119950196B9F7F4
:10F3D000DF91CF910895EF92FF920F931F93CF93F8
:10F3E000DF93EC018B017A010E94C573FE01E8579F
:10F3F000FF4F60837183828393838C819D81DC01C5
:10F40000ED91FC910280F381E02DA701B801DF911D
:10F41000CF911F910F91FF90EF9019941F93CF936D
:10F42000DF93EC01162F0E94C573FE01E857FF4FD2
:10F4300060837183828393838C819D81DC01ED9154
:10F44000FC910190F081E02D612FDF91CF911F9110
:10F4500019940F931F93CF93DF93EC018B016DE50C
:10F4600076E00E94497501151105B9F1F801619125
:10F470008F01662391F1603220F0623211F06C3519
:10F4800041F56CE5CE010E941B74F8013197808133
:10F490008C30D1F044F48930D9F08A30B9F088301A
:10F4A00029F762E616C0823259F024F48D30F1F665
:10F4B00062E70FC08F3231F08C35C1F66CE509C0C0
:10F4C00062E207C06FE205C066E603C06EE601C0F7
:10F4D00064E7CE010E941B74C9CF62E2CE010E9494
:10F4E0001B7480E090E0DF91CF911F910F91089500
:10F4F000FC01848DDF01A80FB11DA35ABF4F2C91D1
:10F50000848D90E001968F739927848FA689B7899F
:10F510002C93A089B1898C91837080648C93938D96
:10F52000848D981306C00288F389E02D80818F7D39
:10F53000808308951F920F920FB60F9211240BB67D
:10F540000F922F933F934F935F938F939F93EF93DC
:10F55000FF932091CD0B3091CE0B8091CB0B9091EE
:10F56000CC0BAC014F5F5F4F5093CC0B4093CB0B58
:10F57000F901E80FF91F80818093CE008091080285
:10F58000909109022091CB0B3091CC0B82179307FD
:10F5900048F48FEF9FEF9093CC0B8093CB0B88E4D4
:10F5A0008093C900FF91EF919F918F915F914F914F
:10F5B0003F912F910F900BBE0F900FBE0F901F9099
:10F5C00018951F920F920FB60F9211242F933F930D
:10F5D0008F939F932091C90B3091CA0B8091CB0BD5
:10F5E0009091CC0B21303105A9F48F3F2FEF92077A
:10F5F00089F41092C8001092CD0089E08093CC006D
:10F6000086E28093CA001092CE001092CC0B10922A
:10F61000CB0B17C0892BA9F41092C8001092CD0013
:10F6200083E08093CC008EE08093CA0088E28093D0
:10F63000C9001092CE0081E090E09093CC0B8093B3
:10F64000CB0B9F918F913F912F910F900FBE0F90F9
:10F650001F9018951F920F920FB60F9211240BB6A0
:10F660000F922F933F934F935F936F937F938F935B
:10F670009F93AF93BF93EF93FF939091C8008091B6
:10F68000CE0094FF08C081E08093C80B8091CD0B21
:10F690009091CE0B57C09091C80B913099F4811185
:10F6A0000EC082E08093C80B0E94C5736093C20BAA
:10F6B0007093C30B8093C40B9093C50B3EC0109204
:10F6C000C80B44C0923009F041C0E091C60BF091E4
:10F6D000C70B9081891721F091E0909307028083F6
:10F6E0002091C60B3091C70B8091C00B9091C10B3C
:10F6F0002817390711F51092C80B8091070288234B
:10F70000D1F08091BE0B9091BF0B892BA1F010928C
:10F71000C900E091BE0BF091BF0B199580E9809371
:10F72000C9001092C8001092CD0083E08093CC00F5
:10F730008EE08093CA00109207028091C60B9091D0
:10F74000C70B01969093C70B8093C60BFF91EF9167
:10F75000BF91AF919F918F917F916F915F914F91E9
:10F760003F912F910F900BBE0F900FBE0F901F90E7
:10F770001895CF92DF92EF92FF920F931F93CF9342
:10F78000DF936C018B0186E090E00E94CF80EC015A
:10F7900090930C0C80930B0CF60101900020E9F77C
:10F7A000CF018C199D090E94CF807C01B6010E9477
:10F7B000DF8FF60101900020E9F73197EC19FD0980
:10F7C000EE0DFF1D1082F982E8821B830A8380916F
:10F7D000A60B9091A70B9D838C83D093A70BC0930E
:10F7E000A60BDF91CF911F910F91FF90EF90DF90CB
:10F7F000CF900895CF92DF92EF92FF920F931F93D5
:10F80000CF93DF93CDB7DEB7EC970FB6F894DEBF9A
:10F810000FBECDBFDC012C91222309F455C064EC4E
:10F8200075E00E9403849A8389837E01B3E0EB0E26
:10F83000F11C01E010E0D02EC12E64EC75E080E0F8
:10F8400090E00E940384F701819391937F010E3130
:10F85000110539F400910B0C10910C0CE980FA8021
:10F8600008C00F5F1F4F892B31F7F4CFF8010481D7
:10F87000158101151105A1F0D8016D917C91C70189
:10F880000E94D68F892B91F7D8011296ED91FC91A9
:10F890001397BE016F5F7F4F8D2D9C2D19950AC068
:10F8A0006DE974E184EA98E00E94227484EA98E0A9
:10F8B0000E94457584EA98E00E94457569E974E103
:10F8C00084EA98E00E942274EC960FB6F894DEBFAA
:10F8D0000FBECDBFDF91CF911F910F91FF90EF90A1
:10F8E000DF90CF900895CF9384EA98E00E940F7341
:10F8F000892BF1F184EA98E00E94ED72C82F8A30DA
:10F9000029F08D3019F0883009F513C0E091A80B6B
:10F91000F0E0E153F44F108267E376E084EA98E088
:10F920000E9449758FEC9BE00E94FA7B1092A80B15
:10F93000DBCF68E084EA98E00E941B748091A80BFA
:10F94000882391F281508093A80BCECF682F84EA50
:10F9500098E00E941B74E091A80BEB3328F681E03D
:10F960008E0F8093A80BF0E0E153F44FC083BCCF1F
:10F97000CF910895FB012481358142815381241761
:10F98000350758F440815181DA01A20FB31F8C93DF
:10F990008481958101969583848380E008958F9278
:10F9A0009F92AF92BF92CF92DF92EF92FF920F930E
:10F9B0001F93CF93DF936115710509F4FFC0FB011D
:10F9C0000085002E000C110B220B330B07301105A4
:10F9D00008F0F4C0DB01EC01F8018827E35DFE4F7D
:10F9E0008F4F0C94818B6CEB74E006C019968C9150
:10F9F000882389F067EC74E0CE01DF91CF911F91ED
:10FA00000F91FF90EF90DF90CF90BF90AF909F90BD
:10FA10008F900C94467461EC74E0EECF19964D9182
:10FA20005D916D917C911C972AE030E0CE01DF91D1
:10FA3000CF911F910F91FF90EF90DF90CF90BF90EB
:10FA4000AF909F908F900C94A4741996CD90DD90F8
:10FA5000ED90FC901C9720E030E0A901C701B601B1
:10FA60000E940C8C87FF09C06FE576E0CE010E94F2
:10FA70004975F7FAF094F7F8F094C701B6010E94BF
:10FA80008A8C4B015C012AE0AB01BC01CE010E94D3
:10FA90005B7468ED75E0CE010E944975C501B40143
:10FAA0000E94B98C9B01AC01C701B6010E949F8BDB
:10FAB0002DEC3CEC4CE45DE30E94A08B20E030E0B8
:10FAC00040E251E40E94708D0E948A8CAB0160E09C
:10FAD00070E02AE0CE010E945B7470C019966D91AF
:10FAE0007C911A97CE01DF91CF911F910F91FF90DA
:10FAF000EF90DF90CF90BF90AF909F908F900C943D
:10FB0000297A16960D911C9117976BE5CE010E94EC
:10FB10001B74019619F48FEF9FEF52C00115110568
:10FB200071F0B801CE010E94CF7C0196A1F3F801DB
:10FB3000028113810115110589F36CE2E7CF6DE5B0
:10FB40002FC016960D911C9117976BE7CE010E945E
:10FB50001B74019601F30115110509F1F80160818B
:10FB60007181CE010E94297A0196A9F26AE3CE0141
:10FB70000E941B74019679F2B801CE010E94CF7CDD
:10FB8000019649F2F801028113810115110519F35B
:10FB90006CE2CE010E941B740196E9F6BCCF6DE7C2
:10FBA000CE010E941B7421E030E0019611F020E0AC
:10FBB00030E088279927821B930B02C080E090E0F9
:10FBC000DF91CF911F910F91FF90EF90DF90CF9039
:10FBD000BF90AF909F908F900895CF93DF93EC01EB
:10FBE000E881F9810284F385E02DCE0119958F3FDC
:10FBF0002FEF920771F0E881F9818132910594F33A
:10FC00000684F785E02D682FCE01199580E090E0FD
:10FC100002C08FEF9FEFDF91CF910895CF92DF92D7
:10FC2000EF92FF92CF93DF93E7E0F8E01382128226
:10FC300088EEC82E83E0D82EE12CF12CC482D58228
:10FC4000E682F78288E393E09183808325ED30E0BC
:10FC50003587248724ED30E03787268720ED30E094
:10FC6000318B208B21ED30E0338B228B22ED30E085
:10FC7000358B248B26ED30E0378B268B118E128E40
:10FC8000138E148EE4EAF8E013821282C482D582C5
:10FC9000E682F7829183808385EC90E09587848764
:10FCA00084EC90E09787868780EC90E0918B808B46
:10FCB00081EC90E0938B828B82EC90E0958B848B2F
:10FCC00086EC90E0978B868B118E128E138E148E9D
:10FCD000EFE1FBE0C6ECD3E0D183C0831282138254
:10FCE00014821582E5E2FBE0D183C0831282138285
:10FCF00014821582EBE2FBE0D183C083128213826F
:10FD000014821582E1E4F9E0D183C0831282138268
:10FD100014821582E1E3FBE0D183C0831282138257
:10FD200014821582E7E4F9E080E5808381E0818335
:10FD3000E7E3FBE0D183C083128213821482158231
:10FD4000EDE3FBE0D183C08312821382148215821B
:10FD5000E3E4FBE0D183C083128213821482158214
:10FD6000EAE4F9E0D183C0831282138214821582FF
:10FD7000138612868AE0848761E0809149090E9497
:10FD80007364E9E4FBE013821282C482D582E682C6
:10FD9000F7828AE493E091838083E5E5FBE0D183F9
:10FDA000C0831282138214821582EBE5FBE0D183BB
:10FDB000C0831282138214821582E1E6FBE0D183B4
:10FDC000C0831282138214821582E7E6FBE0D1839E
:10FDD000C0831282138214821582E2E1FBE0138257
:10FDE0001282C482D582E682F78284EA93E091830C
:10FDF000808388E0848710920D0B10920C0B109278
:10FE00000F0B10920E0B1092110B1092100BA7E516
:10FE1000B9E013961C921E9212978CE593E011960E
:10FE20009C938E93D093EB09C093EA091092EC094E
:10FE30001092ED091092EE091092EF098FEF9FEFEB
:10FE40009093F7098093F6091596FC93EE93149717
:10FE50001092F5091092F409EDE6FBE0D183C0831E
:10FE60001282138214821582E3E7FBE0D183C08300
:10FE70001282138214821582E9E7FBE0D183C083EA
:10FE80001282138214821582EFE7FBE0D183C083D4
:10FE90001282138214821582E5E8FBE0D183C083CD
:10FEA0001282138214821582EBE8FBE0D183C083B7
:10FEB0001282138214821582E1E9FBE080831282B0
:10FEC0001182148613868FEF9FEFDC018783908762
:10FED000A187B287DF91CF91FF90EF90DF90CF9015
:10FEE0000895789484B5826084BD84B5816084BDB2
:10FEF00085B5826085BD85B5816085BD80916E00C8
:10FF0000816080936E0010928100809181008260F8
:10FF10008093810080918100816080938100809135
:10FF200080008160809380008091B1008460809324
:10FF3000B1008091B00081608093B0008091910009
:10FF40008260809391008091910081608093910004
:10FF5000809190008160809390008091A1008260E8
:10FF60008093A1008091A10081608093A100809185
:10FF7000A00081608093A000809121018260809325
:10FF800021018091210181608093210180912001D4
:10FF900081608093200180917A00846080937A0050
:10FFA00080917A00826080937A0080917A008160EB
:10FFB00080937A0080917A00806880937A00109212
:10FFC000C1001092A80B1092A70B1092A60B26E06E
:10FFD00040E052EC61E070E084EA98E00E94B744AF
:10FFE00061E172E184EA98E00E94227466E376E7B8
:10FFF00087E096E00E94B97B6EE074E58CE096E0C5
:020000021000EC
:100000000E94B97B67E176E781E196E00E94B97BC7
:1000100061EB77E58CE895E00E94B97B62EF72E5D1
:1000200086E196E00E94B97B62E276E78AE196E09B
:100030000E94B97B6CE474E58FE196E00E94B97B85
:100040006AE573E583E296E00E94B97B60EC72E5B5
:1000500086E296E00E94B97B6DED72E58AE296E059
:100060000E94B97B69E176E780E396E00E94B97B64
:100070000E94AE4C0EE91BE06801F12CC0E0D0E01C
:10008000CE010E94F88AF60181936F0181508E3F64
:1000900010F4FF24F3942196C630D10589F7F110AE
:1000A00029C065E172E184EA98E00E942274C5EFFC
:1000B000D5E040E150E060E070E0CE010E94928225
:1000C000F80161938F016AE370E0CE010E94CB8F4B
:1000D000009751F0FC012081222331F0EC012196A0
:1000E000FBE0043A1F0729F780919E0B8E7F826008
:1000F00080939E0B0E94F52F0E94FC5461E08DE0DE
:100100000E94736426E040E855E260E070E087E01A
:1001100098E00E94B74485E99CE490930D0B80938E
:100120000C0B80E097E490930F0B80930E0B8CEFF9
:1001300096E49093110B8093100B64E170E080E0E3
:1001400090E00E9497658FE29EE29093E909809388
:10015000E80964EF71E080E090E00E949765A8955F
:100160000E94737C0E941E14029714F00E94563C59
:100170000E94422780916F0790917007892B51F060
:1001800080916B0790916C07039711F00E94464D88
:100190000E9417600E9404470E94A779E0CF0F9346
:1001A0001F93CF93DF938230910510F482E090E0AB
:1001B000E091110CF091120C20E030E0A0E0B0E0F2
:1001C000309719F1408151810281138148175907F5
:1001D000C8F08417950769F4109731F012960C93C4
:1001E000129713961C9327C00093110C1093120CB6
:1001F00022C02115310519F04217530718F49A014E
:10020000BD01EF01DF01F801DBCF21153105F9F068
:10021000281B390B2430310580F48A819B816115BC
:10022000710521F0FB019383828304C09093120C2B
:100230008093110CFE01329644C0FE01E20FF31FC1
:100240008193919322503109398328833AC02091B8
:100250000F0C3091100C232B41F420910C023091A3
:100260000D023093100C20930F0C20910A02309154
:100270000B022115310541F42DB73EB740910E0216
:1002800050910F02241B350BE0910F0CF091100CD4
:10029000E217F307A0F42E1B3F0B2817390778F05D
:1002A000AC014E5F5F4F2417350748F04E0F5F1FBC
:1002B0005093100C40930F0C8193919302C0E0E097
:1002C000F0E0CF01DF91CF911F910F910895CF936F
:1002D000DF93009709F481C0FC01329713821282E8
:1002E000A091110CB091120C109781F420813181F2
:1002F000820F931F20910F0C3091100C2817390793
:1003000051F5F093100CE0930F0C67C0ED0120E065
:1003100030E0CE17DF0740F44A815B819E01411532
:100320005105F1F0EA01F5CFD383C28340815181B9
:10033000840F951FC817D90759F488819981840FB4
:10034000951F0296918380838A819B819383828308
:100350002115310529F4F093120CE093110C3DC0E6
:10036000E901FB83EA8349915991C40FD51FEC172A
:10037000FD0761F480819181840F951F0296E90148
:1003800099838883828193819B838A83E0E0F0E074
:1003900012968D919C911397009719F0FD01DC0145
:1003A000F7CF8D919C9111979D012E5F3F4F820F4A
:1003B000931F20910F0C3091100C2817390769F406
:1003C000309729F41092120C1092110C02C0138273
:1003D0001282B093100CA0930F0CDF91CF9108956F
:1003E0008F929F92AF92BF92CF92DF92EF92FF9245
:1003F000CF93DF93EC01688179818A819B816115BC
:1004000071058105910521F464E279ED8BE597E0B2
:100410002DE133EF41E050E00E94408B49015A0149
:100420009B01AC01A7EAB1E40E945F8B6B017C01E8
:10043000ACEEB4EFA50194010E946D8BDC01CB0101
:100440008C0D9D1DAE1DBF1DB7FF03C00197A109F7
:10045000B04888839983AA83BB83BC01CD019F7771
:10046000DF91CF91FF90EF90DF90CF90BF90AF9052
:100470009F908F9008958F929F92AF92BF92CF924C
:10048000DF92EF92FF9260911002709111028091C1
:10049000120290911302611571058105910521F4F5
:1004A00064E279ED8BE597E02DE133EF41E050E038
:1004B0000E94408B49015A019B01AC01A7EAB1E4BB
:1004C0000E945F8B6B017C01ACEEB4EFA50194013F
:1004D0000E946D8BDC01CB018C0D9D1DAE1DBF1DDF
:1004E000B7FF03C00197A109B04880931002909311
:1004F0001102A0931202B0931302BC01CD019F77A9
:10050000FF90EF90DF90CF90BF90AF909F908F9033
:1005100008956093100270931102809312029093D9
:10052000130208953F924F925F926F927F928F9243
:100530009F92AF92BF92CF92DF92EF92FF920F9372
:100540001F93CF93DF935C016B017A0161157105F5
:1005500019F0FB0191838083E114F10429F0C701B4
:100560000297839708F0C9C0E5012196F501108133
:10057000812F90E00E94BD83892B11F05E01F4CFA2
:100580001D3229F42196F501118101E007C01B32CB
:1005900021F4E5012296F501118100E0E114F10456
:1005A000B1F0F0E1EF16F10429F4B0C010E3E1146A
:1005B000F10401F12AE0E216F104B1F180E1E8165C
:1005C000F10471F0E8E0EE16F104F1F413C0103319
:1005D00041F588818F7D883549F71981229602601F
:1005E000F0E1EF2EF12C88248A94982CA82CAFE00F
:1005F000BA2E20C078E0E72EF12C88248A94982C1B
:10060000A82CEFE1BE2E16C06FEF7FEFCB01970154
:100610000F2C000C440B550B0E941E8B49015A01F4
:1006200009C08AE0E82EF12C69E9862E982CA82CC6
:1006300069E1B62E40E060E070E0CB0127010F2CAD
:10064000000C66087708FE0150ED352E310E29E0CA
:10065000231570F42FEB210F2A3118F439EC332EC7
:1006600006C02FE9210F2A3130F529EA322E310E4A
:10067000232D30E02E153F05F4F44F3FC9F08616C8
:100680009706A806B90688F0A30192010E940E8B76
:10069000232D30E040E050E0620F731F841F951F50
:1006A000621773078407950710F44FEF01C041E00C
:1006B00021961081C8CFC114D10451F0442311F008
:1006C000219703C001FF04C02297F601D183C083A4
:1006D00000FF07C090958095709561957F4F8F4F73
:1006E0009F4F4F3F79F482E290E090931A0C8093F1
:1006F000190C3FEF2FEF9FEF0DC040E030E020E0FE
:1007000090E008C0462F372F282F04C0103309F07F
:1007100067CF5FCF642F732F822FDF91CF911F910F
:100720000F91FF90EF90DF90CF90BF90AF909F9090
:100730008F907F906F905F904F903F900895FC0155
:1007400088279927E89421912032E9F3293010F085
:100750002E30C8F32B3241F02D3239F4689404C0A6
:100760000E942E84820F911D219120532A30C0F3C4
:100770001EF4909581959F4F089591110C941A8ABB
:10078000803219F089508550C8F70895FB01DC01CB
:100790008D91059080190110D9F3990B0895FB01F3
:1007A000DC0105900D920020E1F70895FB01DC01CA
:1007B0000D900020E9F711974150504028F0059026
:1007C00000200D92C9F708951C920895FB01DC01E9
:1007D0004150504030F08D910590801919F400205F
:1007E000B9F7881B990B0895FB01DC01415050407B
:1007F00048F005900D920020C9F701C01D924150AC
:100800005040E0F708954DE05CE00C940784FA0155
:10081000A191B081009719F41097E1F0CD01DC01AE
:10082000CD010D90002011F4C00113C0FB012191F6
:10083000222319F02015D9F7F3CFFB0121912015C0
:1008400019F41E92119606C02223C1F70D900020C4
:10085000A1F7D001FA01A193B08308957AE0979FA0
:10086000902D879F802D910D11240895FC012381E7
:1008700027FF10C0E3E1FCE020813181821793075C
:1008800011F41182108232962CE0E931F207A1F7BF
:100890000E94678180E090E008950F931F93CF93AB
:1008A000DF93009731F46115710519F480E090E051
:1008B0003AC08B01EC016EE070E081E090E00E94B4
:1008C000FE89FC01892B91F380E8838301151105D2
:1008D00071F01387028781E883838091130C9091D4
:1008E000140C892B21F4F093140CE093130C209733
:1008F000C9F0D187C0878381826083838091150C82
:100900009091160C892B71F4F093160CE093150C52
:100910008091170C9091180C892B21F4F093180CEE
:10092000E093170CCF01DF91CF911F910F910895A4
:10093000CF93DF93EC012B8120FF33C026FF0AC049
:100940002F7B2B838E819F8101969F838E838A814B
:1009500090E029C022FF0FC0E881F9818081082E34
:10096000000C990B009719F420622B831AC0319662
:10097000F983E8830EC0EA85FB85199597FF09C0C6
:100980002B81019611F080E201C080E1822B8B83E4
:1009900008C02E813F812F5F3F4F3F832E839927D1
:1009A00002C08FEF9FEFDF91CF9108950F931F93B8
:1009B000CF93DF93CDB7DEB708851985F801838122
:1009C00088608383AE01445F5F4F6A857B85C80181
:1009D0000E941085F8012381277F2383DF91CF9127
:1009E0001F910F9108950F931F93CF93DF93CDB76E
:1009F000DEB708851985F801838188608383AE019D
:100A0000445F5F4F6A857B85C8010E94D988F801E1
:100A10002381277F2383DF91CF911F910F91089529
:100A20002F923F924F925F926F927F928F929F92FE
:100A3000AF92BF92CF92DF92EF92FF920F931F93EC
:100A4000CF93DF93CDB7DEB72B970FB6F894DEBF09
:100A50000FBECDBF6C017B018A01FC01178216829B
:100A6000838181FFCCC1CE0101963C01F6019381C7
:100A7000F70193FD859193FF81917F01882309F40C
:100A8000BAC1853239F493FD859193FF81917F013D
:100A9000853229F4B60190E00E94458AE7CF912C77
:100AA000212C312CFFE1F315D8F08B3279F038F49A
:100AB000803279F08332A1F4232D20611DC08D3264
:100AC00061F0803369F4232D216016C0832D82608C
:100AD000382EE32DE4603E2E2AC0F32DF8601DC0B1
:100AE00037FC2DC020ED280F2A3040F08E32B9F4AB
:100AF00036FC81C1232D2064322E19C036FE06C07B
:100B00008AE0989E200D1124922E11C0EAE02E9EBC
:100B1000200D1124222EF32DF0623F2E08C08C36BA
:100B200021F4832D8068382E02C0883641F4F70105
:100B300093FD859193FF81917F018111B3CF982F10
:100B40009F7D9554933028F40C5F1F4F9FE399834A
:100B50000DC0833631F0833771F0833509F059C009
:100B600021C0F801808189830E5F1F4F8824839400
:100B7000912C530113C02801F2E04F0E511CF801D3
:100B8000A080B18036FE03C0692D70E002C06FEF17
:100B90007FEFC5010E943A8A4C018201F32DFF7755
:100BA0003F2E16C0280122E0420E511CF801A08001
:100BB000B18036FE03C0692D70E002C06FEF7FEF99
:100BC000C5010E94288A4C01F32DF0683F2E820156
:100BD00033FC1BC0822D90E088169906B0F4B60154
:100BE00080E290E00E94458A2A94F4CFF50137FC18
:100BF000859137FE81915F01B60190E00E94458AA0
:100C000021102A9421E0821A91088114910471F72D
:100C1000E8C0843611F0893641F5F80137FE07C087
:100C200060817181828193810C5F1F4F08C0608158
:100C30007181072E000C880B990B0E5F1F4FF32D4F
:100C4000FF763F2E97FF09C090958095709561952E
:100C50007F4F8F4F9F4FF0683F2E2AE030E0A30177
:100C60000E949A8A882E861845C0853731F4232D34
:100C70002F7EB22E2AE030E025C0932D997FB92E29
:100C80008F36C1F018F4883579F0B5C0803719F087
:100C9000883721F0B0C0E92FE061BE2EB4FE0DC050
:100CA000FB2DF460BF2E09C034FE0AC0292F266038
:100CB000B22E06C028E030E005C020E130E002C0DE
:100CC00020E132E0F801B7FE07C0608171818281C6
:100CD00093810C5F1F4F06C06081718180E090E0BE
:100CE0000E5F1F4FA3010E949A8A882E8618FB2D43
:100CF000FF773F2E36FE0DC0232D2E7FA22E8914A6
:100D000058F434FE0BC032FC09C0832D8E7EA82E11
:100D100005C0B82CA32C03C0B82C01C0B92CA4FE6C
:100D20000FC0FE01E80DF11D8081803321F49A2D62
:100D3000997EA92E09C0A2FE06C0B394B39404C044
:100D40008A2D867809F0B394A3FC11C0A0FE06C0DA
:100D5000B21488F4280C922C9B180EC0B21460F4C4
:100D6000B60180E290E00E94458AB394F7CFB214B6
:100D700018F42B1802C0982C212CA4FE10C0B60128
:100D800080E390E00E94458AA2FE17C0A1FC03C048
:100D900088E790E002C088E590E0B6010CC08A2D9B
:100DA000867859F0A1FE02C08BE201C080E2A7FC68
:100DB0008DE2B60190E00E94458A891438F4B601AC
:100DC00080E390E00E94458A9A94F7CF8A94F301D9
:100DD000E80DF11D8081B60190E00E94458A8110E6
:100DE000F5CF222009F442CEB60180E290E00E94C5
:100DF000458A2A94F6CFF6018681978102C08FEF4B
:100E00009FEF2B960FB6F894DEBF0FBECDBFDF91DC
:100E1000CF911F910F91FF90EF90DF90CF90BF90F7
:100E2000AF909F908F907F906F905F904F903F908A
:100E30002F90089520FD09C0FC0123FD05C022FF6D
:100E400002C07383628351834083089544FD17C0B9
:100E500046FD17C0AB01BC01DA01FB01AA0FBB1FA5
:100E6000EE1FFF1F1094D1F74A0F5B1F6E1F7F1FED
:100E7000CB01BA01660F771F881F991F09C033E0A5
:100E800001C034E0660F771F881F991F3150D1F7DA
:100E9000620F711D811D911D08950F931F93CF93B4
:100EA000DF938C01C8010E949884EC0197FD08C073
:100EB0000E94BD83892BB1F7B801CE010E94818ABF
:100EC000CE01DF91CF911F910F9108958F929F9244
:100ED000AF92BF92EF92FF920F931F93CF93DF9346
:100EE0008C01D62F7A01B22E0E9498849C01332760
:100EF0002B32310531F02D32310561F48B2D8068B4
:100F0000B82ED15011F480E068C0C8010E949884C6
:100F100097FDF9CFCB2DCD7F2B2D207309F5803395
:100F2000F9F4AA24AA94AD0E09F443C0C8010E94A2
:100F3000988497FD3EC09C012F7D332728353105CD
:100F400049F4C264D250A9F1C8010E94988497FF65
:100F500007C02FC0B6FE02C0C26001C0C261DA2D58
:100F6000812C912C540120ED280F283080F0C4FFF3
:100F700004C0B8010E94818A19C02A3040F0C6FF1F
:100F8000F8CF2F7D3FEE320F363098F727504C2F99
:100F9000C501B4010E9426874B015C01C260D1509B
:100FA00059F0C8010E94988497FFDDCFC1FD04C0AD
:100FB000AACF812C912C5401C7FF08C0B094A094F3
:100FC00090948094811C911CA11CB11C2C2FB50104
:100FD000A401C7010E941A8781E0DF91CF911F9180
:100FE0000F91FF90EF90BF90AF909F908F900895DA
:100FF0005F926F927F928F929F92AF92BF92CF92A9
:10100000DF92EF92FF920F931F93CF93DF93CDB7B1
:10101000DEB7A0970FB6F894DEBF0FBECDBF5C0160
:10102000962E7A01F9018E010F5F1F4F680180E251
:10103000D8011D928A95E9F7D50113968C9080E02E
:1010400090E0612C712C30E061E070E083FC259130
:1010500083FE21918F01522E211103C080E090E088
:1010600092C02E3511F4009751F1432F50E04817EC
:1010700059073CF42D3559F12D3219F4772009F137
:1010800003C0772009F46AC0452D469546954695DC
:10109000D601A40FB11D452D47708B0102C0000F72
:1010A000111F4A95E2F7A8015C91452B4C936514FA
:1010B00059F0561410F45394E7CF5A94E5CF31E029
:1010C00004C07724739401C0712C0196BFCF7720A0
:1010D00019F08E8180628E83311103C0882483943D
:1010E00017C0F6019E012F5D3F4F8081809581934F
:1010F0002E173F07D1F7F2CFE114F10429F0D70101
:101100008C93F70131967F019A94812C9920F9F004
:10111000C5010E94988497FD18C0FC01FF2723E0B9
:10112000F595E7952A95E1F7EC0DFD1D208130E05E
:10113000AC014770552702C0359527954A95E2F7CF
:1011400020FDDACFB5010E94818A811087CFE1149A
:10115000F10411F0D7011C92C80115C0422F469529
:1011600046954695D601A40FB11D422F47708B01BD
:1011700002C0000F111F4A95E2F7A8015C91452BB0
:101180004C93622EA2CFA0960FB6F894DEBF0FBE8E
:10119000CDBFDF91CF911F910F91FF90EF90DF9026
:1011A000CF90BF90AF909F908F907F906F905F9007
:1011B00008955F926F927F928F929F92AF92BF92AB
:1011C000CF92DF92EF92FF920F931F93CF93DF9313
:1011D0006C01EB015A01FC0117821682512CF601B9
:1011E000E380FE01E3FC8591E3FE8191182FEF017E
:1011F000882309F4EEC090E00E94BD83892B21F082
:10120000C6010E944D87EBCF153241F4FE01E3FC8D
:101210001591E3FE1191EF01153281F4C6010E9490
:10122000988497FDD4C0412F50E09C0133272417A8
:101230003507A9F2B6010E94818ACBC01A3239F46F
:10124000E3FC1591E3FE1191EF0101E001C000E024
:10125000F12C20ED210F2A3080F402606F2D70E018
:1012600080E090E040E20E942687F62EFE01E3FC3B
:101270001591E3FE1191EF01ECCF01FF03C0F110D6
:1012800003C0A7C0FF24FA94183619F01C3651F099
:1012900010C0FE01E3FC1591E3FE1191EF01183639
:1012A00041F408600460FE01E3FC1591E3FE119136
:1012B000EF01112309F48DC0612F70E082E296E006
:1012C0000E941D8A892B09F484C000FD07C0F50126
:1012D00080809180C50102965C0102C0812C912C16
:1012E0001E3651F4F6014681578160E070E0202FF0
:1012F000C4010E941A8773CF1336A9F401FD02C0FE
:10130000FF24F394C6010E94988497FD60C0811465
:10131000910429F0F4018083C40101964C01FA94F0
:10132000F110F0CF50C01B3559F49E01A4016F2D70
:10133000C6010E94F887EC01892B09F044C03EC029
:10134000C6010E944D8797FD42C01F3661F128F407
:10135000143639F1193651F128C0133771F01537A9
:1013600001F123C08114910429F0F4016082C401C9
:1013700001964C01FA94FF2071F0C6010E949884F6
:101380003C0197FD08C00E94BD83892B59F3B6012B
:10139000C3010E94818A81149104A9F0F401108292
:1013A00012C0006203C0006101C00064202FA401CC
:1013B0006F2DC6010E946687811105C0F6018381E9
:1013C000807329F406C000FD0ACF539408CF55203E
:1013D00019F0852D90E002C08FEF9FEFDF91CF9144
:1013E0001F910F91FF90EF90DF90CF90BF90AF9043
:1013F0009F908F907F906F905F9008950F931F93B1
:10140000CF93DF93869F8001879F100D969F100DCD
:101410001124C8010E94CF80EC01009729F0A80197
:1014200060E070E00E94338ACE01DF91CF911F917E
:101430000F910895992788270895FC0105900616B5
:1014400021F00020D9F7C00108953197CF01089508
:10145000FC010590615070400110D8F7809590957F
:101460008E0F9F1F0895DC0101C06D9341505040C5
:10147000E0F70895FC016150704001900110D8F729
:10148000809590958E0F9F1F08950F931F93CF9374
:10149000DF93FB01238121FD03C08FEF9FEF2CC061
:1014A00022FF16C046815781248135814217530798
:1014B00044F4A081B1819D012F5F3F4F3183208390
:1014C0008C93268137812F5F3F4F3783268314C04B
:1014D0008B01EC01FB010084F185E02D1995892B2E
:1014E000E1F6D80116968D919C9117970196179663
:1014F0009C938E931697CE01DF91CF911F910F9100
:101500000895FB01238120FF12C026FD10C08F3FEC
:101510003FEF930761F082832F7D20642383268130
:1015200037812150310937832683992708958FEF1A
:101530009FEF0895FA01AA27283051F1203181F157
:10154000E8946F936E7F6E5F7F4F8F4F9F4FAF4FCB
:10155000B1E03ED0B4E03CD0670F781F891F9A1FDE
:10156000A11D680F791F8A1F911DA11D6A0F711D92
:10157000811D911DA11D20D009F468943F912AE09E
:10158000269F11243019305D3193DEF6CF01089586
:10159000462F4770405D4193B3E00FD0C9F7F6CFB7
:1015A000462F4F70405D4A3318F0495D31FD40527F
:1015B000419302D0A9F7EACFB4E0A6959795879515
:1015C00077956795BA95C9F70097610571050895F4
:1015D0009B01AC010A2E06945795479537952795A0
:1015E000BA95C9F7620F731F841F951FA01D089538
:1015F000F999FECF92BD81BDF89A992780B50895DB
:10160000262FF999FECF1FBA92BD81BD20BD0FB61E
:10161000F894FA9AF99A0FBE01960895DB018F9318
:101620009F930E945F8BBF91AF91A29F800D911DF0
:10163000A39F900DB29F900D11240895A1E21A2E40
:10164000AA1BBB1BFD010DC0AA1FBB1FEE1FFF1F66
:10165000A217B307E407F50720F0A21BB30BE40BB6
:10166000F50B661F771F881F991F1A9469F76095FD
:101670007095809590959B01AC01BD01CF010895B7
:10168000052E97FB1EF400940E94578B57FD07D040
:101690000E941E8B07FC03D04EF40C94578B509580
:1016A0004095309521953F4F4F4F5F4F089590954E
:1016B0008095709561957F4F8F4F9F4F08950E9441
:1016C000728BA59F900DB49F900DA49F800D911DCE
:1016D00011240895B7FF0C945F8B0E945F8B821BCF
:1016E000930B0895A29FB001B39FC001A39F700DFB
:1016F000811D1124911DB29F700D811D1124911D1A
:101700000895EE0FFF1F881F8BBF0790F691E02D05
:1017100019946927962769277827872778270895B6
:101720000E94728B332312F48A1B9B0B0C949A8BAE
:101730000E94728BB7FF0895821B930B0895505837
:10174000BB27AA270E94B78B0C94318D0E94238D52
:1017500038F00E942A8D20F039F49F3F19F426F4C6
:101760000C94208D0EF4E095E7FB0C941A8DE92F74
:101770000E94428D58F3BA176207730784079507D2
:1017800020F079F4A6F50C94648D0EF4E0950B2E00
:10179000BA2FA02D0B01B90190010C01CA01A001C3
:1017A0001124FF27591B99F0593F50F4503E68F11E
:1017B0001A16F040A22F232F342F4427585FF3CF5F
:1017C000469537952795A795F0405395C9F77EF430
:1017D0001F16BA0B620B730B840BBAF09150A1F079
:1017E000FF0FBB1F661F771F881FC2F70EC0BA0FFF
:1017F000621F731F841F48F4879577956795B79587
:10180000F7959E3F08F0B0CF9395880F08F0992781
:10181000EE0F9795879508950E94F68C08F481E065
:1018200008950E94258C0C94318D0E942A8D58F0C9
:101830000E94238D40F029F45F3F29F00C941A8D0B
:1018400051110C94658D0C94208D0E94428D68F38B
:101850009923B1F3552391F3951B550BBB27AA2769
:1018600062177307840738F09F5F5F4F220F331FA3
:10187000441FAA1FA9F335D00E2E3AF0E0E832D06B
:1018800091505040E695001CCAF72BD0FE2F29D06E
:10189000660F771F881FBB1F261737074807AB0740
:1018A000B0E809F0BB0B802DBF01FF2793585F4FB5
:1018B0003AF09E3F510578F00C941A8D0C94658D8A
:1018C0005F3FE4F3983ED4F3869577956795B79597
:1018D000F7959F5FC9F7880F911D9695879597F9A2
:1018E0000895E1E0660F771F881FBB1F621773071B
:1018F0008407BA0720F0621B730B840BBA0BEE1F30
:1019000088F7E09508950E948A8C6894B1110C9430
:10191000658D08950E944A8D88F09F5798F0B92FE1
:101920009927B751B0F0E1F0660F771F881F991F14
:101930001AF0BA95C9F714C0B13091F00E94648DC5
:10194000B1E008950C94648D672F782F8827B85FD5
:1019500039F0B93FCCF3869577956795B395D9F76C
:101960003EF490958095709561957F4F8F4F9F4F76
:101970000895E89409C097FB3EF490958095709582
:1019800061957F4F8F4F9F4F9923A9F0F92F96E9CB
:10199000BB279395F695879577956795B795F11140
:1019A000F8CFFAF4BB0F11F460FF1BC06F5F7F4FDD
:1019B0008F4F9F4F16C0882311F096E911C07723EF
:1019C00021F09EE8872F762F05C0662371F096E8F8
:1019D000862F70E060E02AF09A95660F771F881FC7
:1019E000DAF7880F9695879597F90895990F00086B
:1019F000550FAA0BE0E8FEEF16161706E807F907E1
:101A0000C0F012161306E407F50798F0621B730B7B
:101A1000840B950B39F40A2661F0232B242B252BFC
:101A200021F408950A2609F4A140A6958FEF811D9F
:101A3000811D089597F99F6780E870E060E0089540
:101A40009FEF80EC089500240A94161617061806D6
:101A50000906089500240A941216130614060506B2
:101A60000895092E0394000C11F4882352F0BB0F43
:101A700040F4BF2B11F460FF04C06F5F7F4F8F4FA6
:101A80009F4F089557FD9058440F551F59F05F3FE1
:101A900071F04795880F97FB991F61F09F3F79F090
:101AA00087950895121613061406551FF2CF469512
:101AB000F1DF08C0161617061806991FF1CF869594
:101AC0007105610508940895E894BB276627772778
:101AD000CB0197F908950E94F68C08F48FEF0895D2
:101AE0000E94838D0C94318D0E94238D38F00E94CA
:101AF0002A8D20F0952311F00C941A8D0C94208DD2
:101B000011240C94658D0E94428D70F3959FC1F352
:101B1000950F50E0551F629FF001729FBB27F00D9B
:101B2000B11D639FAA27F00DB11DAA1F649F6627F0
:101B3000B00DA11D661F829F2227B00DA11D621F3F
:101B4000739FB00DA11D621F839FA00D611D221FF9
:101B5000749F3327A00D611D231F849F600D211DDD
:101B6000822F762F6A2F11249F5750409AF0F1F060
:101B700088234AF0EE0FFF1FBB1F661F771F881FC9
:101B800091505040A9F79E3F510580F00C941A8D5A
:101B90000C94658D5F3FE4F3983ED4F3869577957A
:101BA0006795B795F795E7959F5FC1F7FE2B880F6F
:101BB000911D9695879597F90895FA01EE0FFF1FED
:101BC000309621053105A1F16115710561F4803868
:101BD000BFE39B0749F168949038810561F0803834
:101BE000BFEF9B0741F099234AF5FF3FE10531051F
:101BF000210519F1E8940894E795D901AA2329F45D
:101C0000AB2FBE2FF85FD0F310C0FF5F70F4A69526
